:020000040000FA
:107800005469616E59696E673130300000000000C4
:1078100054593230302E3038303030306200000071
:10782000424154333247313339474B3634464200B4
:1078300043414E5F5354440000000000000000002C
:1078400043414E5F43485F300000000000000000ED
:1078500043414E5F3530304B6270730000000000D2
:10786000E8070000E0070000DF070000000000005C
:020000040000FA
:10800000E81E0020DD800000E5800000E780000021
:108010000000000000000000000000000000000060
:10802000000000000000000000000000EF800000E1
:108030000000000000000000F3800000298801001B
:108040005D060100A1060100D10601000107010043
:10805000310701006107010091070100C10701001C
:10806000F10701002108010055080100690801001D
:1080700079080100AD080100BD080100CD0801002C
:1080800001090100450901008D090100D509010020
:108090001D0A0100650A0100750A0100A90A010014
:1080A000DD0A01000D0B0100410B0100750B010001
:1080B000850B0100950B0100C90B0100FD0B0100B0
:1080C000EF3FE8FF0448854600F036F900480047D6
:1080D00091C00100C046C046E81E002016488047F7
:1080E00016480047FEE7FEE7FEE7FEE7FEE7FEE78D
:1080F000FEE7FEE7FEE7FEE7FEE7FEE7FEE7FEE758
:10810000FEE7FEE7FEE7FEE7FEE7FEE7FEE7FEE747
:10811000FEE7FEE7FEE7FEE7FEE7FEE7FEE7FEE737
:10812000FEE7FEE7FEE7FEE7FEE7FEE7FEE7FEE727
:10813000FEE7FEE7FEE70000F58D0100C5800000C8
:1081400030B50B46014600202022012409E00D46EF
:10815000D5409D4205D31D469540491B2546954077
:1081600040191546521E002DF1DC30BD70B50024BB
:108170002546002801DA01244042002901DA0125C0
:108180004942FFF7DDFFAC4200D04042002C00D056
:10819000494270BDF0B51FB40646002082B00546C6
:1081A0004024019100901BE0019922460F46304681
:1081B00000F0B1F8049A059B801A994110D310463B
:1081C0001946224600F097F8361A8F410197224649
:1081D00001200021009F00F08EF838184D410090DA
:1081E0002046641E0028DFDC019B009829463246A9
:1081F00007B0F0BDF0B51FB486B00020009001902C
:1082000002900698069980B204900798090C02041F
:108210000014114307900027089D099806913E46D7
:108220003C4603900398A9B20204000C0390049802
:108230002D0C154348430021224600F05CF8C71975
:10824000714110340E46402CECDB3846029A00F0A7
:1082500052F8009A019B80180090594102980191B0
:10826000103002904028CCDB00980BB0F0BD0346E4
:108270000B439B0703D009E008C9121F08C0042A5A
:10828000FAD203E00B780370401C491C521EF9D24D
:108290007047D2B201E00270401C491EFBD2704709
:1082A0000022F6E710B513460A4604461946FFF7C2
:1082B000F0FF204610BD30B504460020034600E024
:1082C0005B1C934203D2E05CCD5C401BF8D030BD18
:1082D0000321001D401E037812021A43491EF9D5DE
:1082E00010467047034603220870000A491C521EBC
:1082F000FAD51846704710B5202A04DB0146203A0B
:108300009140002010BD914020239C1A0346E34079
:108310001943904010BD10B5202A04DB0846203ACE
:10832000D040002110BD0B46D340D0402024A21ADB
:1083300091400843194610BD064C0125064E05E044
:10834000E36807CC2B430C3C98471034B442F7D376
:10835000FFF7BCFEA4D10100C4D1010070B58C1898
:108360000578401C6B075B0F01D10378401C2A1174
:1083700006D10278401C03E006780E70401C491CB0
:108380005B1EF9D12B0705D40023521E0DD40B70B0
:10839000491CFAE70378401CCB1A921C03E01D78B5
:1083A0000D70491C5B1C521EF9D5A142D8D3002088
:1083B00070BD70B506F0C8FC0524204613F044FEDD
:1083C0000025284606F0B4FC204613F03DFE0126A9
:1083D000304606F089FC204613F036FE284606F0AB
:1083E00083FC204613F030FE304606F0A1FC204608
:1083F00013F02AFE70BDB0B506F0A6FC0524204699
:1084000013F022FE0125284606F092FC204613F0C8
:108410001BFE284606F068FC204613F015FE0020DF
:1084200006F062FC204613F00FFEB0BDF0B581B03F
:1084300006F076FC052013F007FE08270026012031
:1084400006F052FC0524204613F0FEFD204613F0F2
:10845000FBFD06F05BFC0546204613F0F5FD002011
:1084600006F042FC204613F0EFFD76002E437F1EFF
:108470003806E4D1F0B201B0F0BD70B5044600207A
:1084800006F032FC06F060FC052013F0DDFD082646
:10849000E0B2C00906F04CFC0525284613F0D4FDD7
:1084A000012006F021FC284613F0CEFD002006F046
:1084B0001BFC284613F0C8FD284613F0C5FD6400D8
:1084C000761E3006E4D1052013F0BEFD012070BDFC
:1084D000F0B583B0019314460E4607460120384399
:1084E0000290032504E000F08EF86D1E280631D0BE
:1084F00000F067F83846FFF7C0FF00F0A7F8002843
:10850000F1D13046FFF7B9FF00F0A0F80028EAD11A
:1085100000F057F80298FFF7B0FF00F097F8002836
:10852000E1D1019802280BD3451E0026FFF77EFFFC
:108530002070FFF73EFF641C761CF0B28542F5DC2C
:10854000FFF774FF2070FFF756FF00F05CF8202063
:1085500003B0F0BD102003B0F0BDF0B583B01C46F1
:10856000009201910290032504E000F04CF86D1E8A
:10857000280623D000F025F80298FFF77EFF00F0D0
:1085800065F80028F1D10198FFF777FF00F05EF859
:108590000028EAD1002C0CD00026009F3878FFF785
:1085A0006CFF00F053F80028DFD1761C7F1CA64238
:1085B000F4D300F028F8082003B0F0BD102003B079
:1085C000F0BDB0B506F0C0FB0524204613F03CFD1D
:1085D0000125284606F088FB204613F035FD284685
:1085E00006F0A6FB204613F02FFD0025284606F0D6
:1085F0009FFB204613F028FD284606F075FB6420FB
:1086000013F022FDB0BDB0B506F09EFB0524204658
:1086100013F01AFD0025284606F066FB204613F0ED
:1086200013FD284606F084FB204613F00DFD0125BE
:10863000284606F059FB204613F006FD284606F0B2
:1086400077FB642013F000FDB0BD0000B0B506F06C
:1086500067FB0524204613F0F7FC012006F044FBDD
:10866000204613F0F1FC0B4D06F050FB044606F0DB
:1086700035FB002C02D06D1E2804F5D105252846B7
:1086800013F0E2FC002006F02FFB284613F0DCFC80
:108690002046B0BD33210000034801780B2901D8E2
:1086A000491C01707047C046D31A002070B584B0D1
:1086B0000025039502950195009506F00FFB0F200C
:1086C000C6430E4C1036F1B2A0206A461023FFF7C5
:1086D00044FF204613F0B8FC204613F0B5FC912E61
:1086E000F0D3A020B0216A461023FFF736FF2046C2
:1086F00013F0AAFC0248058004B070BD581B0000AE
:10870000C61A002070B5022902D2EB24E0B270BD77
:10871000891EEB250022134605E0401C5B1CDDB2E0
:10872000A94225460EDB04786C40154604E0344629
:108730006E1C072D3546F0D26608E407F7D09A2460
:108740006640F4E7E0B270BDF0B591B00C914178AD
:1087500010AA117083781B025918C3780479240277
:10876000E3181B0459180B0ED3700C0C94700D0AEF
:1087700055700B9108956918099409190A93C9183D
:108780000278D2438918427983791B029A18C379F7
:10879000047A2402E3181B049A188918130A069312
:1087A000C918130C0593C9180792120E0492891860
:1087B000827AC37A1B029A18037B0F90447B2402AF
:1087C000E3181B0498180918020A02928918020C6F
:1087D000019289180D910390000E0E90002003461F
:1087E000014606E032409A40D2B211435B1C082B8E
:1087F0000ED0012635469D400746024602E07F1C0A
:10880000042FEFD010ACE45D2542F8D0521CF6E7FF
:108810000E9C0D980019C3B20F98827B934205D02D
:10882000427A914202D1002011B0F0BD1021FFF731
:1088300069FF0C99CC72019A8A72029A4A72039A61
:108840000A72049ACA71059A8A71069A4A71079A3D
:108850000A710A9ACA70099A8A70089A4A700B9A21
:108860000A7011B0F0BDF0B58DB05522027000272E
:1088700047720B784370CA79059202728A79049222
:10888000C2714A79039282710A7902924271CA7A5C
:10889000089242738A7A019202734E7AC6720C7AF7
:1088A00084720CAA13704D782D02EB188D78C9785C
:1088B000090249190904CB18190E01711D0CC57064
:1088C00009931B0A0B90837038460A91D170079563
:1088D00095700693537031020919089A1202019B90
:1088E000D21812045118089103990902029A8918A2
:1088F000059A1202049BD2181204511805913D46A4
:108900003A4605E02640AE4032436D1C082D0ED09D
:1089100001242146A9400346064602E05B1C042BC5
:10892000F0D00CAFFF5C3942F8D0761CF6E70B9B19
:108930005A72099806994018079940180A994018E0
:10894000059A8018110A4018110C4018110E401891
:10895000089A8018110A4018110C4018110E40187E
:108960005638987310211846FFF7CCFE0DB0F0BDB5
:10897000F0B58FB00446FF20E070A07060700F204B
:10898000C04302900F302070704813F05DFB7049B7
:108990000868632801D8642008606E4F0020388082
:1089A0006D4E0190308008E00B99814222D33888C7
:1089B0001030388080B2A1286DD206F08FF9397856
:1089C000A02003AA1023FFF783FD30802028EED1DA
:1089D00003AD0BA92846FFF7B7FEE97B8842E6D135
:1089E00028785528E3D15D48017800290298DBD129
:1089F0000846D9E73888A0284DD8C0B20021019197
:108A000005E006F06BF93988C8B2A12943D2C1B29A
:108A1000A02003AA1023FFF75BFD308039881031B6
:108A20003980202837D103AD07A92846FFF78CFEEF
:108A3000E97B8842E5D128785528E2D1474800787B
:108A40000028029900D1014607988842D9D24049AE
:108A50000A68962151430B9A824208D9081890421D
:108A600019D30BA90E222046FFF701FCC9E789188C
:108A7000814210D307A90E222046FFF7F8FB0BA86E
:108A80000A99818107980B9008980C9009980D908D
:108A900038880190B5E72078617809020818A17834
:108AA000E2781202511809040818401C24D1002051
:108AB00001903880A020B02103AA1023FFF708FD01
:108AC0003080202818D103AD0BA92846FFF73CFEC3
:108AD000E97B884210D1287855280DD11F480078AD
:108AE000002800D102900B980299884204D20BA969
:108AF0000E222046FFF7BBFB207861780902081898
:108B0000A178E2781202511809040818401C0CD10F
:108B10000020E072A07260722072E071A07160713A
:108B20002071E070A070607020700198388020780B
:108B3000617809020818A178E27812025118090434
:108B400008180749086030880FB0F0BD70110100A7
:108B5000C01A0020C61A0020BC1A0020BF1A00202C
:108B6000CC1A0020F0B581B00091064621480025BE
:108B70000570002A2ED01446C036631B71190F20D1
:108B800008401022101A834200D303461A48027884
:108B9000102A01D0042A1AD1C809FE2707405F2FE6
:108BA00013D80127B8436038C0B29E3282420CD33A
:108BB000009A5219C9B2DFB23B46FFF789FC0F4950
:108BC0000880ED19A542D8D304E0082000E0042075
:108BD0000A490880094801880020042902D0082990
:108BE00000D0012003490870411E8841400001B0B7
:108BF000F0BDC046D21A0020BE1A0020D01A0020B4
:108C00000A4A012313700A4A10700A4A11600A4A7C
:108C100000211160042801D105218901102801D10A
:108C20001D208101054801807047C046BF1A002001
:108C3000BE1A0020C01A0020CC1A0020C41A00203E
:108C4000F0B587B0994D00262E80994B1B688B425A
:108C500024D1994C2188202925D102900092019697
:108C6000964C00272760964D964E2878062809D8FE
:108C700006F034F82068401C2060B042F5D38D48DF
:108C8000042101802F70904C20880107029B31D075
:108C9000884820210180854D019E0BE00120400283
:108CA0008449088006E003A8FFF762FE208081481F
:108CB000802101807F4800883F2807DD874988425E
:108CC0000BDC402812D0802810D010E004280DD0F2
:108CD00008280AD0202809D009E001214A02904240
:108CE00004D0C902884201D001E002262E802888E3
:108CF00007B0F0BDA128019E00D32780009A012A69
:108D00006A4D1ED1187B012856D1DF719F715F71AA
:108D10001F711F73587B012804D1DF729F725F722D
:108D20001F725F7303AF38461946FFF79CFDF87357
:108D30002088002846D01038C1B2A02003AA1023F2
:108D400044E0002AB6D1614801780029B2D002700F
:108D500018785978090208189978DA7812025118A7
:108D6000090408185A490978002901D00F21C9437C
:108D7000884233D2274603AC20461946FFF773FDDD
:108D8000E0733978A02010232246FFF7E6FB029A11
:108D90004849088008288DD13888103038801078EC
:108DA0005178090208189178D278120251180904F2
:108DB0000818484908607DE7597B012911D101282D
:108DC000A3D0A7E7A02003AA10230146FFF7C5FB05
:108DD000384908803D48009901706BE70120C002C6
:108DE0005EE73D480078012812D103AC20461946C1
:108DF000FFF739FDE073A020B02110232246FFF7D2
:108E0000ACFB2C4908800828E4D133480770E1E71F
:108E100018785978090208189978DA7812025118E6
:108E2000090408182B490968214A12685118884218
:108E300003D2204840210180CCE725490978002948
:108E400001D00F21C94388422DD203AF38461946BD
:108E50001C46FFF708FDF8731B480178A02010237B
:108E60003A46FFF77AFB134908800828B2D1164921
:108E70000888103008802078617809020818A178E5
:108E8000E2781202511809040818124908600849CA
:108E90000A6815215143FFF753F900299AD101209F
:108EA0000D49087096E70120C00291E7D81A00200A
:108EB000C01A0020D61A0020BC1A0020DC1A00209C
:108EC000D31A0020818D5B00C61A0020C81A00202A
:108ED000BF1A0020CC1A0020D41A0020FF01000085
:108EE000F0B585B00646434C002727800492101841
:108EF000414A1288904241D201910397404F00208D
:108F0000029038603F4C404D2078052809D805F084
:108F1000E5FE3868401C3860A842F5D33748042184
:108F20000180029820703948018839480278102A57
:108F300001D0042A32D188190346C033049C651A33
:108F40000F2404401020001B854200DB0546DC098D
:108F5000603C01263002E7B27F09052F12D3B443EB
:108F6000E6B29E32B242234C039F0DD301984218C1
:108F7000D9B2EBB23046FFF7F0FA05E01F482021E6
:108F8000018011E01B4C039F1C49088008280BD16D
:108F9000E8B21E4A11880818108005E001208002FE
:108FA00016490880134C039F144800881F2809DDC8
:108FB000202813D001210A0290420FD08902884252
:108FC0000CD00CE0042809D0082808D10F480088EC
:108FD0000499884201D3022700E0012727802088D6
:108FE00002210143022902D1084900220A8005B06A
:108FF000F0BDC046D81A0020C41A0020D61A00209E
:10900000DC1A0020D31A0020818D5B00E01A0020BA
:10901000BE1A0020F0B585B0044600200190042C53
:109020006FD20AF04DFF002801D10AF0C9FF0020DD
:10903000009000BF0098401C00900AF041FF039090
:109040000398002803D0484900988842F2D3039837
:10905000002856D1042145480AF014FF44484549E8
:1090600008802101444A515C4900404A505A414914
:109070000A880121090300F055F9029001200490AB
:1090800020013D4940184078002801D100264BE0DE
:109090002001394940184078012802D13548068816
:1090A00042E0200134494018407802282AD12001AA
:1090B000401805792901304A515C49002B4A505A21
:1090C0002C490A880121090300F02CF906462801E1
:1090D0002A494318280128494018028928014018C4
:1090E0000021C7683046B84706462801224BC01801
:1090F000C2882801C0188178304600F087F80646FB
:1091000012E02DE020011C4940184078032804D0CB
:10911000200140184078132804D120011649401836
:10912000868801E0002004900498002818D02001CF
:1091300012494318200110494018028920014018A3
:109140003146C7680298B847019020010A4BC01801
:10915000C2882001C0188178019800F057F801906A
:10916000019805B0F0BD000050C30000BE00002013
:1091700088130000B800002090C80100D0C801008A
:10918000F8B505460E4614460020009001211C4803
:1091900001751C48007888431A4908700846807891
:1091A0000821084317498870002088710846007814
:1091B000012108431349087008460572002717E08B
:1091C00010480078802108430E49087000BF0E48FF
:1091D000007D0028FBD000200B4908750948C08994
:1091E0002080A41C0748C1890098081800907F1CA3
:1091F000B742E5D331460098FEF7A2FF80B2F8BD32
:1092000040610040005004404060004010B50346FB
:10921000012908D1094CA41A9C4202D99C18A0B279
:109220000BE0064809E0022906D1934202DD9C1AB0
:10923000A0B202E0002000E0184610BDFFFF0000D1
:1092400010B504460121202001F0B2FF0020324970
:109250000870012131480175002031490875152039
:1092600012F0DAFB2C488078E17808432A498870AC
:10927000084680782178084327498870207880281C
:1092800006D108460079E17949000843224908716E
:1092900021488078E17A08431F498870A078002827
:1092A00003D10846007908710FE0A078012806D1A3
:1092B00019480079602108431749087105E01648EC
:1092C0000079802108431449087113488079217975
:1092D00008431149887108468079617908430E492D
:1092E0008871207AC872607A8872084600783821BE
:1092F000884309490870084600786178C900084326
:1093000005490870A07A08730846007801210843CF
:109310000149087010BD0000005004404061004049
:1093200040600040F8B504460E461746002E01D1B5
:1093300000250FE0A64201DC3D460BE00094009CB6
:1093400020467843009031460098FEF7F9FE0090E1
:10935000009885B22846F8BD0146042904D28A0047
:10936000024BD218508800E000207047E41400201F
:109370000146042903D28A00024B985C00E00020D9
:1093800070470000E4140020FFB587B00446089839
:10939000844203DA0A988068002802D124480190A8
:1093A00042E00898001B82B20292002625460A98E5
:1093B000806800212F463A46334604960591069070
:1093C000FEF718FF05460E46002328463146029A4E
:1093D000FEF7E0FE05460E46304600210A464940AB
:1093E0005040014302D0124801901DE003950A98B5
:1093F000C068039DA84202D30020019014E00A989F
:10940000C1680398401A039009990398FEF798FEE3
:1094100003900398000C0004002802D00448019037
:1094200002E0039880B2019001980BB0F0BD0000FB
:10943000FFFF000010B508480078802188430649E6
:10944000087001210548017500200549087515209F
:1094500012F0E2FA10BD00000050044040610040EC
:1094600040600040F8B505460E4614461F462146AA
:109470002846FEF77BFE80B2F8BD0000FFB587B03E
:1094800006460A984068002801D1029035E00A9803
:1094900001684068081803900025344600212746DB
:1094A000039806950491059038462946049B059A31
:1094B000FEF7A0FE04460D460A98406802460023C7
:1094C000019020462946FEF765FE04460D4600231E
:1094D00020462946099AFEF75DFE04460D462846B9
:1094E00007492140002359405840014303D0044814
:1094F000C043029001E0A0B2029002980BB0F0BD10
:109500000000FFFF10B5FE4800688079030012F0EC
:1095100069FA07059ED8F5F4F3F2F100F8480068FF
:109520004079030012F05EFA0805138A2A8A468AF7
:10953000638A0FF0B1F80020F1490968C873F04858
:1095400000684079401CEE49096848717DE0ED49AA
:109550004969EB4A1268D27A885C0FF015F9E8483D
:1095600000684079401CE64909684871E448006891
:109570004079401CE2490968487166E009F010FA38
:10958000002810D10FF000F9DD4800684079401C38
:10959000DB4909684871DA4800684079401CD849BD
:1095A0000968487105E00FF0A1F80020D449096866
:1095B00048714AE009F0F4F9002811D111200FF0A8
:1095C000E3F8CF4800684079401CCD4909684871EC
:1095D000CB4800684079401CC9490968487105E0DA
:1095E0000FF084F80020C649096848712DE009F0A1
:1095F000D7F900281BD1C2480068C07A401CC04976
:109600000968C872BE480068C07ABE4909788842B5
:109610000DDB0020BA490968C872B9490968486277
:10962000B74800688079401CB549096888710FF017
:109630005DF80020B2490968487106E00FF056F85D
:109640000020AF490968487100BF00BF32E3AC4851
:109650000068407C002817D0AA48C068002803D0C2
:10966000A848C168192088470020A54909684862B0
:10967000A34800688079401CA149096888710020CE
:109680009F49096848711BE09D480068406A282886
:1096900007D29B480068406A401C994909684862A3
:1096A0000EE0002096490968486295480068807974
:1096B000401C9349096888710020914909684871E4
:1096C000F8E28F4800684079030012F08BF9080532
:1096D00018A42FA44CA480A40EF0DEFF002088491B
:1096E0000968C873864800684079401C8449096845
:1096F000487197E0D4E2C7E230E25DE194E081494D
:1097000049697F4A1268D27A885C0FF03DF87C483C
:1097100000684079401C7A490968487178480068B7
:109720004079401C7649096848717BE009F038F9B6
:10973000002811D101200FF027F871480068407906
:10974000401C6F49096848716D4800684079401CA9
:109750006B490968487105E00EF0C8FF00206849B0
:10976000096848715EE009F01BF9002828D16449B6
:109770000968C97A24225143634A12688918604AE9
:109780001268D27B885C0EF0FFFF5D480068C07BEA
:10979000401C5B490968C87359480068C07B24288D
:1097A00014D3574800684079401C554909684871EE
:1097B000534800684079401C51490968487105E0E8
:1097C0000EF094FF00204E49096848712AE009F024
:1097D000E7F8002818D14A480068C07A401C484978
:1097E0000968C87246480068C07A464909788842C4
:1097F0000ADB002042490968C87241480068807944
:10980000401C3F49096888710EF070FF00203C49F8
:109810000968487106E00EF069FF002038490968C0
:10982000487100BF00BF45E2354800684079030039
:1098300012F0D8F80A0614B92BB948B978B995B915
:109840000EF02AFF00202E490968C8732C480068D2
:109850004079401C2A4909684871ABE029494969A7
:10986000274A1268D27A885C0EF08EFF244800687E
:109870004079401C224909684871214800684079B4
:10988000401C1F490968487194E009F089F80028D4
:1098900011D14A200EF078FF194800684079401C29
:1098A000174909684871164800684079401C1449F6
:1098B0000968487105E00EF019FF00201049096899
:1098C000487177E009F06CF8002824D1FF200EF0F1
:1098D0005BFF0B480068C07B401C09490968C873DE
:1098E00007480068C07B24281BD3054800684079DE
:1098F000401C03490968487101480068407905E047
:1099000074070020A41A002070070020401CEA49B8
:109910000968487105E00EF0E9FE0020E649096893
:10992000487147E009F03CF8002811D1FF200EF003
:109930002BFFE14800684079401CDF490968487105
:10994000DD4800684079401CDB490968487105E042
:109950000EF0CCFE0020D849096848712AE009F0D1
:109960001FF8002818D1D4480068C07A401CD2499A
:109970000968C872D0480068C07AD049097888421E
:109980000ADB0020CC490968C872CB48006880799E
:10999000401CC949096888710EF0A8FE0020C6491C
:1099A0000968487106E00EF0A1FE0020C24909686E
:1099B000487100BF00BF7DE1BF48006840790300E7
:1099C00012F010F80C0715C32CC349C366C382C339
:1099D0009FC30EF061FE0020B7490968C873B648FE
:1099E00000684079401CB44909684871B4E0B34943
:1099F0004969B14A1268D27A885C0EF0C5FEAE4859
:109A000000684079401CAC4909684871AA48006860
:109A10004079401CA849096848719DE008F0C0FFE2
:109A2000002811D177200EF0AFFEA34800684079DE
:109A3000401CA149096848719F4800684079401C52
:109A40009D490968487105E00EF050FE00209A49D2
:109A50000968487180E008F0A3FF002811D10C20AC
:109A60000EF092FE944800684079401C92490968C3
:109A70004871914800684079401C8F4909684871D5
:109A800005E00EF033FE00208B490968487163E061
:109A900008F086FF002810D10EF076FE8648006898
:109AA0004079401C844909684871834800684079BE
:109AB000401C81490968487105E00EF017FE00203E
:109AC0007D490968487147E008F06AFF002811D114
:109AD00013200EF059FE784800684079401C764902
:109AE00009684871744800684079401C72490968E7
:109AF000487105E00EF0FAFD00206F4909684871D1
:109B00002AE008F04DFF002818D16B480068C07AA1
:109B1000401C69490968C87267480068C07A67498B
:109B2000097888420ADB002063490968C8726248E4
:109B300000688079401C6049096888710EF0D6FD84
:109B400000205D490968487106E00EF0CFFD002055
:109B500059490968487100BF00BFABE0564800682A
:109B60004079030011F03EFF080513872A874787D5
:109B700063870EF091FD00204F490968C8734E4875
:109B800000684079401C4C49096848717AE04B49AB
:109B90004969494A1268D27A885C0EF0F5FD464858
:109BA00000684079401C444909684871424800688F
:109BB0004079401C40490968487163E008F0F0FEB4
:109BC000002811D149200EF0DFFD3B4800684079A4
:109BD000401C394909684871374800684079401C81
:109BE00035490968487105E00EF080FD00203249D2
:109BF0000968487146E008F0D3FE002810D10EF045
:109C0000C3FD2D4800684079401C2B490968487104
:109C1000294800684079401C27490968487105E0D7
:109C20000EF064FD00202449096848712AE008F01C
:109C3000B7FE002818D120480068C07A401C1E4991
:109C40000968C8721C480068C07A1C4909788842B3
:109C50000ADB002018490968C87217480068807933
:109C6000401C1549096888710EF040FD002012491A
:109C70000968487106E00EF039FD00200E490968B8
:109C8000487100BF00BF15E000200B4909688871CA
:109C9000094909684871062007490968C87009E040
:109CA0000EF024FD00200449096848710249096842
:109CB000887100BF00BF10BD74070020A41A0020E7
:109CC00010B56A4800684079030011F08BFE090660
:109CD00010C627C644C6608EC6000EF0DDFC634881
:109CE00000684079401C614909684871BCE06049DE
:109CF00049695E4A1268D27A885C0EF045FD5B487D
:109D000000684079401C5949096848715748006803
:109D10004079401C554909684871A5E008F040FEAB
:109D2000002811D17F200EF02FFD504800684079A7
:109D3000401C4E49096848714C4800684079401CF5
:109D40004A490968487105E00EF0D0FC00204749F7
:109D50000968487188E008F023FE002810D10EF051
:109D600013FD424800684079401C40490968487129
:109D70003E4800684079401C3C490968487105E04C
:109D80000EF0B4FC00203949096848716CE008F015
:109D900007FE002822D135480068C07A401C3349AC
:109DA0000968C87231480068C07A31490978884228
:109DB0000FDB00202D490968C8722C4800684079E3
:109DC000401C2A49096848710020284909684862EE
:109DD00008E0002025490968487103E00020234974
:109DE000096848710EF082FC3EE020480068407C23
:109DF000002816D01E48C068002803D01C48C1683F
:109E000019208847002019490968486217490968DC
:109E10004871164909688871052014490968C87095
:109E20001AE012480068406A282807D20F480068E4
:109E3000406A401C0D49096848620DE000200B494A
:109E400009684862094909684871084909688871C0
:109E5000052006490968C87006E00EF047FC00209E
:109E600002490968487100BF00BF10BD7407002097
:109E7000A41A002010B50024F7480068807A012851
:109E80007ED1F5480068C07900287AD0F248006891
:109E90008079002804D0012874D0022873D191E180
:109EA000ED480068007B24286ED2EB480068C0793A
:109EB00001287AD1002475E0E7480068C07A24219F
:109EC0004843E64909684018E3490968097B415C51
:109ED000E1480068C07A24225043E14A12688018A1
:109EE000DD4A1268127B805C814229D0DA48006822
:109EF000C07A24214843DA4909684018D6490968DC
:109F0000097B415CD4480068C07A24225043D34A7C
:109F100012688018D04A1268127B8154CE480068BB
:109F2000407B242805D3CC480068007BCA490968D7
:109F30004873C9480068007BC7490968887308E00E
:109F4000C5480068407B242803D20120C249096823
:109F50008871C1480068007B401CBF4909680873CC
:109F6000BD480068007B242808D3BB480068407BBC
:109F7000242803D20120B84909688871B64805E051
:109F8000D3E1CDE169E0BAE138E00EE00068007BA2
:109F9000242804D2B04800688079012800D103E069
:109FA000601CC4B2242C87D356E0002413E0AA48D6
:109FB0000068C07A24214843A94909684018015D16
:109FC000A5480068C07A24225043A44A1268801829
:109FD0000155601CC4B2242CE9D300209E490968B5
:109FE000487323209C490968887301209A490968AD
:109FF000887124209849096808732DE0002096494B
:10A000000968087394480068C07A401C924909683E
:10A01000C87291480068C07A92490978884217DB73
:10A020008D480068007C012804D102208A49096813
:10A03000887106E0002088490968887186490968A6
:10A04000C871002084490968C87283490968087486
:10A05000002081490968487161E17F4800684079C2
:10A06000030011F0BFFC080513A62AA651A68EA670
:10A0700001207949096808740EF00EFB76480068E3
:10A080004079401C74490968487199E075494969EB
:10A09000714A1268D27A885C0EF076FB6E480068CE
:10A0A0004079401C6C49096848716B4800684079E8
:10A0B000401C69490968487182E008F071FC002879
:10A0C0001BD165490968497B491CC8B20EF05CFB8D
:10A0D00061480068407B60490968C8735E48006851
:10A0E0004079401C5C49096848715B4800684079C8
:10A0F000401C59490968487105E00EF0F7FA002044
:10A100005549096848715BE008F04AFC00282BD1EA
:10A1100051490968C97A24225143504A1268891862
:10A120004D4A1268D27B885C0EF02EFB4A480068CC
:10A13000C07B401C48490968C87347480068C07B19
:10A1400045490968897B88421ADD4348006840799F
:10A15000401C4149096848713F4800684079401CEB
:10A160003D49096848710BE00EF0C0FA3A480068B2
:10A17000407B39490968C87300203749096848712C
:10A180001EE008F00DFC00280CD1334909688871E5
:10A19000242031490968C8732F49096848732E493A
:10A1A000096888730EF0A2FA00202B4909684871EB
:10A1B00006E00EF09BFA002027490968487100BFAD
:10A1C00000BFACE0244800684079030011F00AFCAD
:10A1D00008050F8E268E4C8E688E0EF05DFA1E4896
:10A1E00000684079401C1C490968487185E01D4998
:10A1F0004969194A1268D27A885C0EF0C5FA164885
:10A2000000684079401C1449096848711248006888
:10A210004079401C1049096848716EE008F0C0FBA5
:10A22000002811D149200EF0AFFA0B4800684079A0
:10A23000401C094909684871074800684079401C7A
:10A2400005490968487105E00EF050FA00200249FE
:10A250000968487151E00000740700207007002071
:10A260006C070020A41A002008F09AFB002810D1E7
:10A270000EF08AFA9C4800684079401C9A490968A7
:10A280004871994800684079401C974909684871AD
:10A2900005E00EF02BFA00209349096848712CE084
:10A2A00008F07EFB00281AD18F480068C07A401C55
:10A2B0008D490968C8728C480068C07A8B49097852
:10A2C00088420CDB002088490968C8728649096801
:10A2D000887185490968487183490968C8710EF019
:10A2E00005FA002080490968487106E00EF0FEF981
:10A2F00000207D490968487100BF00BF0FE00EF0E3
:10A30000F5F900207849096848717749096888712A
:10A3100075490968087374490968C87200BFE2E0AA
:10A320000020714909688872DDE06F480068807A12
:10A330000228F4D16C480068007A002879D06A4875
:10A3400000684079030011F04DFB0B0711BB25BBE2
:10A3500041545EBB7590BB000EF09EF962480068E8
:10A360004079401C604909684871B7E05F49496914
:10A3700008780EF009FA5C4800684079401C5A4998
:10A3800009684871584800684079401C5649096876
:10A390004871A3E008F004FB002810D10EF0F4F996
:10A3A000514800684079401C4F49096848714E483F
:10A3B00000684079401C4C490968487105E00EF07E
:10A3C00095F9002048490968487187E008F0E8FAE3
:10A3D000002807D1444800684079401C4249096878
:10A3E000487103E000204049096848710EF07EF989
:10A3F00074E00EF051F93C4800684079401C3A493D
:10A40000096848716AE0394949690978491CC8B244
:10A410000EF0BAF9344800684079401C32490968A6
:10A420004871314800684079401C2F4909684871DB
:10A4300054E054E008F0B4FA00280FD10EF0FEF812
:10A4400029490968887001200EF072F926480068D1
:10A450004079401C24490968487105E00EF046F92E
:10A46000002021490968487138E01F480068807859
:10A4700011280CD100201C4909680872AA201A4929
:10A4800009688870002018490968487011E016486A
:10A4900000684078401C14490968487012480068F8
:10A4A0004078032805D308F01BFB00200E490968FB
:10A4B00048700EF01BF900200B49096848710DE047
:10A4C0000EF014F900200849096848710649096826
:10A4D0004870AA2004490968887000BF03E0002082
:10A4E00001490968887210BD74070020A41A002071
:10A4F00070B5002508E06D1C1B48854202D209F0AA
:10A500008BFD01E0002503E009F0DAFC0028F2D120
:10A5100000BF0221002009F0E1FC0321002009F026
:10A52000DDFC0521002009F0D9FC0721002009F0FD
:10A53000D5FC002408E00020A1000C4A5054A100E2
:10A5400089184880601CC4B2042CF4D30120084947
:10A55000087000204870052088700020C8700548E9
:10A560000549088070BD000050C30000E4140020BD
:10A57000BA00002088130000B8000020F8B58D480C
:10A580000078030011F02EFA060405163D5EFDFC6E
:10A590000EE109F015FD00208649C8704870084694
:10A5A0008078002802D10320087002E0022081494F
:10A5B0000870FDE07F488078002804D07D488078CE
:10A5C000401E7C49887009F07BFC00280BD109F003
:10A5D000F7FC00207749C8700846807800280FD122
:10A5E000032008700CE07348C078401C7149C870A3
:10A5F0000846C078052803D30520087009F00CFD33
:10A60000D6E009F05DFC00280ED104216A4809F06B
:10A6100039FC00206749C87048706848684908805C
:10A620000420644908700CE06248C078401C61490D
:10A63000C8700846C078052803D30520087009F0C3
:10A64000EBFCB5E05B49497809015E4A515C490081
:10A65000594A505A5A490A8801210903FEF762FEF5
:10A660000090012553484078000156494018407831
:10A67000002801D100243CE04E48407800015149B7
:10A6800040184078012802D14D48048831E04948FB
:10A69000407800014B4940184078022812D14549C2
:10A6A00049780901474A89180879FEF755FE04469A
:10A6B000404949780901434A89180879FEF758FE4C
:10A6C000054616E03B48407800013E494018407876
:10A6D000032806D0374840780001401840781328F6
:10A6E00006D134484078000136494018848800E09B
:10A6F0000025002D2FD02F48407800013249431803
:10A700002C48407800012F49401802892948407898
:10A71000000140182146C7680098B84706462548FA
:10A7200040780001274BC018C288224840780001B9
:10A73000C01881783046FEF769FD06461D4840780E
:10A74000800022494018468001201A494978890032
:10A750001E4A50540AE000201649497889001B4AD5
:10A760008918488013494978890050541148407825
:10A77000401C1049487008464078042809D301E07D
:10A7800013E007E009F01CFC00200A494870032090
:10A7900008700DE009F094FB002803D10120054961
:10A7A000087001E009F038FC02E0FFF7A1FE00BFED
:10A7B00000BFF8BDBA000020BE00002088130000D2
:10A7C000B800002090C80100D0C80100E4140020A7
:10A7D00010B509F03FFB002405E00020A100074A66
:10A7E0005054601CC4B2042CF7D3002004490870F4
:10A7F0000520887003480449088010BDE414002037
:10A80000BA00002088130000B800002070B504468C
:10A81000002000F0AFF8002000F0DAF8002000F08F
:10A820009BF8002000F0C4F8002000F087F800201A
:10A8300000F0AEF800BF012000F08EF8012000F01B
:10A84000B7F8002521E0002000F086F8002000F095
:10A85000AFF880202040002806D0012000F08AF8C0
:10A86000012000F0B5F805E0002000F083F800209A
:10A8700000F0AEF800BF012000F06EF8012000F0FB
:10A8800097F86006040E681CC5B2082DDBDB0120BA
:10A8900000F054F8012000F07BF870BD70B504465C
:10A8A0000D46012000F066F8012000F091F800202C
:10A8B00000F052F8002000F07BF8002000F03EF895
:10A8C000002000F065F800BF012000F045F80120ED
:10A8D00000F06EF8002628E0002000F03DF800208F
:10A8E00000F066F880202040002803D0012000F00E
:10A8F00041F802E0002000F03DF8802028400028C8
:10A9000003D0012000F064F802E0002000F060F8BD
:10A9100000BF012000F020F8012000F049F8600697
:10A92000040E6806050E701CC6B2082ED4DB01208A
:10A9300000F004F8012000F02BF870BD10B50446BB
:10A94000002C04D08121032009F0F4FB03E08021D6
:10A95000032009F0EFFB10BD10B50446002C04D015
:10A960008121042009F0E6FB03E08021042009F0A6
:10A97000E1FB10BD10B50446002C04D0812102205B
:10A9800009F0D8FB03E08021022009F0D3FB10BDC1
:10A9900010B50446002C04D08121044809F0CAFBFC
:10A9A00003E08021014809F0C5FB10BD010700004C
:10A9B00010B50446002C05D081210720000209F0C3
:10A9C000B9FB04E080210720000209F0B3FB10BDB1
:10A9D00010B50446002C04D08121044809F0AAFBDC
:10A9E00003E08021014809F0A5FB10BD020700002B
:10A9F00010B5F920FFF70AFF8820FFF707FF902026
:10AA0000FFF704FF9820FFF701FF08210846FFF732
:10AA100045FFE820FFF7FAFE12210846FFF73EFF48
:10AA2000A020FFF7F3FE70210846FFF737FFA820AC
:10AA3000FFF7ECFE70210846FFF730FFB020FFF76C
:10AA4000E5FE70210846FFF729FFB820FFF7DEFE7C
:10AA500000210846FFF722FFC020FFF7D7FE0021A4
:10AA60000846FFF71BFFC820FFF7D0FE002108466D
:10AA7000FFF714FFD020FFF7C9FE2F210846FFF78C
:10AA80000DFFD820FFF7C2FE2F210846FFF706FF73
:10AA9000E020FFF7BBFE2F210846FFF7FFFE402016
:10AAA000FFF7B4FE00210846FFF7F8FE0A20FFF783
:10AAB000ADFE002405E000210846FFF7EFFE601C14
:10AAC000C4B25A2CF7DB00240AE000200B490855D9
:10AAD0000B4908550B4908550B490855601CC4B271
:10AAE0005A2CF2DB8120FFF791FE00200749087005
:10AAF0008870C8700871487010BD000024120020D2
:10AB00007E120020D8120020321300208600002080
:10AB100010B58020FFF77AFE10BD00000020044928
:10AB20000870012003490870002048707047000039
:10AB30008B0000208600002010B5484800780028CF
:10AB40007AD046488078030010F04CFF0604434A50
:10AB5000535A687E414800794149085C3F49097968
:10AB6000404A515C884209D13C4800793E49085C22
:10AB70003A4909793D4A515C88421BD037480079EF
:10AB80003749085C35490979364A505433480079C9
:10AB90003549085C31490979344A50542F48C07806
:10ABA000002803D004202D49887011E001202B4992
:10ABB00088700DE000202949C87008460079401CC3
:10ABC0000871084600795A2802DB002008710870D5
:10ABD00041E04020FFF71AFE0220204988703AE049
:10ABE0001E4A11791079FFF759FE03201B4988701E
:10ABF00031E00A20FFF70AFE0420184988702AE095
:10AC0000164A1279194B995C144A1279154B985CC3
:10AC1000FFF744FE0520114988701CE00F480079B9
:10AC2000401C0E490871084600795A2805DB0020AF
:10AC300008710870C87003E00EE001200749C87071
:10AC400000200649887006E00020044908708870DA
:10AC5000C870087100BF00BF10BD00008600002052
:10AC6000241200207E120020D8120020321300206F
:10AC700010B50EF02DF9012811D10E4800780528E5
:10AC800006D1FF22A532002101200FF0A1FD0FE027
:10AC90004B22D200002101200FF09AFD08E0002095
:10ACA0000549888048800022114601200FF090FD60
:10ACB00010BD0000D20000201A00002058221152BE
:10ACC000704710B504460121022000F071FA0021FE
:10ACD000022000F06DFA10BD014600205322525CA4
:10ACE00010231A40002A08D05322525C0C231A4029
:10ACF0009210032A18D1032016E05422525A01233D
:10AD0000DB031A40002A0ED05322525C0C231A4057
:10AD10009210032A05D05322525C9207920F032A05
:10AD200001D1022000E00120704702460020582394
:10AD30009B5A0B40002B01D0012000E000207047FF
:10AD4000014600226020405AFF231B0218400005E4
:10AD5000020F1001014BC01870470000005504405D
:10AD600010B5002A0AD056231B5A0C02234356243E
:10AD7000235256231B5A8B43235209E056231B5A56
:10AD80000C02A3435624235256231B5A0B4323522F
:10AD900010BD0000F8B504460D46012700263448D2
:10ADA000844203D10121022000F002FA2878401EDB
:10ADB000A0702088FF2101310843208020884008AE
:10ADC00040002080A878401EC1B25A200155687901
:10ADD0000007000CE97909020843A97908435C21BE
:10ADE0000853288981B240200153A868C000C10CD3
:10ADF00042200153A88981B244200153E868C00071
:10AE0000C10C46200153288A81B248200153286989
:10AE1000C000C10C4A200153A88A81B24C200153C2
:10AE20006869C000C10C4E2001535020005B297995
:10AE300009020843502108535020005B29798843B8
:10AE40005021085300E0761C5020005B4007400F63
:10AE50002979884202D007488642F4D15020005B0D
:10AE60004007400F2979884200D000273846F8BDB6
:10AE700000540440FFFF000030B5034600201C8949
:10AE80008C4209DD082A05D218244C431D682C1970
:10AE9000A05C02E0002000E0002030BD10B50246BA
:10AEA00013898B4205DD18234B431468E318987C03
:10AEB00000E0002010BD0146FF22C889C007C00F76
:10AEC00000280AD00120C88100E0521EC889C007AE
:10AED000C00F002801D0002AF7D1C889C007C00FD1
:10AEE00000280FD10220C8810420C881487A400878
:10AEF00040004872487A38239843487200204872CC
:10AF0000012070470020FCE70246507A01231843D5
:10AF10005072507A0B78DB0018435072087A01287F
:10AF200008D1888850814868000C0123DB0318434E
:10AF3000908108E0087A002805D150814868800097
:10AF40001A4B18409081487A012804D1507A402346
:10AF50001843507206E0487A002803D1507A402303
:10AF6000984350720878002811D1C87A1072087B73
:10AF70001070487B5070887B9070CB7BD370087CBE
:10AF800010714B7C5371887C9071CB7CD371887A23
:10AF9000002803D00120C002D08101E00820D08128
:10AFA000FF200130D081012070470000FC1F00000D
:10AFB000002904D0427A80231A43427203E0427A85
:10AFC00080239A434272704730B5024600200F4BEF
:10AFD0005024A45A0D022C435025AC525024A45A9C
:10AFE0008C43AC5200E05B1E5024A45A6407640FEB
:10AFF0008C4201D0002BF6D15024A45A6407640F70
:10B00000002C01D0002000E0012030BDFFFF000037
:10B01000827A80231A40802A00D081727047000013
:10B0200070B5044600250023002D02D001266020C3
:10B0300006530420C88188890126F6033040002881
:10B0400008D0012010728889C004C0084E8930439E
:10B05000506006E00020107288890F4E304080104A
:10B060005060087AD072002304E0CE5C10460C30A9
:10B07000C6545B1CD07A9842F7DCC889042630405D
:10B08000002804D1C889F6023040002801D00020F1
:10B0900070BDD07AFCE70000FC1F0000027C80231A
:10B0A0001A40802A00D00174704710B50246FF2371
:10B0B000D089C007C00F00280AD00120D08100E04D
:10B0C0005B1ED089C007C00F002801D0002BF7D12C
:10B0D000D089C007C00F002801D0002010BD507AD1
:10B0E000012420435072507A3824A0435072C87A09
:10B0F0001072487A00280FD1087B1070487B50707E
:10B10000887B9070CC7BD470087C10714C7C54711F
:10B11000887C9071CC7CD471FF200130D0814000BC
:10B12000D081107ADAE70000F8B504460D46002019
:10B13000002C00D100BF002A00D100BF012C01D19A
:10B1400041263043012A01D112263043022C01D17D
:10B15000C0263043022A01D130263043134E3070CE
:10B1600076788027BE43114F7E70012C08D1FF21D5
:10B1700000BF0E4EB3781E460E4033468B42F8D1C8
:10B180000A4E76784027BE43084F7E70012A0BD1C5
:10B190000026009603E000BF009E761C0096FF2765
:10B1A0006937009EBE42F6D9F8BD00000004024097
:10B1B000002905D0054A12780243044B1A7004E0B6
:10B1C000024A12788243014B1A70704720040240F1
:10B1D000002905D0054A927E0243044B9A7604E08A
:10B1E000024A927E8243014B9A76704700080240E1
:10B1F00001200649087000BF0448007880210840FB
:10B200000028F9D00120024908707047000C024064
:10B210001401002070B5034614460020002B01D114
:10B22000C0B202E005468035E8B2012902D1051D11
:10B23000E8B206E0022903D105460835E8B200E08D
:10B24000C0B2012C02D1851CE8B200E0C0B2084DAA
:10B25000A870AD7801263543054EB570002201E097
:10B2600000BF521C7D252D01AA42F9D970BD0000F6
:10B27000000C024070B500242448007920210840C9
:10B28000002801D0224D3FE000F046F80546214855
:10B29000007880210840002836D01E488078084079
:10B2A000002801D01A4D02E000F036F80546194892
:10B2B00080780007840F022C01DBAD0804E0012C2C
:10B2C00001D16D0800E000BF124880788007C00FF0
:10B2D000002801D02D0101E00C2045430D480078E5
:10B2E0004007840F002C02D1601CC4B207E0032C7D
:10B2F00003D1601C4006040E01E06006040E2146E6
:10B300002846FCF71DFF0546284670BD0004024094
:10B3100000127A00000C024000B5C0229178F82299
:10B3200011401C4A12781143EA2923D00ADC0A464C
:10B33000E03A130010F056FB0A181C20242A2A2A8F
:10B340002A161A2AED291FD004DCEB2916D0EC2985
:10B350001CD117E0F02903D0F82917D10E4817E0C7
:10B360000E4815E00E4813E00E4811E00E480FE0BD
:10B370000E480DE00E480BE00E4809E00E4807E0CD
:10B380000E4805E00E4803E00E4801E00D4800BFFE
:10B3900000BF00BD201C02400090D003006CDC0206
:10B3A0000048E80100366E010024F400001BB700DD
:10B3B00000127A00808D5B0000093D00C0C62D00A0
:10B3C00080841E0040420F0010B50446204600F065
:10B3D00049FD002010BD000010B590211348FCF776
:10B3E0005FFF124812490860124848600620088131
:10B3F0000020887206220F490D4800F04BFA002108
:10B400000B48FFF705FE80210B48FCF749FF0A486F
:10B410000A4948600A4B04220A49084800F0B6FB72
:10B4200055210648FFF73AFE10BD0000EC0700204A
:10B43000CC07002000C701007C080020D8070020AE
:10B44000C9B3000090C601000C4A127812060B4BDB
:10B450005B781B041A43094B9B781B021A43074B6A
:10B46000DB781A43104642084240D20083085A4013
:10B470001146034A5140034A116070478B06002071
:10B480000102000090060020F8B504460F46A07A9D
:10B490004006400E002874D10025ACE01820684317
:10B4A00021680818407C01283CD1012118206843FC
:10B4B00022681018017400260CE0182068432168E7
:10B4C00008180830815D18206843226810188155DB
:10B4D000701CC6B2082EF0D30021182068432268E1
:10B4E000101801741820684322681018417418203D
:10B4F00068432268101841611820684322681018B8
:10B5000081742C20684361680818406A002809D0BB
:10B5100018236B432268D0182C236B436268D2181F
:10B52000516A884718206843216808184069FF213C
:10B53000C94388425DD818206843216808184069CB
:10B54000C119182068432268101841611820684307
:10B550002168081841692C206843626810188069C6
:10B56000814246D31820684321680818807C5528FA
:10B570003FD0552118206843226810188174002696
:10B5800024E03CE01820684321680818805D2C21E5
:10B590006943626851181031895D08401821694378
:10B5A0002268511888551820684321680818805D62
:10B5B0002C216943626851180831895D08431821BC
:10B5C0006943226851188855701CC6B2082ED9D319
:10B5D0002C20684361680818806A002809D0182365
:10B5E0006B432268D0182C236B436268D218916A8F
:10B5F0008847681C85B22089A84200DD4EE7F8BD67
:10B6000010B50446002010F02FFD022841D121483A
:10B610000078002802D101201E4908701D480078DA
:10B6200001281FD11B484078401C1A494870214608
:10B630005A20FCF785FD17494978884229D800200F
:10B640001449487008468078401C88700846807805
:10B650000A2803D30020887002200870002010F010
:10B6600033FD16E00B480078022812D109484078D3
:10B67000401C0849487021467D20C000FCF760FD51
:10B6800004494978884204D800200249487010F0E3
:10B690001BFD10BD6800002000B587B00021684682
:10B6A0000171042141710C480290411003910B4932
:10B6B000049105910A480690FFF78EFE01A810F04C
:10B6C00067FD00F019FB00F00FF80021054808F0B5
:10B6D0009DFD07B000BD0000FFFF1F00FFFFFF1F23
:10B6E0001DB900000205000010B5FF2002306549B9
:10B6F0004860002008720120087000204872012074
:10B7000088726148FFF7D7FB5E495F48FFF7FCFB93
:10B7100001215D48FFF74CFC5C485A494860002015
:10B720000872012008700020487201208872564873
:10B730001030FFF7C0FB534953481030FFF7E4FBCC
:10B74000012151481030FFF733FC5048401E4D494D
:10B750004860002008720120087000204872012013
:10B76000887249485030FFF7A6FB4649464850309A
:10B77000FFF7CAFB012144485030FFF719FC43484A
:10B78000C13840494860002008720120087000203C
:10B790004872012088723C484030FFF78CFB3949E1
:10B7A00039484030FFF7B0FB012137484030FFF700
:10B7B000FFFBFF201230334948600020087201204F
:10B7C000087000204872012088722F486030FFF70F
:10B7D00072FB2C492C486030FFF796FB01212A4868
:10B7E0006030FFF7E5FBFF2021302649486000204C
:10B7F00008720120087000204872012088722248D7
:10B80000A030FFF758FB1F491F48A030FFF77CFB13
:10B8100001211D48A030FFF7CBFB3F204001194913
:10B820004860002008720120087000204872012042
:10B83000887215482030FFF73EFB1249124820302D
:10B84000FFF762FB012110482030FFF7B1FB1048E1
:10B850000C494860002008720120087000204872DE
:10B860000120887208483030FFF725FB054906485B
:10B870003030FFF749FB012103483030FFF798FBD8
:10B8800010BD0000C815002010550440020400003F
:10B89000DF070000F0B50B46144643600481002129
:10B8A00036E0002216E02C254D4346687519AD5C44
:10B8B00018274F430668F619B5542C254D434668A2
:10B8C0007519AD5C18274F430668F6190836B5544C
:10B8D000551CEAB2082AE6D3002518274F4306680C
:10B8E000F619357418274F430668F619757418272A
:10B8F0004F430668F619B57418274F430668F619C2
:10B90000F57418274F430668F61975614D1CA9B2E6
:10B9100005898D42C5DC00258572F0BD70B50446F1
:10B92000606800F0EFFD0546E27A23460C332946B5
:10B93000094800F0AFFD09496068884203D0491CFE
:10B940006068884206D1E17AA28890B222460C3221
:10B9500002F04AFD70BD0000CC070020DF070000A8
:10B96000F8B5054600262C46002C07D000BF03E0A2
:10B97000FF20A055701CC6B2082EF9D304F06CFB52
:10B98000C0000821084007462068884338432060EB
:10B99000F8BDF8B5054600262C46002C07D000BFA0
:10B9A00003E0FF20A055701CC6B2082EF9D304F0A6
:10B9B000C5FB07462068000C00043843206004F0F3
:10B9C0007DFC0004070C3F04208880B238432060CF
:10B9D000F8BDFEB5054600260020019001F000FDEF
:10B9E0000A210090FCF7ACFB074604F069FB0A2132
:10B9F0000090FCF7BBFB80B201902C46002C07D0D6
:10BA000000BF03E0FF20A055701CC6B2082EF9D37A
:10BA100007210906206888430199091209060722AF
:10BA200012061140084320606068000A0002019974
:10BA3000C9B208436060FF21090260688843390C7D
:10BA40000902FF221202114008436060110260687F
:10BA50008843390A09041202114008436060606893
:10BA60000002000A3906090E09060843606004F066
:10BA7000E7FAC007C00FC0070090206840004008E8
:10BA800000990843206003F0EBFD0007000F0090D1
:10BA900020680009000100990843206003F0DAFDE6
:10BAA000022806D101210907206888434018206038
:10BAB00004E00121090720688843206004F086FA29
:10BAC0000001F02108400090206888430099084355
:10BAD000206004F039FBFF2806DDFF2109042068FF
:10BAE0008843401820600BE004F02EFB0004FF2187
:10BAF00009040840009020688843009908432060AA
:10BB0000FEBDFEB50546002600200190002704F08A
:10BB1000AFFA64210090FCF729FB80B2019000206D
:10BB200001F070FC87B22C46002C07D000BF03E068
:10BB3000FF20A055701CC6B2082EF9D32068000A59
:10BB400000020199C9B208432060FF21090420685E
:10BB5000884339120904FF2212041140084320606F
:10BB600020680002000A3906090E09060843206011
:10BB700003F07CFD28300002FF21090208400090FC
:10BB800020688843009908432060FEBDFFB581B05E
:10BB900004460F46002500260020009027600398E9
:10BBA00020810498E0600020207400BF9DE01C20EC
:10BBB0006843216808586A01616888501C206843FE
:10BBC0002168081880686A016168891848601C202B
:10BBD00068432168081840686A01616889188860AC
:10BBE0001C20684321680818C0686A0161688918C8
:10BBF000C8601C20684321680818007C6A016168DD
:10BC0000891808741C20684321680818407C6A0160
:10BC10006168891848741C20684321680818807C72
:10BC20006A016168891888831C20684321680818A4
:10BC3000C07C6A0161688918887400206A016168A3
:10BC40008918C8741C2068432168081840680028B7
:10BC500013D01C20684321680818C07C002805D137
:10BC6000401E6A0161688918C8831AE00020C04339
:10BC70006A0161688918C88313E01C206843216841
:10BC80000818C07C002805D000206A016168891866
:10BC9000C88306E000206A0161688918C883012012
:10BCA0000090002607E000216A01606880181430C7
:10BCB0008155701CC6B2690160684018808BB04223
:10BCC000F1DC1C20684321680818406900280AD06C
:10BCD0006B016268D218104614301C236B43226833
:10BCE000D21851698847681CC5B22089A84200DD76
:10BCF0005DE7009805B0F0BD00B58BB056480790E1
:10BD0000002108A801706846017608A8417000204B
:10BD100052498872082108A8C170002004E000225E
:10BD200009A90A54411CC8B208A9C9788142F6DCA5
:10BD30004B48FFF7C0F806A94948FFF7E5F8464821
:10BD4000401C0790002108A801706846017608A8E9
:10BD50004170002041498872082108A8C170002064
:10BD600004E0002209A90A54411CC8B208A9C978F4
:10BD70008142F6DC3A484030FFF79DF806A9384882
:10BD80004030FFF7C1F8452000010790002108A8C6
:10BD900001706846017608A8417000202F4988721A
:10BDA000082108A8C170002004E0002209A90A5453
:10BDB000411CC8B208A9C9788142F6DC2848503035
:10BDC000FFF779F806A926485030FFF79DF81120B3
:10BDD00040010790002108A801706846017608A874
:10BDE000417000201D498872082108A8C1700020F8
:10BDF00004E0002209A90A54411CC8B208A9C97864
:10BE00008142F6DC16482030FFF755F806A91448A1
:10BE10002030FFF779F8FD20C0000290002168462D
:10BE200001730171417381730821C173002004E023
:10BE3000002204A90A54411CC8B26946C97B814248
:10BE4000F6DC07481030FFF736F801A90448103037
:10BE5000FFF75AF80BB000BDEE060000C815002031
:10BE60008055044030B585B0044600252068019017
:10BE7000A1796846C1726179417200210172017035
:10BE800000BF05E020460830415D03A841556D1C08
:10BE90006846C07AA842F5D8112149010198401A94
:10BEA0001BD023210901401A11D011494018002844
:10BEB00002D0012817D104E069460E48FFF7F5F8D3
:10BEC00012E069460B484030FFF7EFF80CE0694696
:10BED00008485030FFF7E9F806E069460548203089
:10BEE000FFF7E3F800E000BF00BF05B030BD000081
:10BEF00062FDFFFF80550440F0B585B004460F4653
:10BF000000250026207C4006400E55287ED100BF2B
:10BF100076E1690160684018807C002877D169016A
:10BF20006068401840686A016168891889688842B9
:10BF300009D26901606840184068C0196A016168E7
:10BF4000891848605AE1690160684018C068AF49C3
:10BF5000884208D8690160684018C068401C6A01BE
:10BF600061688918C860690160684018C07C002851
:10BF700021D1002607E000216A0160688018143092
:10BF80008155701CC6B2690160684018808BB04250
:10BF9000F1DC1C20684321680818406900280AD099
:10BFA0006B016268D218104614301C236B43226860
:10BFB000D21851698847690160684058009069014A
:10BFC00060684018017C6846017100214171690177
:10BFD00060684018017F6846817169016068401897
:10BFE000417C6846C171002608E06901606840181C
:10BFF0001430815D02A88155701CC6B26901606869
:10C000004018808BB042F0DCE06801E0FCE01DE00D
:10C01000002806D06846E16888476A016168891887
:10C02000C874690160684018C07C002804D16A01A6
:10C03000616889184860E1E06901606840184068FB
:10C04000C01B6A01616889184860D7E069016068AF
:10C05000401880680028EED0690160684018C08BE5
:10C060000028E8D0690160684018C08B6A016168E7
:10C070008918C968884207D1690160684018C08B77
:10C080006249C94388427DD16901606840184068AF
:10C090006A01616889188968884209D26901606803
:10C0A00040184068C0196A01616889184860A5E0B5
:10C0B00000206A0161688918486069016068401859
:10C0C000C0685249884208D8690160684018C06851
:10C0D000401C6A0161688918C860002607E00021D9
:10C0E0006A016068801814308155701CC6B26901FD
:10C0F00060684018808BB042F1DC1C2068432168E6
:10C100000818406900280AD06B016268D2181046EE
:10C1100014301C236B432268D21851698847690187
:10C12000606840580090690160684018017C68466A
:10C13000017100214171690160684018017F684602
:10C140008171690160684018417C6846C1710026B0
:10C1500008E06901606840181430815D02A88155CB
:10C16000701CC6B2690160684018808BB042F0DC78
:10C17000E068002808D06846E16888476A0161687D
:10C18000891800E015E0C874690160684018C07C37
:10C19000002804D16A016168891848602EE06901AD
:10C1A000606840184068C01B6A016168891848606F
:10C1B00024E01C20684321680818406800280FD03C
:10C1C0000020C0436A0161688918C8831C20684345
:10C1D0002168081840686A0161688918886008E069
:10C1E00000206A0161688918C8836A01616889183A
:10C1F000886000206A0161688918C860681CC5B23F
:10C200002089A84200DD84E605B0F0BD0000FFFFF4
:10C210007CB500BF192128480078FBF791FF044640
:10C2200026486043264A81180022012009F0C0FEFA
:10C2300020460A2250436430001981B200220120B6
:10C240000BF044FC01200A2262431219D1B20A22E7
:10C25000624312190090D0B201231A4608F00AF97D
:10C2600064220721002006F033FA0120009001909B
:10C270000B20604382B20B20604381B20023012077
:10C280000AF074FF6F20604381B201200BF0C4FEFE
:10C29000002505E00121284609F0C4FD681CC5B24F
:10C2A0000F2DF7DB21460B2251436431C8B20CF04D
:10C2B000FFF80CF0E7F87CBD63000020672B00005E
:10C2C000A08601000020054908700549087005494D
:10C2D000087005490870054908707047640000201F
:10C2E0006500002063000020620000206100002043
:10C2F000F0B589B000BF00BF00BF00BF00BF00BFE6
:10C3000000BF00BF00BF052155480078FBF718FFAC
:10C310000446E1B2012009F02FFC032150480078C7
:10C32000FBF724FF0B214843643080B20690E1B252
:10C3300001231846069A08F077FB494909788A00D4
:10C3400088180621FBF712FFFF21F531484380B220
:10C3500007900798FBF70AFFC7B23946012009F09A
:10C3600047F803213E480078FBF700FF0B214843C4
:10C37000643080B208900022012008990BF0A6FBDF
:10C38000032137480078FBF7F1FE36494843364928
:10C390004018039000220120039909F009FE0321AF
:10C3A0002F480078FBF7E2FE0B21484380B204904F
:10C3B00003212B480078FBF7D9FE0B21484386B2B6
:10C3C0000120F1B20090049AD0B201231A4608F07D
:10C3D00051F864220721002006F07AF90321204851
:10C3E0000078FBF7C3FE0B21484385B20120009083
:10C3F00000232A46294601900AF0B8FE0321184876
:10C400000078FBF7B3FE6F21484380B2059001200E
:10C4100005990BF001FE154800783C2805DA134811
:10C420000078401C1149087002E03C200F49087058
:10C430000E4800781D2805DC09480078401C084992
:10C4400008700BE006480078002802D10449087003
:10C4500004E003480078401E0149087009B0F0BDAF
:10C4600064000020672B0000A0860100650000200A
:10C47000002000BF06E00021044A1154044A115470
:10C48000411CC8B25A28F6DB704700002412002075
:10C49000D8120020FFB581B004460F463D462089E2
:10C4A000A8422DDD1820684321680818007C002868
:10C4B00026D1002609E00498815D1820684322688F
:10C4C000101808308155701CC6B2082EF3D3012114
:10C4D000182068432268101841742C206843616852
:10C4E0000818006A00280BD018236B432268D21862
:10C4F000104608302C236B436268D218116A8847B3
:10C5000005B0F0BD01460620104BCA1A99420FD063
:10C5100008DCCA1FFA3A002A12D0102A0AD01F2AB1
:10C5200010D10BE0C02A07D0C12A0BD100200BE0AC
:10C53000012009E0022007E0032005E0042003E0D9
:10C54000052001E0062000BF00BF70474103000046
:10C5500010B504467D21C90061430846322103F02D
:10C5600083FB10BD014800687047000044000020B4
:10C5700001480068704700004000002010B50549E0
:10C5800009886522514308466421FBF7EFFD80B21C
:10C5900010BD00004E0000200148007870470000E8
:10C5A0005300002001480078704700004C00002034
:10C5B00010B50CF08DFC01282ED100F065F801209B
:10C5C00000F068F803F0AEFB84B2204600F044F8B7
:10C5D00003F054FD84B2204600F04AF803F090FEC8
:10C5E000012805D100F03EF8012000F047F805E0F1
:10C5F000002000F037F8002000F040F80020134938
:10C60000086013480068134988421ED21048006829
:10C61000801C0F49086018E000200D4908600B4895
:10C6200000680C49884204D208480068801C074909
:10C630000860002000F028F8012000F02BF800200E
:10C6400000F00AF8002000F013F810BD44000020AC
:10C6500040000020FFFFFF7F014908807047000075
:10C660004E00002001490870704700005300002070
:10C6700001490880704700005000002001490870FF
:10C680007047000054000020014908707047000006
:10C690004C00002001490870704700005200002043
:10C6A0000021014A117170470060004000220149D9
:10C6B0004A75704700600040002201494A76704781
:10C6C000006000400021014A117270470060004084
:10C6D0000021014A11737047006000400021014AA7
:10C6E00011747047006000400021014A11757047C5
:10C6F000006000400021014A117670470060004050
:10C70000002201494A73704700600040002201493D
:10C710004A7470470060004010B51C4C1C492068EA
:10C7200088421ED106221B49201DFBF7C4FD0028AC
:10C7300017D10D22184920460A30FBF7BCFD00280E
:10C740000FD10622154920461730FBF7B4FD00280B
:10C7500007D10622124920461D30FBF7ACFD002808
:10C760000DD000F073FE0A480E49086007480FF02C
:10C770009AFD0C4A242105480FF0C0FD04E0242254
:10C7800021460848FBF773FD10BD00000002500071
:10C790007AA7A55AA1060020A70600209B06002024
:10C7A00095060020C8190020002008490870084993
:10C7B00008700120074908700020074908700748E1
:10C7C0000749086000200749087070478306002069
:10C7D00082060020850600208A060020250600002B
:10C7E000B40600209406002010B504469120604352
:10C7F00084B20A212046FBF7B9FC84B20521204609
:10C80000FBF7B4FC052901DB601D84B2204610BD96
:10C8100070B5A8B0054600240026A0216846FBF7A5
:10C820003FFD00F093FC1E490A68142169435050F3
:10C8300000211B4802681420684310184160184802
:10C840000268142068431018816015484068002869
:10C8500024D000BF17E06006060E282E00D316E095
:10C860000F480168142060430858B1006A465050D0
:10C870000B4801681420604308184168701C800050
:10C880001150601CC4B20648007AA042E3DC00BF2D
:10C8900062000348694643680220984728B070BD8B
:10C8A000181A002030B5A9B000240025A02101A845
:10C8B000FBF7F6FC00BF25E06006050E00F046FC25
:10C8C0001F490A6814216143505000211C48026826
:10C8D0001420604310184160194802681420604316
:10C8E00010188160282D0BD2154801681420604370
:10C8F0000858A90001AA50500021681C800011505E
:10C90000601CC4B20E48007AA042D5DC0C484068D6
:10C91000002813D00A48007A4000282806D3084887
:10C92000282201A943680220984707E00448007ABA
:10C930004200034801A943680220984729B030BD4E
:10C94000181A002010B50CF0C3FA01287ED1FFF7A9
:10C950000FFE4F49884216D20F204E494871887108
:10C9600008468078002801D1052048704948807821
:10C97000052802D100204749487000204549087227
:10C98000487208702AE0FA20424948718871424989
:10C99000088803F09DFA4048807800280CD13D4972
:10C9A000087008464079C8700846807908710020F0
:10C9B00088704870487211E00120364908700846B6
:10C9C000407A00280AD101204872084640788870D1
:10C9D00008464079C8700846807908712D488078EB
:10C9E0002C494978884213DD00202A49C87008463E
:10C9F0000079401C0871084600798979884220DB5B
:10CA000000202449087108468078401E887018E08C
:10CA1000204880781F494978884212DA00201D4951
:10CA200008710846C078401CC8700846C07849792B
:10CA3000884206DB00201749C87008468078401CF1
:10CA4000887015488078002805D100E013E00120A7
:10CA5000104908721BE010480088732803DB02208D
:10CA60000C49087213E00C48008870280FDC002085
:10CA7000084908720BE00020064908700846407912
:10CA8000C87008468079087100200872487210BD8D
:10CA9000B80B0000FC0800206C00002000200449B6
:10CAA00088704870C870087108724872704700003A
:10CAB000FC0800200020064908808870054988701D
:10CAC0004870FA20C87008710020087248727047D8
:10CAD0006C000020FC08002070B503F053F90446F8
:10CAE00003F062F905460CF0F3F901282ED1052177
:10CAF0001A48FEF7D3F9552804D100201849887048
:10CB0000088027E0012D04D1002015498870088095
:10CB100020E00120124988701248844202DB201A6A
:10CB200084B200E000240A212046FBF71FFB052900
:10CB300001DB601D84B20C48844200DD04460A21FA
:10CB40002046FBF713FB0649088003E00020044958
:10CB500088700880FFF7F6FE70BD0000CC0700204B
:10CB60006C000020AA0A0000C60700001CB50020C7
:10CB70000090019000F0EAFA0B49086000200B4990
:10CB8000096808600A48006800280CD0074909684D
:10CB900008680A21FBF7D4FA0090012269460520B3
:10CBA000034B1B6898471CBD8407002078070020B2
:10CBB000800700200020084948800849088008496B
:10CBC0000880084908700849887208490880488028
:10CBD00001200871704700002C0000202000002078
:10CBE0002200002024000020B007002026000020A2
:10CBF000F8B503F0A9F8074603F0B8F80090FFF77E
:10CC0000D1FC012860D10521C548FEF747F9552818
:10CC100002D00098012807D10020C2490870C249FB
:10CC20000880C249887256E0BE480078002810D1BA
:10CC30000120BC4908703D462846E917890F0918AC
:10CC400089030D0CBA48854200DD0546B6480580CB
:10CC500041E0B648807A4000B4490F520846867ACF
:10CC60000EE07000B1490D5A701E4000085A710064
:10CC7000AE4A5052701E400011460D52701EC6B290
:10CC8000002E08DD7000A949095A701E4000A74A0D
:10CC9000105A8142E5DBA548807A401CA34988727E
:10CCA0000846807A052816DB002088720846C58869
:10CCB0002846E917890F09188D109D48854200DD27
:10CCC00005469948058006E0002096490870964977
:10CCD0000880964988729448058896480088A8423A
:10CCE00057DA94480088281A84B2924800790128BB
:10CCF00027D190484088A0420BDA8E4840880A30FD
:10CD00008C49488008464088A04204DD084644809B
:10CD100001E088484480874844882046E117890F0D
:10CD200009188C100A2C00DA0A248248008800199D
:10CD30008049088008460088A84201DD0846058031
:10CD4000CDE07C484088142805DD7A4840881438B6
:10CD50007849488002E00020764948807548448838
:10CD60002046E117890F09188C100A2C03DA0120DC
:10CD700070490871B3E06F480088A04205DD6D4836
:10CD80000088001B6B490880A9E0002069490880E1
:10CD9000A5E068480088A84259DD66480088401B25
:10CDA00084B264480079012827D162484088142859
:10CDB00005DD6048408814385E49488002E0002064
:10CDC0005C4948805B4844882046E117890F091870
:10CDD0008C100A2C03DA0220564908717FE055486E
:10CDE0000088001953490880084600885049884245
:10CDF00075DD08464F49088071E04E484088A042E2
:10CE00000BDA4C4840880A304A4948800846408836
:10CE1000A04204DD0846448001E04648448045487D
:10CE200044882046E117890F09188C100A2C00DA73
:10CE30000A24404800882919884202DA3D480580C2
:10CE40004DE03C480088001B3A49088047E03948DB
:10CE500044882046E117890F09188C100A2C3EDD02
:10CE600034484088142805DD324840881438314958
:10CE7000488002E000202F4948802E484488204600
:10CE8000E117890F09188C102A480079012813D15D
:10CE90000A2C03DA02202749087120E0254800887F
:10CEA000001924490880084600882149884216DD77
:10CEB00008462049088012E00A2C03DA01201D49A7
:10CEC00008710CE01B480088A04205DD1948008865
:10CED000001B1849088002E0002016490880164807
:10CEE0000088502804DC134800881349088016E0A5
:10CEF0001048008810490988884204DD0D480088E0
:10CF00000D4908800BE00B4800880B490988081A76
:10CF100084B2502C03DB0748008807490880F8BD1D
:10CF2000CC0700202400002020000020B0070020B3
:10CF3000E02E0000260000202200002010B504464C
:10CF400064204443A1212046FBF7FAF8044620461A
:10CF500010BD00007CB5002400200190009000F07E
:10CF60003FFA05460A21FBF7EBF804460122694621
:10CF7000042000F07BFC0098401C002814D17D2088
:10CF8000C00020181149086008460068019001227D
:10CF900001A9032000F0A8FC0120009001226946AD
:10CFA000042000F0A1FC0FE0009801280CD17D20A6
:10CFB0000001201805490860084600680190012218
:10CFC00001A9032000F090FC7CBD0000DC000020E3
:10CFD00010B501200F49087000200F49096808604A
:10CFE0000D49096848600C490968886000F07EF9BD
:10CFF000FFF7BCFDFFF756FC08480068002807D083
:10D0000001220548016808310020044B1B6898473D
:10D0100010BD00001D070020180700201407002085
:10D0200010B5184800681849884229D11748006887
:10D03000002804D015480068804715490870154835
:10D040000068002804D0134800688047124908701F
:10D0500012480068002804D0104800688047104932
:10D06000088010480068002805D00E4800688047F6
:10D070000D49088002E00D480B49088000F078F85F
:10D0800010BD000028070020785634120407002045
:10D090001C070020080700201E0700200C070020A6
:10D0A0002007002010070020220700201027000082
:10D0B00010B50023174C2360174C2370174C2370B6
:10D0C000174C2370174C2380174C2380174C237068
:10D0D000174C13682360174C53682360164C9368F1
:10D0E0002360164CD3682360154C13692360002815
:10D0F0000CD0144B1860134C0B682468A3600023F9
:10D10000104C246823600F4C246863600E4B014C64
:10D11000236010BD28070020240700201C070020E2
:10D120001E07002020070020220700201D070020E6
:10D1300004070020080700200C070020100700202B
:10D14000140700201807002078563412054800689C
:10D150000549884203D1054800688068704700206F
:10D16000C043FBE728070020785634121807002038
:10D1700070B50024002500263048007801285CD1D5
:10D180002F480078002858D12E480078012854D123
:10D190002D4805882D490988694308462C49FAF726
:10D1A000CFFF85B2E1200001854207D819216943EC
:10D1B00008460921FAF7C4FF044600E0244C25483C
:10D1C0000068006800192349096808602148006860
:10D1D0000068204909684968884207D31D480068EB
:10D1E00000681C4909684968461A0AE0194800683D
:10D1F00040680021C943081A16490968096840189F
:10D20000461C1548864218D3344601462046FAF794
:10D2100097FF04460F48006841680F4860430818AC
:10D220000C490968486001200C49087009480068E9
:10D230008068001907490968886070BD1C070020D4
:10D240001D0700201E0700202007002022070020C5
:10D250001027000018070020A086010024070020E6
:10D2600000220C4B1A600C4B0A681A600B4B4A6880
:10D270001A600B4B8A681A600A4BCA681A600A4B1C
:10D280000A691A60002801D0084A1060084A014B58
:10D290001A607047280700200407002008070020B4
:10D2A0000C0700201007002014070020180700209A
:10D2B0007856341210B50A48006800280ED0094884
:10D2C000007801280AD1002006490870012206488A
:10D2D000016808310020024B1B68984710BD000010
:10D2E0001407002024070020180700201CB5002088
:10D2F000009001900024FFF729FF04460E480068C3
:10D30000046000200C49096848600B49096888607E
:10D310000A48006800280DD007480068006800909F
:10D320000548006840680190022269460120034BCD
:10D330001B6898471CBD00002C0700203007002008
:10D34000F8B505460C4616460027002D17D00E48A6
:10D350000560FFF7FBFE07462068B84203D90A487C
:10D360000068076003E0084920680968086006490A
:10D370006068096848600449A0680968C860034893
:10D38000066000F005F8F8BD2C07002030070020EB
:10D3900070B500240025FFF7D9FE04460F48006849
:10D3A0000068A04200D903E00C4800680068251A14
:10D3B0000A480068406840190849096888600748B9
:10D3C0000068806805490968C968884205D903482A
:10D3D0000068C06801490968886070BD2C0700209A
:10D3E00001480068806870472C070020002801D0A1
:10D3F000024A1060024A1160704700002C070020AA
:10D4000030070020014610480268142048431018D5
:10D4100082680D480368142048431818C068824287
:10D420000BD909480268142048431018C2680648FE
:10D4300003681420484318188260034802681420C7
:10D440004843101880687047181A0020002005E033
:10D4500019490A5C19490A54411CC8B20628F7DB6D
:10D46000002006E016490A5C1449891D0A54411C33
:10D47000C8B20D28F6DB002006E012490A5C0F490D
:10D4800013310A54411CC8B20628F6DB002006E01E
:10D490000D490A5C094919310A54411CC8B20628D1
:10D4A000F6DB002005E0002204491F310A54411C2C
:10D4B000C8B20128F7DB7047A1060020CC19002074
:10D4C000A70600209B0600209506002010B500202E
:10D4D00005490860486008724872887202F0C2FD0F
:10D4E0000149C87210BD00000809002070B5002471
:10D4F000002502F0B7FD6D49C87202F099FC0446A0
:10D5000002F0A0FC0546FFF74DF801286FD101217C
:10D510006748FDF7C3FC552807D10020634908720E
:10D520004872086048608872BFE0FF2C01D0FF2D70
:10D530006BD1FF2C2ED1FF2D2CD000205B4908721F
:10D540000120487263200860FF201430684348605F
:10D5500048680A21FAF7F4FD544948604868662192
:10D56000FAF7EEFD5149486008464068632801D942
:10D57000632048604D484068112803D34B484068F9
:10D58000192803D90120494988728EE000204749B3
:10D5900088728AE0FF2C01D1FF2D2DD10120434953
:10D5A00008720020487263204860FF2014306043F6
:10D5B000086008680A21FAF7C3FD3C49086008685A
:10D5C0006621FAF7BDFD39490860084600686328FE
:10D5D00001D96320086035480068112803D3334817
:10D5E0000068172804D90120304988725DE055E0B1
:10D5F00000202E49887258E063202C49086048605A
:10D6000000208872087248724FE001202749087292
:10D610004872FF2014306043086008680A21FAF756
:10D620008FFD2249086008686621FAF789FD1F49C5
:10D63000086008460068632801D963200860FF205D
:10D64000143068431949486048680A21FAF778FDA0
:10D650001649486048686621FAF772FD1349486028
:10D6600008464068632801D9632048600F48006875
:10D6700011280BD30D480068172807D80B484068BD
:10D68000112803D309484068192803D90120074904
:10D6900088720AE000200549887206E000200349EC
:10D6A0000872487208604860887270BD08090020DE
:10D6B000CC070020FFB583B006460D461746002470
:10D6C0000020029000BF1420784380190190002EA2
:10D6D00057D00198002854D02B4806602A49069854
:10D6E00048600846077200BF45E0FFF72FFD029033
:10D6F000200129580298814204D820012858401C52
:10D70000002806D1204902980A681421614350502C
:10D7100006E0200129581C4802681420604311507B
:10D72000200140194068401C002807D100211648FC
:10D730000268142060431018416008E0200140197D
:10D7400041681148026814206043101841602001AC
:10D75000401981680C480268142060431018C160A9
:10D7600020014019017B084802681420604310180A
:10D770000161601CC4B20448007AA042B5DC00F02C
:10D7800005F807B0F0BD0000181A002070B500249D
:10D7900000250026FFF7DAFC054600BF4EE02A48C8
:10D7A0000168142060430858A84239D82648016807
:10D7B0001420604308582E1A23480168142060433F
:10D7C0000818406881192048026814206043101826
:10D7D00081601D48016814206043081881681A4858
:10D7E0000268142060431018C068814224D916488A
:10D7F00001681420604308180069002803D02046FF
:10D80000FFF706F818E01048016814206043081874
:10D81000C1680D48026814206043101881600BE055
:10D8200009480168142060430818406806490A68DE
:10D830001421614351188860601CC4B20248007A08
:10D84000A042ACDC70BD0000181A002010B500BF6B
:10D8500014244C432318002805D0002B03D0024C7D
:10D8600020606260217210BD181A0020F8B50546CC
:10D870000E4614462B000EF0B5F8050412192027A9
:10D880002E001748FBF774F8164908701448FAF789
:10D890001FFD07466421FAF753FC30601CE0A0042A
:10D8A000020C31461020FBF75DF915E0A004020CD4
:10D8B00031463020FBF756F90EE0A004020C314649
:10D8C0005020FBF74FF907E0A004020C314670200E
:10D8D000FBF748F900E000BF00BF0020F8BD0000E2
:10D8E000061400208D00002070B505460E46144633
:10D8F0002B000EF077F805041C232A31380030681D
:10D90000002802D1FAF7D2FE10E0642231685143B8
:10D9100008461649FAF7E6FC00201549087001226E
:10D9200064211248FBF78CF9114908701CE0A0042F
:10D93000020C31461020FBF7D3FA15E0A004020CCC
:10D9400031463020FBF7CCFA0EE0A004020C314641
:10D950005020FBF7C5FA07E0A004020C3146702006
:10D96000FBF7BEFA00E000BF00BF70BDF813002057
:10D970008C00002000B5AFB050211BA8FAF790FC36
:10D9800000201A90142115A8FAF78AFC00201290A2
:10D99000139014901190402101A8FAF781FC002007
:10D9A0003F49086001221BA9FFF760FF1B98401C3C
:10D9B000002801D11A9001E01B981A90394815905F
:10D9C0003948169039481790002018903848199017
:10D9D00015AA1AA93748FFF76BFB02221CA90120E0
:10D9E000FFF744FF1C98401C002801D1129001E071
:10D9F0001C9812901C98401C002801D1139001E043
:10DA00001D9813902C48149012A92C48199AFFF7CE
:10DA100097FC08221EA90220FFF728FF1E98401C31
:10DA2000002801D1019001E01E9801901F980290FA
:10DA300023480390012069460874801E05902149FF
:10DA40000791012101A80177881E09901D490B91BA
:10DA5000012109A80173881E0D901A490F91012117
:10DA60000DA80173042201A91748199BFFF722FE94
:10DA700001221BA90320FFF7F9FE14491B98086037
:10DA80001B98401C002806D1FF20F53008600122B9
:10DA90000320FFF729FF0E48014908602FB000BDA1
:10DAA00090000020A5C5000099C500007DC50000BC
:10DAB000E9D800008C13002076841E009813002003
:10DAC0000F2700009F860100A8130020DC00002023
:10DAD000A33AA55A00B585B014216846FAF7E0FBD1
:10DAE00000200F4908600F4800900F4801900F4830
:10DAF0000290002003900E48049069460D48FFF7FD
:10DB0000AFFB0D480499FFF771FC04210B48049A00
:10DB1000FFF79CFE0A480249086005B000BD0000FE
:10DB200090000020A5C5000099C500007DC500003B
:10DB3000E9D800008C13002098130020A8130020BF
:10DB4000A33AA55A00200B4908800B4908800B49CD
:10DB5000088001200A49087000200A4908730A4910
:10DB6000088048800120087100200649488008800C
:10DB700070470000320000203400002036000020F2
:10DB800038000020BC0700203A000020FEB502F05B
:10DB900015F9009002F01CF90190FEF703FD012831
:10DBA0006BD10521D448FDF779F9552807D100201C
:10DBB000D2490870D2490880D249888067E001982C
:10DBC000012807D10020CD490870CD490880CD49F2
:10DBD00088805CE0C9480078002808D10120C74946
:10DBE0000870009D0A206843C54908804FE00098EE
:10DBF00081B2C448007B4200C248801D8152801F10
:10DC0000067B11E07100BF48801D455A701E41001F
:10DC1000BC48801D415A72008152701E4100B948B3
:10DC2000801D4552701EC6B2002E0ADD7100B54837
:10DC3000801D415A701E4200B248801D805A8142A8
:10DC4000E0DBB048007B401CAE4908730846007B0F
:10DC5000032807DB00200873084605890A2068436B
:10DC6000A74908800020A74908804880A448008868
:10DC700088800120A149087009E000209F490870B0
:10DC80009F4908809F4908804880087388809C4885
:10DC900005889D480088A84256D29B480088281ACB
:10DCA00084B299480079012826D197484088A0423B
:10DCB0000BDA95484088801C934948800846408884
:10DCC000A04204DD0846448001E08F4844808E482D
:10DCD000448803212046FAF749FA84B2022C00DA7C
:10DCE000022489480088001987490880084600886E
:10DCF000A84200D90D80CDE083484088062805DD84
:10DD000081484088801F8049488002E000207E4989
:10DD100048807D48448803212046FAF727FA84B2D8
:10DD2000022C03DA012078490871B3E076480088B4
:10DD3000A04205DD74480088001B73490880A9E0F3
:10DD4000002071490880A5E06F480088A84259D991
:10DD50006D480088401B84B26B480079012827D1A8
:10DD600069484088062805DD67484088801F664965
:10DD7000488002E0002064494880634844880321C9
:10DD80002046FAF7F3F984B2022C03DA02205E4946
:10DD900008717FE05C48008800195B4908800846EC
:10DDA00000885A49884275DD08465749088071E065
:10DDB00055484088A0420BDA53484088801C52499D
:10DDC000488008464088A04204DD0846448001E0BF
:10DDD0004D4844804C48448803212046FAF7C6F950
:10DDE00084B2022C00DA02244748008829198842AC
:10DDF00002D245490D804DE043480088001B42494E
:10DE0000088047E04048448803212046FAF7AEF9ED
:10DE100084B2022C3EDD3C484088062805DD3A48A5
:10DE20004088801F3849488002E0002036494880F9
:10DE30003548448803212046FAF798F984B23248DD
:10DE40000079012813D1022C03DA02202E4908712F
:10DE500020E02D48008800192B49088008460088DA
:10DE60002A49884216DD08462749088012E0022C1C
:10DE700003DA0120244908710CE023480088A042FD
:10DE800005DD21480088001B1F49088002E00020B2
:10DE90001D4908801C4800881D490988884203DA0A
:10DEA000194800880F2804DA1748008818490880A4
:10DEB0000AE01548008816490988081A0F2803DB6C
:10DEC0001148008812490880114807880B480078DB
:10DED00000280DD06C20474364213846FAF730F90A
:10DEE00007460A48874200D907460A490F8002E0E0
:10DEF000002008490880FEBDCC0700203800002023
:10DF000032000020BC0700203A000020C6070000B5
:10DF1000360000203400002000200749088007490F
:10DF200008800749088048800120087100200549C1
:10DF30004880088070470000340000203600002030
:10DF40003A000020BC070020002002490870024966
:10DF500008707047840000208500002010B5FEF78F
:10DF600021FB012813D103210C48FCF797FF55280A
:10DF700005D100200A4908700A4908700CE001F038
:10DF80006BFF0749087001200649087004E0002073
:10DF9000034908700349087010BD0000CC07002039
:10DFA0008400002085000020F0B5A9B004460E468C
:10DFB0000025002700202890A0216846FAF770F974
:10DFC000FFF7C4F826490A681421614350502448D9
:10DFD0000168142060430818C068B0420CD2204881
:10DFE0000168142060430818C1681D4802681420A5
:10DFF00060431018416005E019480168142060432F
:10E000000818466016484068002826D0002517E00A
:10E010006806070E282F00D316E011480168142067
:10E0200068430858B9006A4650500D4801681420EA
:10E03000684308184168781C80001150681CC5B2FC
:10E040000748007AA842E3DC00BF6A00044869463A
:10E0500043680220984701202890289829B0F0BDF5
:10E06000181A002010B500F0EDFD00F0D7F80CF004
:10E0700049FD00F00DFB00F001F810BD70B54148FE
:10E080000078912800D070BD00F0BEF8012876D14C
:10E090003D4800883D49088008468078F021884343
:10E0A00020303A49887008468078000900013549D7
:10E0B000097A0907090F0843344988703148807A82
:10E0C000401E3049887208460089401C0881084675
:10E0D0000089C988884216DA08202C4988720024F1
:10E0E0000EE0284841882848001D415C2748C01C94
:10E0F000015524484088401C22494880601CC4B215
:10E10000072CEEDB2DE01F4800891E49C988884294
:10E110001CD11C4800791B498978401AC5B2681C7B
:10E120001A49887200240EE0164841881648001DDE
:10E13000415C1648C01C015512484088401C1149DA
:10E140004880601CC4B2AC42EEDB0AE000F006FD81
:10E1500000200C4908700C490888092100F0B8F922
:10E1600091E7012000F0BCFC084A917A1088921CCB
:10E1700000F070F905490888002100F0C1F800BFDF
:10E1800081E700007C17002018170020A816002047
:10E190001B49097E002932D01949897E0C2251433E
:10E1A000174A515A174A118000200CE01449897E01
:10E1B0000C225143124A8918891C0A5C1149891C96
:10E1C0000A54411CC8B20828F0DB0D49897E0C2294
:10E1D00051430B4A8918897A0A4A91720121D172F6
:10E1E0000749097E491E064A11761146897E491C57
:10E1F00091761146897E022901DB002191767047D4
:10E20000741600209C1600200349487B012802D187
:10E210000021014A517370478C17002010B5334814
:10E220004068002861D13148007B03000DF0DAFB23
:10E2300007590512212E3D4A59002D480078002823
:10E2400007D000202A4908702A490888012100F0D7
:10E250003FF947E026480078002809D000202449EB
:10E26000087025494A8808880123091D00F040F9F3
:10E2700038E01F480078002807D000201C490870AB
:10E280001C490888022100F023F92BE01848007887
:10E29000002809D000201649087017494A880888C4
:10E2A0000923091D00F024F91CE01148007800281A
:10E2B00007D000200E4908700E490888092100F097
:10E2C00007F90FE00A480078002809D00020084923
:10E2D000087009494A8808880323091D00F008F9D5
:10E2E00000E000BF00BF00F039FC10BD8C1700201B
:10E2F0007C17002018170020B4160020704700007B
:10E3000070B504460D4634480088A04263D1002D04
:10E3100061D13248007822284ED004DC20283DD03C
:10E32000212856D141E0902802D0912851D115E002
:10E330002A48C08801280AD100202849087000F026
:10E340000DFC27490888002100F0C2F805E00320F1
:10E3500000F0C6FBA020214908703BE01F4800895F
:10E360001E49C98888420AD100201C49087000F063
:10E37000F5FB1B490888002100F0AAF80DE01748BA
:10E38000807A002806D000F0E9FB1449087B00F0F1
:10E3900089FB02E0032000F0A3FB1BE0062000F055
:10E3A0009FFB11200D49087014E0062000F098FB37
:10E3B00011200A4908700DE000200849087000F09B
:10E3C000CDFB08494A8808880923091D00F090F808
:10E3D00000E000BF00BF70BD901600207C17002039
:10E3E00018170020B416002070B50346184C247E80
:10E3F000022C00DB70BD164C647E0C256C43144D62
:10E400002B5300200AE0155C114C647E0C267443EB
:10E410000F4EA419A41C2554441CE0B28842F2D328
:10E420000B4C647E0C267443094EA419A172344629
:10E43000247E641C35462C762C46647E641C6C76E7
:10E440002C46647E022C01DB00246C7600BFD1E7F1
:10E4500074160020F0B585B007460D4616461A48DA
:10E460000780002406E031781748801C0155761C8F
:10E47000601CC4B2AC42F6DB2C4605E0AA2112486F
:10E48000801C0155601CC4B2082CF7DB0E480088C4
:10E49000019008216846C172002141720172017029
:10E4A000002406E00848801C015D03A80155601C9B
:10E4B000C4B2082CF6DB69460448FCF7F6FD0120DF
:10E4C0000149887205B0F0BD9016002090550440B7
:10E4D00070B504460D46294620460CF03FFA70BD43
:10E4E00070B504460D46294620460CF045FA70BD2D
:10E4F000F8B504460D4616461F463B4632462946A9
:10E5000020460CF03AFAF8BDF8B507460E46154617
:10E510005C480078002804D009213846FFF7D8FF6E
:10E52000F8BD002D01D0602D04DD09213846FFF72C
:10E53000CFFFF5E7544807804580002406E0317896
:10E540005148001D0155761C601CC4B2AC42F6DB7C
:10E5500000204C49487008468580FF2088727F2043
:10E5600008730846808808282EDA0120C8800846EB
:10E5700080884880012008814348008843490880FA
:10E5800008468078F02188434049887008468078A2
:10E59000000900013B4909790907090F08433B4974
:10E5A000887038480079401C8872002407E036489B
:10E5B000001D015D3548C01C0155601CC4B23148C6
:10E5C0008088A042F3DC4AE00721681CF9F7CEFD01
:10E5D000002907D0072128460830F9F7C7FD294947
:10E5E000C88005E00721681CF9F7C0FD2549C880EF
:10E5F00006202449488001200881234800882349B7
:10E60000088008468078F021884310301F498870C0
:10E6100008468078000900011A4989880905090F10
:10E6200008431A49887008464088FF210902884338
:10E63000144989880902FF22120211400843134934
:10E64000488008208872002407E00F48001D015D03
:10E650000E48001D0155601CC4B2062CF5DB0120DC
:10E6600000F03EFA094A917A1088921CFFF7F2FEF8
:10E67000902004490870054908880021FFF740FEF2
:10E6800000BF4DE77C17002018170020A8160020B7
:10E6900010B5FFF77DFD1448C07A002822D012483B
:10E6A00080780009002806D0012807D002280AD067
:10E6B000032810D10CE000F09DF90FE000F09EF867
:10E6C00000F05AFA0AE000F011F800F055FA05E0FF
:10E6D00000F000F902E0FFF711FE00BF00BF0020CC
:10E6E0000149C87210BD00009C16002010B54048BA
:10E6F0000078112800D010BD3E4800883F21490114
:10E70000884200D0F7E73B4880780007000F38497F
:10E71000097A0907090F88420CD000203449087093
:10E7200000F01CFA34494A8808880423091DFFF7C1
:10E73000DFFEE0E72E480089401C2D49088108468D
:10E74000807A401E887208460089C98888421BDA90
:10E750002848807A082800D0CDE700240EE025481C
:10E76000C01C015D224842882348001D8154204876
:10E770004088401C1E494880601CC4B2072CEEDB58
:10E78000062000F0ADF930E0194880881849498822
:10E79000401A1849897A884203DA1648807A08288C
:10E7A00000D0A8E700240EE01248C01C015D10480C
:10E7B00042881148001D8154601CC4B20C48408836
:10E7C000401C0B4948800A4840880949898888428A
:10E7D000EADB00200649087000F0C0F906494A88C3
:10E7E00008880023091DFFF783FE00BF83E70000B0
:10E7F0007C1700209C160020B416002070B532480B
:10E80000007880210840802800D170BD2F48008802
:10E810003F214901884200D0F7E72C48807A082838
:10E8200000D0F2E72948807805072D0F2D022748F0
:10E830004088000A0543082D00DAE6E70020224957
:10E8400048700620488008468580012008810820FD
:10E8500088720020C8728988481C0721F9F786FC55
:10E86000002909D018498988084608300721F9F796
:10E870007DFC1549C88007E013498988481C072199
:10E88000F9F774FC1049C8801048008810490880C6
:10E8900008464580002407E00C48001D015D0C4837
:10E8A000001D0155601CC4B2062CF5DB042000F0ED
:10E8B00017F9102004490870054A51881088FFF79D
:10E8C0000FFE00BFA1E700007C1700209C1600206F
:10E8D000B416002010B544480078A02808D042485B
:10E8E0000078912804D040480078A12800D010BDBD
:10E8F0003E4800883F21490188420AD03C490888A7
:10E900000921FFF7E5FD00F029F9002036490870DC
:10E91000EDE73648807A08280AD035490888092169
:10E92000FFF7D6FD00F01AF900202F490870DEE746
:10E930002E4880780007000F002804D0012825D039
:10E94000022843D12EE028484078002800D048E033
:10E950002648C078002803D101202349487003E0ED
:10E960002248C078204988721F480078912803D037
:10E970001E4800791C49087391201B49087000F05B
:10E98000EDF81949087B00F08DF82AE01648407828
:10E99000002800D025E0A12013490870032000F0D2
:10E9A0009FF81EE010484078002800D019E00E487B
:10E9B0000078A02809D10E4908880821FFF788FDB2
:10E9C00000F0CCF80020084908700AE008490888DF
:10E9D0000521FFF77DFD00F0C1F800200249087015
:10E9E00000BF00BF00BF82E77C1700209C160020FC
:10E9F0001817002010B5284800788021084080288A
:10EA000000D110BD24480078002806D02348008893
:10EA10003F214901884200D0F3E72048807A1F490E
:10EA200089780907090F884203DD1C48807A082885
:10EA300000D0E6E7194880780007000F002805D0CD
:10EA4000164880780007000F072800DDD9E7134833
:10EA5000008813490880114880780007000F48801B
:10EA6000002407E00D48C01C015D0D48001D015544
:10EA7000601CC4B20A484088A042F3DC002006496A
:10EA8000087000F06BF806494A8808880023091DC1
:10EA9000FFF72EFD00BFB4E77C1700209C16002076
:10EAA000B41600207F2805DC7D21C90041430A4AB5
:10EAB00091600DE0F12808DBF92806DC0107090F59
:10EAC00064225143044A916002E00449024A916081
:10EAD0000221014A517370478C17002018F0010081
:10EAE00000B503000CF07EFF0729050B11171D234D
:10EAF00029000121144A11731449516022E00221B6
:10EB0000114A1173114951601CE003210E4A11731F
:10EB10000F49516016E004210B4A11730D495160F1
:10EB200010E00521084A1173002151600AE0062116
:10EB3000054A11730849516004E00021024A11732B
:10EB4000516000BF00BF00BD8C170020A86100000D
:10EB5000F824010028230000F049020000200149A8
:10EB6000087370478C170020024909880918014A68
:10EB7000118070478C17002010B52F48007810289E
:10EB800018D12E48408860280ADD2D488078000979
:10EB90000001801C2A49887022202749087025E03E
:10EBA00027488078000900012549887020202249E3
:10EBB00008701BE020480078112816D11E48807A82
:10EBC000002800D010BD1C484078002800D0F9E78C
:10EBD0000820194988721A488078000900011849EC
:10EBE000887020201449087000E0EBE7FD20C00089
:10EBF0001349088008468078F02188433030104956
:10EC000088700846C0780020C87008460079142033
:10EC10000871032088720220FFF762FF084A917A88
:10EC20001088921CFFF716FC054908880021FFF7A1
:10EC300067FB00BFC6E700007C170020B416002069
:10EC4000A8160020244A118852888A4242D0224ABB
:10EC500052888A4204DA204A52888A1A90B207E01F
:10EC60001D4A52880023DB439A1A521C521890B254
:10EC7000194A5180127B002A10D0174A5268002A84
:10EC80000CD0154A5268824205D9134A5268121AAA
:10EC9000114B5A6002E000220F4B5A600E4A527B21
:10ECA000022A17D10C4A9268002A0CD00A4A9268AC
:10ECB000824205D9084A9268121A074B9A6002E00C
:10ECC0000022054B9A60044A9268002A02D1012270
:10ECD000014B5A73704700008C17002010B505F0E7
:10ECE0006FFB10BD00BF704710B504468020204365
:10ECF00001460320400205F01DFA10BD10B5102199
:10ED00000320400205F016FA10BD000010B50224E1
:10ED1000024805F05FFA0446204610BD01060000D7
:10ED200010B50021014805F005FA10BD01060000EC
:10ED300010B50446802020430146024805F0FAF948
:10ED400010BD00000106000010B51021014805F0BB
:10ED5000F1F910BD0106000030B503460C46002154
:10ED6000002000BF07E08D0065599D4201D10120C0
:10ED700003E04D1CE9B29142F5DB00BF30BDF8B5B0
:10ED800005460E4600240EE0601CC7B207E0BA003C
:10ED90005119A200501900F00AF8781CC7B2B74206
:10EDA000F5DB601CC4B2701EA042EDDCF8BD10B5EE
:10EDB00003680C68A34204D90B889AB203680B60FD
:10EDC000026010BD70B505460024002600BF0AE0B1
:10EDD0000848005D295D884203D00126285D054969
:10EDE0000855601CC4B2082CF2DB002E01D000F0E4
:10EDF00003F870BD73000020FEB500260027002038
:10EE00000290019000240025009001F039F8064698
:10EE100001F04AF8074601F03DF8029001F04EF883
:10EE2000019001F023F86B490870F0203040001188
:10EE30000A2805DBF02030400011C01C044303E029
:10EE4000F02030400011044324023007000F0A284C
:10EE500004DB3007000FC01C044302E03007000F42
:10EE600004432402F020384000110A2805DBF0207A
:10EE700038400011C01C044303E0F020384000116A
:10EE8000044324023807000F0A2804DB3807000F68
:10EE9000C01C044302E03807000F0443F02102982D
:10EEA000084000110A2805DB029808400011C01C28
:10EEB000054304E0F02102980840001105432D02AB
:10EEC00002980007000F0A2805DB02980007000FD0
:10EED000C01C054303E002980007000F05432D0204
:10EEE000F0210198084000110A2805DB019808402C
:10EEF0000011C01C054304E0F021019808400011F6
:10EF000005432D0201980007000F0A2805DB019830
:10EF10000007000FC01C054303E001980007000F25
:10EF200005432D4802782D492046FFF715FF00289C
:10EF300007D02948027829492846FFF70DFF002805
:10EF400002D1002026490860254800682149097837
:10EF500088422AD22048027820492046FFF7FCFE4A
:10EF6000002807D01C4802781C492846FFF7F4FE09
:10EF7000002815D11A4801680068401C184A106022
:10EF8000880016490C50104601680068401C10604B
:10EF9000880012490D50104801781048FFF7EFFE25
:10EFA0000F4800780C49087003E00A4800780A49C5
:10EFB000087009480078009007E00A49009880002E
:10EFC000064A11500098401C009000984828F4D33D
:10EFD000FEBD00007000002072000020041100201F
:10EFE00080000020FFFF00002E480078401C2D49C3
:10EFF00008702D480078401C2B4908702B48007879
:10F00000401C2A4908702A480068401C28490860AA
:10F0100008460068FF219131884202D90020244926
:10F02000086020480078C82802D900201D490870CF
:10F030001D480078842802D900201B4908701B480D
:10F040000078502802D9002018490870194818493A
:10F050000968405C18490870184812490978405CF2
:10F0600017490870174810490978405C164908701C
:10F0700016480E490978405C154908701548094939
:10F080000978405C14490870144806490978405CC6
:10F0900013490870134803490978405C1249087005
:10F0A00070470000C3060020C4060020C5060020EB
:10F0B000C80600201FCC0100BC060020AFCD010017
:10F0C000BD06002077CE0100BE060020C3CF0100A0
:10F0D000C0060020FBCE0100BF06002013D00100B7
:10F0E000C1060020DBD00100C206002010B5044696
:10F0F000204600F049FA204600F002F810BD00005A
:10F1000010B50446B148007800287DD1B048008889
:10F11000B049884278DAB048007800284FD0AF482C
:10F120000078002803D0AA480088AD490880AD487F
:10F130000078002818D1A6480188A948008819300D
:10F14000814206D30120A7490870A1480088A4493C
:10F1500008809F480088A249098888421CDA9C4898
:10F1600000889F49088017E09D48018898480088DA
:10F170001930814206D300209A49087094480088CB
:10F18000974908809248008895490988884203DD9C
:10F190008F4800889249088092480078002857D10B
:10F1A00091480078042803D08C480078002807D0C4
:10F1B00087480088822803DA05208B490870A1E07F
:10F1C00089480078032803D084480078002809D0B3
:10F1D0007F480088FF211931884203DA04208249E0
:10F1E00008708FE080480078022803D07B480078C0
:10F1F00000280AD076480088FF21AF31884204DA1F
:10F200000320794908707DE0DFE077480078012825
:10F2100003D072480078002808D06D4800887349F0
:10F22000884203DA0220704908706BE06E4800786B
:10F23000002803D069480078002863D0644800881B
:10F240003721090188425DDA01206749087059E0D9
:10F2500064480078012855D163480078012803D01C
:10F260005E480078002809D05948008837210901F4
:10F27000884203DB00205C49087043E05A4800786C
:10F28000022803D055480078002808D0504800884C
:10F290005649884203DB01205349087032E0524846
:10F2A0000078032803D04D480078002809D048484A
:10F2B0000088FF21AF31884203DB02204A490870F1
:10F2C00020E049480078042803D04448007800280A
:10F2D00009D03F480088FF211931884203DB032011
:10F2E000414908700EE040480078052803D03B48AB
:10F2F0000078002806D036480088822802DB0420E7
:10F3000039490870FDF734F9394988425DD33948E5
:10F31000008800193749088030480078002808D054
:10F3200000202E490870334908802F480078324960
:10F33000087000F0F7FC00281FD12E4800882F49E4
:10F34000884239DB00202B4908802B480078264969
:10F350000978884205DA28480078401C2649087058
:10F360002AE02548007820490978884224DD22488F
:10F370000078401E204908701EE01E480088204981
:10F38000884219DB00201B4908801B480078164979
:10F390000978884205DA18480078401C1649087038
:10F3A0000AE01548007810490978884204DD1248BF
:10F3B0000078401E104908700F4800780A49097803
:10F3C000884202D100200B49088010BD0B000020AC
:10F3D000020000201027000012000020080000207A
:10F3E000040000200A000020060000207602000031
:10F3F000B80B00001800002007000020C05D0000CE
:10F40000407E050000200B4908700B490870012060
:10F410000A4908700A49087000200A4908700A4918
:10F4200008700A4908800A4908800A4908800A4980
:10F430000870704706000020070000200800002028
:10F44000090000200A0000200B0000200C00002012
:10F450000E000020100000201200002000200B49A8
:10F4600008700B49087001200A4908700A490870A1
:10F4700000200A4908700A4908700A4908800A49A8
:10F4800008800A4908800A49087070470600002071
:10F490000700002008000020090000200A000020CA
:10F4A0000B0000200C0000200E00002010000020A7
:10F4B00012000020F1B500272D480078002804D064
:10F4C0000320F9F749FF2B4908802B4800881928A9
:10F4D00047D300202849088028480078142829D2DA
:10F4E0000320F9F739FF0746002407E060002449AC
:10F4F000085AB84200DD05E0601CC4B21F4800781D
:10F500008442F3DB00BF1D48057808E0681E400018
:10F510001B49085A69001A4A5052681EC5B2A542D2
:10F52000F4DC600016490F5214480078401C13495F
:10F53000087016E00026052405E060001049085A0E
:10F540008619601CC4B20F2CF7D30A213046F8F795
:10F55000F7FD084908800020084908700120094982
:10F560000870054801880098081803490880F8BD0C
:10F5700009000020020000201600002000000020EA
:10F58000880700201200002023490988234A91425D
:10F590002BDB0021224A1180224A1180224909884E
:10F5A000AF221201914207DC20490978002916D0C8
:10F5B0001D490988914212DD02211D4A1170002166
:10F5C0001C4A117005211C4A11700021174A117044
:10F5D00001211A4A11700021194A11701AE01249CA
:10F5E00009880918104A118014E000210C4A118082
:10F5F0000D4A11800B490988124A914205DD00210C
:10F600000B4A1170094A117004E00649098809186B
:10F61000044A1180704700000200002010270000FB
:10F620000E0000200C000020100000200900002027
:10F630000B0000200600002007000020080000202A
:10F640000A000020B80B0000014800787047000055
:10F65000FC0800200148007A70470000FC080020E8
:10F660000148807870470000FC08002001480088AD
:10F67000704700006C000020F8B5002300250095BD
:10F680000024002200BF94E001259D40ACB20D880B
:10F6900025400095009DA5426FD11A468D79012D18
:10F6A0000DD1464D03263602AD192D5C012696403C
:10F6B0003543424E03273F02F61935540CE03F4DC7
:10F6C00003263602AD192D5C01269640B5433B4E0C
:10F6D00003273F02F6193554CD78002D4ED1374D12
:10F6E00060352D5CCE78002E01D1012600E0002689
:10F6F0009640B543314E603635548D78002D2ED16D
:10F700002E4D19267601AD192D5C8E78002E01D173
:10F71000012600E000269640B543284E19277F01B8
:10F72000F61935540D79002D0ED1244D50352D5C30
:10F730000E79002E01D1012600E000269640B54347
:10F740001E4E5036355423E01C4D50352D5C0E793D
:10F7500096403543EEB2194D50352E5418E0174DF2
:10F7600019267601AD192D5C8E7896403543134EDF
:10F7700019277F01F61935540AE018E00F4D60355E
:10F780002D5CCE7896403543EEB20C4D60352E544C
:10F790004D79012D0AD1094D30352D5C0126964059
:10F7A0003543EEB2054D30352E5400E000BF5D1CF0
:10F7B000ABB2082B00DA67E7F8BD00000000044098
:10F7C000FFB5074615461E4600243846019900F04D
:10F7D0001FF8002802D0012004B0F0BD00240CE086
:10F7E0000A2060430949085CB04204D129462046FA
:10F7F00000F05EF807E0601C84B20A206043034911
:10F80000085C0028ECD100BF0020E5E720010020C3
:10F810000246002A03D1402901DD01207047032A56
:10F8200003D1022901DD0120F8E7042A03D12029B0
:10F8300001DD0120F2E7052A03D1202901DD0120A5
:10F84000ECE70C2A03D1102901DD0120E6E70D2A9F
:10F8500005D1012903DD402901DA0120DEE70E2A66
:10F8600003D1202901D10120D8E70020D6E70000EC
:10F8700010B5064A03231B02D218125C8A43034BBD
:10F88000032424021B191A5410BD00000000044078
:10F8900010B5064A03231B02D218125C0A43034B1D
:10F8A000032424021B191A5410BD00000000044058
:10F8B00070B502460020B1E00A2353435A4C1B198D
:10F8C0005B1C440004191B199B788B427DD10A23D1
:10F8D0005343554C1B195B1C440004191B195B78DE
:10F8E000082B33D10A2353434F4C1B195B1C440094
:10F8F00004191B574D4C4E4D6419E35C01242343FE
:10F900000A245443484D6419641C45004519645742
:10F91000464D474EAD192B550A235343424C1B19F4
:10F920005B1C440004191B57404C35466419E35CCA
:10F93000022423430A2454433B4D6419641C4500AC
:10F9400045196457394DAD192B5564E00A235343CB
:10F95000354C1B195B1C440004191B195B78092BDF
:10F9600034D10A235343304C1B195B1C4400041947
:10F970001B572E4C2E4D6419E35C402423430A246C
:10F980005443294D6419641C450045196457274D9B
:10F99000274EAD192B550A235343234C1B195B1CCF
:10F9A000440004191B57214C35466419E35C80243C
:10F9B000A3430A2454431C4D6419641C4500451993
:10F9C00064571A4DAD192B5525E025E00A23534302
:10F9D000154C1B195B1C440004191B57134C144D88
:10F9E0006419E35C0A2454430F4D6419641C4500F8
:10F9F0004519641965780124AC402343DCB20A231D
:10FA00005343094D5B195B1C450045195B57074D76
:10FA1000074EAD19EC5404E0431CD8B2032800DAB9
:10FA20004AE700BF70BD0000200100200000044034
:10FA300075080000F8B50024FCF7B4FD012861D179
:10FA400000F0D0FA044664220721002002F040FEB4
:10FA5000012C21D100F044FB00280ED000F0F6FA72
:10FA6000054600F0E7FA064601200346024629460D
:10FA70000090304604F0FEFC50E000F0E7FA054646
:10FA800000F0D8FA064601200023024629460090DD
:10FA9000304604F0EFFC41E0022C21D100F020FBC5
:10FAA00000280ED000F0D2FA054600F0C3FA064650
:10FAB00001200346024629460090304604F0DAFC55
:10FAC0002CE000F0C3FA054600F0B4FA0646002028
:10FAD00001231A4629460090304604F0CBFC1DE075
:10FAE00000F0FEFA054600F0B1FA064600F0A2FA70
:10FAF0000746012003462A4631460090384604F066
:10FB0000B9FC0BE00020034602460146009004F0D9
:10FB1000B1FC00220721104602F0DAFDF8BD00001A
:10FB2000FEB547480078012809D1FCF73BFD0128C4
:10FB300002D1FCF76DFB82E0FCF79AFC7FE0FCF75A
:10FB400031FD012879D1FCF713FD3E49884271D37C
:10FB50003D480088032805DA3B480088401C3A49A4
:10FB6000088011E000203849088000F069FA054655
:10FB700000F084FA06460A21F8F7E2FA04462A461B
:10FB80002146012007F0A2FF00F09EFB054600F091
:10FB900059FB07460A21F8F7D3FA044600F050FA59
:10FBA00006462A46214606F003FAFFF743FF00F017
:10FBB0000DFA04462146012005F0DEFF00F058FA58
:10FBC0000546FF21F531F8F7D1FAC4B221460120EC
:10FBD00005F00EFCFFF738FD0446FFF747FD05462C
:10FBE000FFF73EFD064623462A463146012004F033
:10FBF0001BFF00F09DF804462146012008F00CFA96
:10FC000000F03AFB044600F077FA054600F02AFAC5
:10FC1000064600F037FB074600F074FA33463A46D2
:10FC20000146009501940290012007F09FFA06E03A
:10FC300003E0FFE7FCF75CFB01E0FCF719FCFEBD0D
:10FC4000B5000020B80B00006600002001490860E4
:10FC500070470000F006002002480068401C01497F
:10FC600008607047EC060020F3B581B0064600201E
:10FC70000E49086000F01EF8044600F01BF8054627
:10FC80002F1B3046029903F0B9FC00900AE000F007
:10FC900011F805462F1B06480068002802D00448CA
:10FCA0000068804700988742F1D3FEBDEC06002033
:10FCB000F00600200148006870470000EC060020B4
:10FCC0000B490978012901D101200FE00849097881
:10FCD000022901D1022009E005490978032901D14F
:10FCE000042003E00121024A117001207047000046
:10FCF0008506002010B5094B1B8899B20A12C8B2BC
:10FD0000D3433133064C2370C3432333637013460C
:10FD10005633A37003467133E37010BDB406002060
:10FD20008B06002001480088704700003200002048
:10FD300001480078704700008400002001480078E6
:10FD4000704700008500002010B5002205210648FC
:10FD5000FBF792F80402012205210348FBF78CF817
:10FD6000201880B210BD0000CC07002010B506227C
:10FD700005210348FBF780F8C006C00F10BD000046
:10FD8000CC07002010B5042205210648FBF774F8C3
:10FD90000402052211460348FBF76EF8201880B2D2
:10FDA00010BD0000CC07002010B506220521024836
:10FDB000FBF762F8C01110BDCC07002010B502227D
:10FDC00005210248FBF758F810BD0000CC070020C1
:10FDD00010B5062205210348FBF74EF88006C00F38
:10FDE00010BD0000CC07002010B5042202210348FA
:10FDF000FBF742F8C007C00F10BD0000CC07002081
:10FE000010B5052202210348FBF736F8C007C00FE2
:10FE100010BD0000CC07002010B5002204210348CB
:10FE2000FBF72AF84006400F10BD0000CC07002069
:10FE300010B5002201210248FBF71EF810BD00009A
:10FE4000CC07002010B5012211460248FBF714F838
:10FE500010BD0000CC07002010B50222032102488B
:10FE6000FBF70AF810BD0000CC07002010B50322F4
:10FE700000210248FBF700F810BD0000CC0700206D
:10FE800010B5002211460248FAF7F6FF10BD000037
:10FE9000CC07002010B5042200210248FAF7ECFF3D
:10FEA00010BD0000CC07002010B50122002102483F
:10FEB000FAF7E2FF10BD0000CC07002010B50522C4
:10FEC00000210248FAF7D8FF10BD0000CC0700203F
:10FED000322815DA3C498978012903DD01213A4AA3
:10FEE000517070E038498978002905DD2F286ADCD7
:10FEF0000021354A517066E00021334A517062E0BA
:10FF00003E2817DA322815DB2F498978022903DDCC
:10FF100002212D4A517056E02B498978012905DDCF
:10FF20003B2850DC0121284A51704CE00121264A2F
:10FF3000517048E0502817DA3E2815DB22498978AD
:10FF4000032903DD0321204A51703CE01E498978D2
:10FF5000022905DD4D2836DC02211B4A517032E0B2
:10FF60000221194A51702EE0622817DA502815DB59
:10FF700015498978042903DD0421134A517022E0D0
:10FF800011498978032905DD5F281CDC03210E4A0D
:10FF9000517018E003210C4A517014E073280FDAF5
:10FFA00062280DDB08498978042905DD70280ADC00
:10FFB0000421054A517006E00421034A517002E011
:10FFC0000521014A51707047FC0800200148007863
:10FFD00070470000070000200148007870470000CB
:10FFE000A40000200148007870470000A300002012
:10FFF000F8B5002600240025FDF7F2F907460A218E
:020000040001F9
:10000000F8F79EF8054609480068854200D303E0EA
:1000100006480068461B34467D200001844200D318
:100020000446034804600068F8BD0000DC000020BE
:10003000D80000200148007870470000AD00002083
:1000400001480079704700009C000020014840787A
:1000500070470000AD000020014880797047000023
:100060009C00002001484079704700009C0000205F
:1000700001480088704700002200002010B50024CD
:10008000FFF7DEFF00280AD10A4800880A498842A3
:1000900002DB0846074908800648048808E005484E
:1000A0000088FCF74BFF84B20448844200DB04461E
:1000B000204610BD34000020C6070000CE0400001A
:1000C000002005490988054A914202DB1146024A8F
:1000D000118001490888704734000020C6070000DD
:1000E0000148007870470000BD06002001480078F4
:1000F00070470000BF0600200148007A70470000EA
:100100000809002070B500240B48C07A01280DD1E1
:100110000949098888B2FCF767FB05460A21F8F708
:1001200025F884B2632C04DD632402E002480088D1
:1001300084B2204670BD00000809002001480088F4
:1001400080B270470809002010B500240A21034836
:100150000088F8F70BF884B2204610BD020000209A
:1001600001480078704700000B00002010B5002403
:10017000044804F02FF8002801D0012400E00024F6
:10018000204610BD0307000010B50024054804F008
:1001900021F8002802D00120044601E00020044696
:1001A00010BD00000507000010B50024054804F04C
:1001B00011F8002802D00120044601E00020044686
:1001C00010BD00000707000010B50024062004F051
:1001D00001F8002801D0012400E00024204610BDD1
:1001E00010B50024054803F0F5FF002802D00120D7
:1001F000044601E00020044610BD00000607000090
:1002000010B50024044803F0E5FF002801D00124C4
:1002100000E00024204610BD0305000010B50024B6
:10022000044803F0D7FF002801D0012400E0002497
:10023000204610BD040500000148807A7047000088
:100240000809002070B50024FFF7FAFE002803D14A
:10025000FDF7C6F804460DE0FFF7F2FE012806D1CF
:10026000FDF7BEF80546FCF769FE044602E0FDF71F
:10027000B7F80446204670BD0148407A7047000038
:100280000809002070B500240B48C07A01280DD160
:100290000949898888B2FCF7A7FA05460A21F7F7C9
:1002A00065FF84B2632C04DD632402E00248808889
:1002B00084B2204670BD00000809002001488088F3
:1002C00080B270470809002070B50024FFF7B8FE1F
:1002D000002803D1FDF796F804460FE0FFF7B0FEC3
:1002E000012807D10020FDF78DF80546FCF726FE12
:1002F000044603E00020FDF785F80446204670BD63
:1003000001480078704700003800002070B50546AD
:100310000024032D00D170BD002D01D0012D1BD173
:1003200081210320800203F005FF8021134803F0A0
:1003300001FF32211248FFF797FC002409E0A200D8
:10034000104BD2189178A200985A03F0F3FE601C6B
:10035000C4B23B2CF3DB0FE0022D0DD1002409E0E9
:10036000A200094BD2189178A200985A03F0E2FE3D
:10037000601CC4B23B2CF3DB00BFCCE702060000DC
:10038000A0860100B8C40100A4C50100F8B5002191
:1003900000240023002200BF0AE001258D40ABB2FB
:1003A00005881D402C469C4200D10A464D1CA9B22E
:1003B0001029F2DB0588FF2D1FDC284D6D7E068895
:1003C000B543264E757635462D7E0688B543234EB9
:1003D000357635466D7E8678F607F60F96403543BE
:1003E0001E4E757635462D7E867802273E4076086D
:1003F00096403543194E357622E0184DED7E06883D
:10040000B543164EF5763546AD7E0688B543134E98
:10041000B5768578ED07ED0F1646083EB5400F4ED0
:10042000F67E35430D4EF5768578022635406D080B
:100430001646083EB540094EB67E3543074EB576A2
:100440000025009505E000BF6D462D786D1CEEB2CD
:1004500000966D462D78012DF5D9F8BD206B04402E
:10046000C107C90F002905D00021394A11710022A6
:1004700038490A7102210140002905D00021344A7F
:100480001172002233490A7204210140002905D06B
:1004900000212F4A117300222E490A7308210140BE
:1004A000002905D000212A4A1174002229490A7422
:1004B00010210140002905D00021254A1175002294
:1004C00024490A7520210140002905D00021204A35
:1004D000117600221F490A7640210140002904D0EC
:1004E00000221B494A711B494A71802101400029A1
:1004F00004D0002216494A7216494A72FF2101317E
:100500000140002904D0002211494A7311494A735D
:10051000012149020140002904D000220C494A74FB
:100520000C494A74012189020140002904D00022AB
:1005300007494A7507494A750121C9020140002946
:1005400004D0002202494A7602494A7670470000E8
:100550000060004000610040C107C90F002905D0BC
:1005600001223C490A7100213B4A117102210140DC
:10057000002905D0012237490A720021364A11723A
:1005800004210140002905D0012232490A730021CB
:10059000314A117308210140002905D001222D495B
:1005A0000A7400212C4A117410210140002905D041
:1005B000012228490A750021274A1175202101408E
:1005C000002905D0012223490A760021224A11760A
:1005D00040210140002905D001221E494A71002214
:1005E0001D494A7180210140002905D00122194985
:1005F0004A72002218494A72FF2101310140002944
:1006000005D0012213494A73002213494A7301217C
:1006100049020140002905D001220E494A740022F6
:100620000D494A74012189020140002905D00122A7
:1006300008494A75002208494A750121C90201404A
:10064000002905D0012203494A76002202494A7650
:1006500070470000006100400060004010B50C4889
:100660000078002803D00B4A5068916888470848F2
:100670004078002803D0084A5068916888470448A9
:100680008078002803D0054A50689168884710BDDB
:100690000060004070020020F00300207005002080
:1006A00010B508480079002803D0074A106951693D
:1006B000884704484079002803D0044A506891686C
:1006C000884710BD0060004070020020FC0300203D
:1006D00010B50848007A002803D0074AD069116A8B
:1006E00088470448407A002803D0044A506891683B
:1006F000884710BD00600040700200200804002000
:1007000010B50848007B002803D0074A906AD16AD8
:1007100088470448407B002803D0044A5068916809
:10072000884710BD006000407002002014040020C3
:1007300010B50848007C002803D0074A506B916B25
:1007400088470448407C002803D0044A50689168D8
:10075000884710BD00600040700200202004002087
:1007600010B50848007D002803D0074A106C516C72
:1007700088470448407D002803D0044A50689168A7
:10078000884710BD00600040700200202C0400204B
:1007900010B50848007E002803D0074AD06C116DC0
:1007A00088470448407E002803D0044A5068916876
:1007B000884710BD0060004070020020380400200F
:1007C00010B50848407F002803D0074A5068916858
:1007D00088470448007F002803D0044A906DD16DFB
:1007E000884710BD006000404404002070020020D3
:1007F00010B508484078002803D0074A506891682F
:10080000884704480078002803D0044A506E916E4F
:10081000884710BD20600040500400207002002076
:1008200010B509480079002803D0084A106F516FAD
:1008300088470548001D4078002803D0044A5068C6
:100840009168884710BD00002060004070020020C1
:100850005C04002010B5034AD06F78329168884755
:1008600010BD00007002002010B5024A5068916867
:10087000884710BDF402002010B50948007C00280C
:1008800003D0084A5068916888470548103040787E
:10089000002803D0044A50689168884710BD0000C2
:1008A00020600040000300208004002010B5024AB0
:1008B00050689168884710BD0C03002010B5024AAB
:1008C00050689168884710BD1803002010B509488A
:1008D000007F002803D0084A50689168884705487F
:1008E0001C304078002803D0044A5068916888473B
:1008F00010BD00002060004024030020A40400205C
:1009000010B50C480078002803D00B4A5068916855
:10091000884708484078002803D0084A5068916802
:10092000884704488078002803D0054A50689168B9
:10093000884710BD4060004030030020B004002014
:100940003006002010B50D480079002803D00C4A6D
:100950005068916888470948001D4078002803D0F6
:10096000084A5068916888470448001D807800282C
:1009700003D0054A50689168884710BD4060004028
:100980003C030020BC0400203C06002010B50D48AC
:10099000007A002803D00C4A5068916888470948BB
:1009A00008304078002803D0084A5068916888478A
:1009B000044808308078002803D0054A50689168C0
:1009C000884710BD4060004048030020C804002054
:1009D0004806002010B50D48007B002803D00C4AC3
:1009E00050689168884709480C304078002803D047
:1009F000084A50689168884704480C30807800287D
:100A000003D0054A50689168884710BD4060004097
:100A100054030020D40400205406002010B50D48D3
:100A2000007C002803D00C4A506891688847094828
:100A300010304078002803D0084A506891688847F1
:100A4000044810308078002803D0054A5068916827
:100A5000884710BD4060004060030020E004002093
:100A60006006002010B5024A50689168884710BDA2
:100A70006C03002010B50948007E002803D0084A06
:100A8000506891688847054818304078002803D09E
:100A9000044A50689168884710BD000040600040DB
:100AA00078030020F804002010B50948007F0028D2
:100AB00003D0084A50689168884705481C30407840
:100AC000002803D0044A50689168884710BD000090
:100AD00040600040840300200405002010B5084851
:100AE0000078002803D0074A506891688847044876
:100AF0004078002803D0044A50689168884710BDA8
:100B000060600040900300201005002010B50948E7
:100B10000079002803D0084A506891688847054842
:100B2000001D4078002803D0044A50689168884727
:100B300010BD0000606000409C0300201C050020E8
:100B400010B50948007A002803D0084A5068916817
:100B50008847054808304078002803D0044A506888
:100B60009168884710BD000060600040A803002025
:100B70002805002010B5024A50689168884710BDCA
:100B8000B403002010B5024A50689168884710BD30
:100B9000C003002010B50948007D002803D0084A92
:100BA000506891688847054814304078002803D081
:100BB000044A50689168884710BD0000606000409A
:100BC000CC0300204C05002010B50948007E002809
:100BD00003D0084A50689168884705481830407823
:100BE000002803D0044A50689168884710BD00006F
:100BF00060600040D80300205805002010B5094867
:100C0000007F002803D0084A50689168884705484B
:100C10001C304078002803D0044A50689168884707
:100C200010BD000060600040E40300206405002067
:100C300010B5FE4800688079002806D001286ED0E3
:100C400002286DD003286CD104E2F848006840798E
:100C500003000AF0C7FE0A0614BC2BBC47BC67BCE5
:100C60009BBC07F019FD0020F0490968C873EF48E4
:100C700000684079401CED4909684871AEE0EC49D4
:100C80000969EA4A1268D27A885C07F07DFDE74874
:100C900000684079401CE54909684871E3480068EC
:100CA0004079401CE1490968487197E001F078FEFD
:100CB000002810D107F068FDDC4800684079401C2E
:100CC000DA4909684871D94800684079401CD74919
:100CD0000968487105E007F009FD0020D34909685B
:100CE00048717BE001F05CFE002811D1012007F083
:100CF0004BFDCE4800684079401CCC4909684871DA
:100D0000CA4800684079401CC8490968487105E034
:100D100007F0ECFC0020C549096848715EE05FE01F
:100D2000FEE0A3E101F03CFE002828D1BF4909689C
:100D3000C97A24225143BF4A12688918BB4A1268F3
:100D4000D27B885C07F020FDB8480068C07B401C5F
:100D5000B6490968C873B5480068C07B242814D315
:100D6000B24800684079401CB04909684871AF48F2
:100D700000684079401CAD490968487105E007F0FA
:100D8000B5FC0020A9490968487127E001F008FE78
:100D9000002815D1A5480068C07A401CA3490968FD
:100DA000C872A2480068C07AA1490978884207DB66
:100DB00000209E490968C87201209C490968887111
:100DC00007F094FC002099490968487106E007F093
:100DD0008DFC002095490968487100BF00BF4FE1B4
:100DE00092480068407903000AF0FCFD0805139161
:100DF0002A914791709107F04FFC00208B490968B8
:100E0000C8738A4800684079401C8849096848715D
:100E100084E087490969854A1268D27A885C07F0BC
:100E2000B3FC824800684079401C804909684871D9
:100E30007E4800684079401C7C49096848716DE033
:100E400001F0AEFD002811D1262007F09DFC774867
:100E500000684079401C754909684871734800680A
:100E60004079401C71490968487105E007F03EFC73
:100E700000206E490968487150E001F091FD00289A
:100E80001DD1012007F080FC68480068C07B401C31
:100E900066490968C87365480068C07B242814D374
:100EA000624800684079401C6049096848715F48A1
:100EB00000684079401C5D490968487105E007F009
:100EC00015FC002059490968487127E001F068FDC8
:100ED000002815D155480068C07A401C534909685C
:100EE000C87252480068C07A51490978884207DBC5
:100EF00000204E490968C87202204C49096888716F
:100F000007F0F4FB002049490968487106E007F042
:100F1000EDFB002045490968487100BF00BFAFE004
:100F200042480068407903000AF05CFD0805138B15
:100F30002A8B478B638B07F0AFFB00203B49096886
:100F4000C8733A4800684079401C384909684871BC
:100F50007EE037490969354A1268D27A885C07F021
:100F600013FC324800684079401C304909684871D8
:100F70002E4800684079401C2C490968487167E098
:100F800001F00EFD002811D1252007F0FDFB2748B8
:100F900000684079401C2549096848712348006869
:100FA0004079401C21490968487105E007F09EFB23
:100FB00000201E49096848714AE001F0F1FC002850
:100FC00010D107F0E1FB194800684079401C17492F
:100FD00009684871154800684079401C1349096840
:100FE000487105E007F082FB00201049096848714C
:100FF0002EE001F0D5FC002815D10C480068C07A1D
:10100000401C0A490968C87208480068C07A084943
:101010000978884207DB002004490968C872032068
:1010200002490968887107F061FB05E07407002038
:10103000A41A002070070020002012490968487196
:1010400006E007F053FB00200E490968487100BF15
:1010500000BF15E000200B4909688871094909683B
:101060004871062007490968C87009E007F03EFB8F
:10107000002004490968487102490968887100BF65
:1010800000BF10BD7407002010B56A4800684079A1
:1010900003000AF0A7FC090610C627C644C6608EE6
:1010A000C60007F0F9FA634800684079401C6149BE
:1010B00009684871BCE0604909695E4A1268D27AE1
:1010C000885C07F061FB5B4800684079401C594927
:1010D00009684871574800684079401C55490968BB
:1010E0004871A5E001F05CFC002811D14F2007F009
:1010F0004BFB504800684079401C4E4909684871D4
:101100004C4800684079401C4A490968487105E02C
:1011100007F0ECFA002047490968487188E001F0BF
:101120003FFC002810D107F02FFB424800684079AF
:10113000401C4049096848713E4800684079401C9D
:101140003C490968487105E007F0D0FA00203949A8
:10115000096848716CE001F023FC002822D1354871
:101160000068C07A401C33490968C8723148006879
:10117000C07A3149097888420FDB00202D4909687F
:10118000C8722C4800684079401C2A490968487197
:10119000002028490968486208E0002025490968BC
:1011A000487103E0002023490968487107F09EFA5E
:1011B0003EE020480068407C002816D01E48C068E9
:1011C000002803D01C48C16819208847002019490D
:1011D00009684862174909684871164909688871A1
:1011E000052014490968C8701AE012480068406A6E
:1011F000282807D20F480068406A401C0D4909683A
:1012000048620DE000200B490968486209490968F5
:101210004871084909688871052006490968C8703D
:1012200006E007F063FA002002490968487100BF30
:1012300000BF10BD74070020A41A002010B50024C0
:10124000F7480068807A01287ED1F5480068C079A7
:1012500000287AD0F24800688079002804D001285C
:1012600074D0022873D191E1ED480068007B2428F6
:101270006ED2EB480068C07901287AD1002475E06D
:10128000E7480068C07A24214843E64909684018C5
:10129000E3490968097B415CE1480068C07A24227F
:1012A0005043E14A12688018DD4A1268127B805C64
:1012B000814229D0DA480068C07A24214843DA49BB
:1012C00009684018D6490968097B415CD448006820
:1012D000C07A24225043D34A12688018D04A126838
:1012E000127B8154CE480068407B242805D3CC482B
:1012F0000068007BCA4909684873C9480068007BD8
:10130000C7490968887308E0C5480068407B2428FD
:1013100003D20120C24909688871C1480068007B76
:10132000401CBF4909680873BD480068007B242839
:1013300008D3BB480068407B242803D20120B84969
:1013400009688871B64805E0D3E1CDE169E0BAE10A
:1013500038E00EE00068007B242804D2B048006822
:101360008079012800D103E0601CC4B2242C87D30B
:1013700056E0002413E0AA480068C07A24214843BC
:10138000A94909684018015DA5480068C07A24226F
:101390005043A44A126880180155601CC4B2242C22
:1013A000E9D300209E490968487323209C490968B5
:1013B000887301209A49096888712420984909682E
:1013C00008732DE000209649096808739448006866
:1013D000C07A401C92490968C87291480068C07A76
:1013E00092490978884217DB8D480068007C012803
:1013F00004D102208A490968887106E000208849E2
:101400000968887186490968C8710020844909689B
:10141000C8728349096808740020814909684871C5
:1014200061E17F480068407903000AF0DBFA0805B3
:1014300013A62AA651A68EA6012079490968087428
:1014400007F02AF9764800684079401C7449096819
:10145000487199E075490969714A1268D27A885CC5
:1014600007F092F96E4800684079401C6C490968A1
:1014700048716B4800684079401C694909684871A7
:1014800082E001F08DFA00281BD165490968497B8B
:10149000491CC8B207F078F961480068407B604990
:1014A0000968C8735E4800684079401C5C49096857
:1014B00048715B4800684079401C59490968487187
:1014C00005E007F013F900205549096848715BE011
:1014D00001F066FA00282BD151490968C97A242203
:1014E0005143504A126889184D4A1268D27B885C71
:1014F00007F04AF94A480068C07B401C484909681F
:10150000C87347480068C07B45490968897B8842A1
:101510001ADD434800684079401C41490968487118
:101520003F4800684079401C3D49096848710BE01C
:1015300007F0DCF83A480068407B39490968C8730D
:1015400000203749096848711EE001F029FA002897
:101550000CD1334909688871242031490968C8735E
:101560002F49096848732E490968887307F0BEF847
:1015700000202B490968487106E007F0B7F8002001
:1015800027490968487100BF00BFACE024480068E3
:10159000407903000AF026FA08050F8E268E4C8E3D
:1015A000688E07F079F81E4800684079401C1C4995
:1015B0000968487185E01D490969194A1268D27A9B
:1015C000885C07F0E1F8164800684079401C14492F
:1015D00009684871124800684079401C1049096840
:1015E00048716EE001F0DCF9002811D1252007F0E8
:1015F000CBF80B4800684079401C094909684871DC
:10160000074800684079401C05490968487105E0B1
:1016100007F06CF8002002490968487151E00000A9
:1016200074070020700700206C070020A41A002017
:1016300001F0B6F9002810D107F0A6F86448006858
:101640004079401C624909684871614800684079E6
:10165000401C5F490968487105E007F047F8002021
:101660005B49096848712CE001F09AF900281AD109
:1016700057480068C07A401C55490968C8725448E8
:101680000068C07A5349097888420CDB0020504931
:101690000968C8724E49096888714D4909684871DE
:1016A0004B490968C87107F021F8002048490968CA
:1016B000487106E007F01AF80020454909684871AA
:1016C00000BF00BF0FE007F011F800204049096893
:1016D00048713F49096888713D49096808733C4968
:1016E0000968C87200BF71E0002039490968887232
:1016F0006CE037480068807A022867D13448006877
:10170000007A00285ED0324800684079002804D072
:1017100001280CD0032846D11BE006F0BDFF2C4861
:1017200000684079401C2A490968487149E0002056
:1017300007F02AF8264800684079401C24490968C7
:101740004871234800684079401C21490968487164
:1017500037E006F06BFF002812D11D480068407882
:10176000401C1B49096848701948006840780328E4
:1017700012D301F0B5F900201549096848700BE053
:101780000020134909680872AA2011490968887065
:1017900000200F490968487006F0A8FF00200C4996
:1017A000096848710DE006F0A1FF002008490968AA
:1017B0004871074909684870AA2005490968887076
:1017C00000BF03E0002002490968887210BD0000D4
:1017D00074070020A41A0020F8B504460D46002620
:1017E0000C2060431D49085C002801D00120F8BD91
:1017F0000C2060431949401885600C206043401854
:101800008068002801D10120F1E701210C2060430C
:10181000124A115400222046E317DB0E1B185B11FD
:101820005B01E31A9B000E4FDB19E717FF0E3F1910
:101830007F11DA550AF008F900222046E317DB0E83
:101840001B185B115B01E31A9F00064BFB18E7179F
:10185000FF0E3F197F11DA553046C8E770020020AD
:10186000006000400061004000BFFEE709480088BA
:10187000401C08490880084600880749884208DD5E
:1018800006480078002804D0084602490880012054
:101890008870704798000020DC050000A30000203D
:1018A00010B50B488078012810D10A48007801282B
:1018B00002D1094802F060FA06480078022802D1F5
:1018C000054802F059FA00200249087010BD0000D6
:1018D00098000020A3000020AD0000207047000009
:1018E00010B500F0FFFD012803D100200149088058
:1018F000887010BD98000020F0B505460E461746CA
:1019000000243A463146284600F0FAFD00BF42E086
:1019100000202101394A126850522101374A1268C9
:101920008918488000212001344A1268801881807B
:101930002001324A12688018C18020012F4A1268A3
:101940008018017220012D4A12688018417220010E
:101950002A4A1268801881722001284A1268801869
:10196000C17200202101254A1268891808730021DC
:101970002001224A126880184173002021011F4A69
:10198000126889188873002120011C4A1268801887
:10199000C173601CC4B21A484078A042B8DC64200D
:1019A0001849096808807D20C000164909684880E8
:1019B00015481449096888807D200001114909688B
:1019C000C88010490968088110480E490968488193
:1019D0000F480C490968888140000A490968C88194
:1019E0003220084909680882FF20F5300549096856
:1019F0004882044909688882F0BD00000007002081
:101A0000F4060020FC0600204C0400001027000013
:101A10003075000038B5002404E000201349085553
:101A2000601C84B2282CF8D30121684641700170F3
:101A30006A460F490D48FFF75FFF7D21C90032203C
:101A400000F04EF90B490C4800F068F90948643081
:101A500000F0FAF80748C83000F006F9074800F02F
:101A600019F9074800F02CF938BD000014140020C3
:101A700028C8010028230000B80B000054240000EF
:101A80001027000013480078002803D101201149D5
:101A900008701EE00F480078012803D102200D498C
:101AA000087016E00B480078022803D1032009498A
:101AB00008700EE007480078032803D10420054988
:101AC000087006E003480078042802D1002001498C
:101AD00008707047A3000020F8B5002400250026F8
:101AE0003348007800281ED132480078002803D1FE
:101AF00001203049087016E02E480078012803D1F3
:101B000002202C4908700EE02A480078022803D1F0
:101B100003202849087006E026480078032802D1EF
:101B20000020244908702248007801280BD10124A4
:101B300017250026204801233246294600902046DA
:101B400001F08EFD33E01A48007802280CD1012400
:101B50003B2500261848401C0123324629460090A8
:101B6000204601F07DFD22E01148007803280DD1C8
:101B7000FEF766FA002803D101201049087102E03F
:101B800000200E49087109F0FFFE10E008480078B7
:101B900004280CD1FEF766FA002803D1012007497A
:101BA000487102E000200549487109F0EDFEF8BDDA
:101BB000A3000020A4000020AD0000209C00002015
:101BC00010B50446230009F00DFF093306090C0D7A
:101BD0000E0F31323600FFF77FFF2DE0FFF752FF87
:101BE0002AE029E028E027E001F016FD13480078FC
:101BF00003280ED11248007800280AD1FEF72CFAEB
:101C0000002803D101200F49887102E000200D490E
:101C100088710A480078012805D109480078002811
:101C200001D1FAF73FFE08F0B1F905E004E003E066
:101C3000FFF71CFE00E000BF00BF10BDA4000020A5
:101C4000A30000209C00002001460020054A1268E5
:101C500052898A4201DC012002E0024A12681181A5
:101C600070470000FC06002001460020084A126868
:101C700012898A4201DB012009E0054A1268928933
:101C80008A4201DC012002E0014A1268518170475A
:101C9000FC06002001460020084A126852898A4248
:101CA00001DB012009E0054A1268D2898A4201DC81
:101CB000012002E0014A126891817047FC06002071
:101CC00001460020054A126892898A4201DB012000
:101CD00002E0024A1268D18170470000FC06002031
:101CE000024600200C4B1B681B8A934201DD012039
:101CF00010E08A4201DB01200CE0074B1B689B8847
:101D00008B4201DC012005E0034B1B681A80024B6B
:101D10001B68598070470000FC0600200246002026
:101D20000C4B1B681B8A934201DD012010E08A42A4
:101D300001DB01200CE0074B1B685B88934201DB51
:101D4000012005E0034B1B689A80024B1B68D98079
:101D500070470000FC06002070B5044600250C20EA
:101D60006043FE49096840184068002807D00C21EC
:101D70006143FA4A126889184868804705460C2072
:101D80006043F6490968085C002873D10C20604361
:101D9000F249096840188068002874D02001F04991
:101DA00009684018C07A02280AD1032D08D10C20F6
:101DB0006043EA4A1268801881680120884762E01F
:101DC0002001E74909684018C07A02280AD1042D89
:101DD00008D10C206043E14A126880188168022013
:101DE000884750E02001DE4909684018C07A02287F
:101DF0000AD1052D08D10C206043D84A12688018FA
:101E00008168032088473EE02001D54909684018D1
:101E1000C07A02280AD1062D08D10C206043CF4A8F
:101E2000126880188168042088472CE02001CC4982
:101E300009684018C07A02280AD1072D08D10C2061
:101E40006043C64A126880188168052088471AE0F6
:101E50002001C34909684018C07A02280BD1082D17
:101E600009D10C206043BD4A1268801881680620A1
:101E7000884708E00DE00C206043B84A12688018DB
:101E80008168002088472001B54909684018C5725B
:101E90000CE30C206043B1490968085C012873D148
:101EA0000C206043AD49096840188068002874D050
:101EB0002001AB4909684018C07A03280AD1022DD5
:101EC00008D10C206043A54A12688018816801205F
:101ED000884762E02001A24909684018C07A0428B6
:101EE0000AD1022D08D10C2060439C4A1268801848
:101EF00081680220884750E020019949096840180C
:101F0000C07A05280AD1022D08D10C206043934ADB
:101F1000126880188168032088473EE020019049BC
:101F200009684018C07A06280AD1022D08D10C2071
:101F300060438A4A126880188168042088472CE030
:101F40002001874909684018C07A07280AD1022D64
:101F500008D10C206043814A1268801881680520EE
:101F600088471AE020017E4909684018C07A08288D
:101F70000BD1022D09D10C206043784A12688018D9
:101F800081680620884708E00DE00C206043734A12
:101F9000126880188168002088472001704909680C
:101FA0004018C57282E20C2060436C490968085CE5
:101FB0000228F7D1002D7DD1200169490968085A0E
:101FC00068490968098A884275DA20016449096804
:101FD000085A0A3081B22001614A12681152200168
:101FE0005F490968085A5F490968098A884231DBF4
:101FF00020015B490968401840885A4909680988E6
:10200000884227DB20015649096840184088554915
:102010000968498888421DDC00202101504A126865
:102020008918488020014E4909684018807A0028A4
:10203000B8D10C20604349490968401880680028DD
:10204000B0D00C206043454A126880188168012096
:1020500088472BE2200142490968085A414909682A
:10206000098A88429EDB20013D4909684018408862
:102070003C4909688988884294DB2001384909680D
:102080004018408837490968C98888428ADC00209E
:102090002101334A126889184880200130490968B3
:1020A0004018807A0028D4D10C2060432B4909685D
:1020B000401801E063E00BE080680028C9D00C20E4
:1020C0006043264A12688018816802208847EDE143
:1020D00000202101224A1268891848802101204AE3
:1020E00012688918C872002120011D4A12688018E0
:1020F000C18020011A4A1268801841722001184AD2
:10210000126880188172184801782001144A1268F8
:102110008018017200202101114A126889188880F4
:1021200021010F4A12688918087321010C4A1268AC
:102130008918487321010A4A126889188873002196
:102140002001074A12688018C1730C2060430349BC
:102150000968401880680028B9D007E0F806002018
:1021600000070020FC060020F40600200C2060433D
:10217000CF4A1268801881680020884796E1012DB7
:10218000A5D12001CB4909684018C07AA84225D0C2
:1021900000212001C74A12688018418000202101D7
:1021A000C44A12688918C8802001C24909684018C9
:1021B000C572C14800782101BE4A12688918487268
:1021C00000202101BB4A126889188880BA4801782A
:1021D0002001B84A12688018017267E12001B549F0
:1021E00009684018007AB4490978884220D0B2487A
:1021F00000782101AF4A1268891808722001AD49A0
:1022000009684018407AAC490978884209D0200111
:10221000A8490968401880882101A64A12688918CF
:10222000C88000212001A34A12688018818012E032
:102230002001A049096840188088A04988420AD234
:1022400020019C490968401880880A302101994A78
:1022500012688918888020019649096840184088CA
:10226000964988420AD2200192490968401840885C
:102270000A3021018F4A12688918488020018D494F
:1022800009684018407A8C490978884205D00120B5
:102290002101884A126889188872200185490968D5
:1022A00040184088864909680988884204DB002173
:1022B0002001804A1268115220017E4909684018A5
:1022C000807A00287ED10C20604379490968401843
:1022D0008068002877D02001764909684018408836
:1022E000774909680989884214DB20017149096826
:1022F0004018007B00280DD10C2060436C4A126806
:10230000801881680320884701202101694A1268EA
:10231000891808732001674909684018408868498E
:1023200009684989884214DB20016249096840181C
:10233000407B00280DD10C2060435D4A1268801854
:10234000816804208847012021015A4A12688918AF
:10235000487320015749096840184088584909685E
:102360008989884214DB2001524909684018807B22
:1023700000280DD10C2060434D4A126880188168F6
:1023800005208847012021014A4A1268891888736C
:102390002001484909684018408849490968C989A5
:1023A000884210DB2001434909684018C07B00289F
:1023B0007CD10C2060433E4A126880188168062058
:1023C000884701E007E03BE001202101394A12681B
:1023D0008918C8736AE02001364909684018407AB4
:1023E00001282ED13448007802282AD12001314911
:1023F00009684018C08832490968498A884255DB13
:1024000020012C490968401880882D490968898A6B
:1024100088424BDB0C2060432549096840188068DE
:10242000002843D00C206043214A1268801881683C
:1024300007208847002021011E4A12688918487227
:1024400034E020011B4909684018407A02282DD148
:1024500019480078012829D1200116490968401837
:10246000C08817490968898A88421FDB2001114901
:1024700009684018808812490968498A884215DB32
:102480000C2060430A4909684018806800280DD074
:102490000C206043064A126880188168082088472B
:1024A00000202101034A12688918487270BD00009B
:1024B000F806002000070020F4060020F0FF0000CE
:1024C000FC06002010B5002400BF04E02046FFF702
:1024D00043FC601CC4B202484078A042F6DC10BD48
:1024E000F406002010B50024044801F073FE002813
:1024F00000D000E00124204610BD000003040000CD
:1025000010B5074B14781C7054785C70054B19603B
:10251000054B186003461833044C236010BD0000BF
:10252000F4060020F8060020FC060020000700202A
:1025300010B50446012C09D164220C21002000F0C2
:10254000C7F80121022003F06DFC08E000220C21F5
:10255000104600F0BDF80021022003F063FC10BD1E
:1025600010B5002404210848F8F798FC552801D13B
:10257000012407E0042000F0C1FF002801D000245E
:1025800000E00124204610BDCC07002010B5044611
:10259000012C09D164221C21002000F099F80121AE
:1025A000062003F03FFC08E000221C21104600F04A
:1025B0008FF80021062003F035FC10BD10B5002473
:1025C000062000F09BFF002801D0012400E0002439
:1025D000204610BD10B50446012C09D164221721F4
:1025E000002000F075F80121042003F01BFC08E036
:1025F00000221721104600F06BF80021042003F0A0
:1026000011FC10BD002000BF704710B50446022C1D
:102610001CD100220D21104600F05AF8FDF760FD94
:10262000002809D064220B21002000F051F801217C
:102630000D2003F0F7FB38E000220B21104600F0DC
:1026400047F800210D2003F0EDFB2EE0032C1CD1F8
:1026500000220B21104600F03BF8FDF741FD002859
:1026600009D064220D21002000F032F801210D2054
:1026700003F0D8FB19E000220D21104600F028F8E5
:1026800000210D2003F0CEFB0FE0012C0DD16422C0
:102690000D21002000F01CF800220B21104600F054
:1026A00017F801210D2003F0BDFB10BD10B500246B
:1026B000FCF7D0FF022801D1022406E0FCF7CAFF94
:1026C000012801D1032400E00124204610BD0000B0
:1026D00010B5064B1B78834207DD242905D224233D
:1026E0004343034C24681B195A5410BDA41A0020FC
:1026F0006C07002010B5744800684079030009F0A9
:1027000071F90B0711D325D35A6D77D38DA8D30058
:1027100005F0C2FF6C4800684079401C6A490968AE
:102720004871CFE069494969087806F02DF8664894
:1027300000684079401C6449096848716248006833
:102740004079401C604909684871BBE000F028F9F5
:10275000002811D17F2006F017F85B480068407907
:10276000401C594909684871574800684079401C25
:102770005549096848711DE0534800684078401C7D
:1027800051490968487050480068407803280BD3C5
:1027900000204D4909684870AA204B490968887093
:1027A000032049490968C87005F0A0FF0020464988
:1027B0000968487186E000F0F3F8002807D1424824
:1027C00000684079401C40490968487103E00020D6
:1027D0003D490968487105F089FF73E005F05CFF29
:1027E000394800684079401C37490968487169E0F8
:1027F000364949690978491CC8B205F0C5FF324815
:1028000000684079401C3049096848712E480068CA
:102810004079401C2C490968487153E000F0C0F829
:1028200000280FD105F00AFF2749096888700120A8
:1028300005F07EFF244800684079401C2249096861
:10284000487105E005F052FF00201F4909684871F2
:1028500038E01D480068807818280CD102201A49F9
:102860000968087000201849096848700420164952
:102870000968C87011E0144800684078401C12498B
:1028800009684870104800684078032805D300F0B4
:1028900027F900200C490968487005F027FF00203F
:1028A0000949096848710DE005F020FF002006493C
:1028B00009684871044909684870AA2002490968F2
:1028C000887000BF00BF10BD74070020A41A00204C
:1028D00010B5314800684079002804D001280CD098
:1028E000032848D11DE005F0D7FE2B480068407949
:1028F000401C2949096848714BE028490969087852
:1029000005F042FF244800684079401C22490968CC
:102910004871214800684079401C1F490968487186
:1029200037E000F03DF800280CD101201A49096871
:102930000870002018490968487004201649096881
:10294000C87011E0144800684078401C12490968BA
:102950004870114800684078032805D300F0C0F89B
:1029600000200D490968487005F0C0FE00200A49A2
:10297000096848710DE005F0B9FE002006490968B4
:102980004871054909684870AA2003490968887098
:1029900000BF00BF10BD000074070020A41A002073
:1029A00010B505F043FE04461F4800680078002873
:1029B00038D01D480068C078042833D3002C09D1D2
:1029C000002119480068C07A820017480068143056
:1029D000815027E014480068C07A810012480068DE
:1029E000143040581149884211D20F480068C07A0B
:1029F00081000D48006814304058401C0A4909689D
:102A0000C97A8A0008490968143188500AE000F040
:102A100067F8002104480068C07A82000248006814
:102A200014308150204610BD74070020B80B000000
:102A300000B587B00120694608710848029008482F
:102A4000039008480490084805900848069001A99A
:102A5000074800F00FF807B000BD0000992D0100F5
:102A6000C143010071BB010089C8010088C8010091
:102A700074140020F8B506460F4600240025394698
:102A8000304600F0EFF900BF14E000250EE0002111
:102A9000242060430B4A126880184155242060436B
:102AA000094A126880184155681CC5B2242DEED31E
:102AB000601CC4B205480078A042E6DC00F010F8C3
:102AC000F8BD00006C07002070070020A41A002049
:102AD000012002490968087170470000740700204E
:102AE00010B500F073F90020034909680870024925
:102AF0000968C87010BD000074070020074800680E
:102B0000C078062808D105480068C079002803D19C
:102B1000012002490968C87170470000740700204D
:102B200010B555480068C078030008F05BFF0867DF
:102B30001D1A1714110E056650484068002803D06E
:102B40004E4841680020884793E000F0E5F890E0A7
:102B500000F0C6F88DE000F0D1F88AE0FFF7B8FE8B
:102B600087E0FFF7C7FD84E044484068002803D0B1
:102B700042484168012088473F480068407C00285F
:102B80001AD03E48C068002803D03C48C168C8201D
:102B9000884700203849096848623748006800784B
:102BA000002804D0042034490968C87024E00220B9
:102BB00031490968C8701FE02F480068406A401C0E
:102BC0002D49096848622C480068406A7D21C90087
:102BD000884211D3002028490968486226480068C5
:102BE0000078002804D0042023490968C87003E055
:102BF000022021490968C8703BE000BF1F484068B7
:102C0000002803D01D484168002088471A48006802
:102C1000407C002813D01948C068002803D017480A
:102C2000C168C820884700201349096848621248D3
:102C30000068C078401C10490968C87018E00E4848
:102C40000068406A401C0C49096848620A480068EC
:102C5000406A7D21C90088420AD3002006490968DC
:102C6000486205480068C078401C03490968C8707C
:102C700000BF00BF10BD000074070020A41A002090
:102C800010B515480068C078072824D001201249E3
:102C90000968487408E011488068002802D00F498C
:102CA00088688047FFF73CFF0B480068C07806281B
:102CB000F1D109480068007A0028ECD10648006884
:102CC000C0790028E7D104480068807A0028E2D162
:102CD00001490968487410BD74070020A41A002037
:102CE00010B5054800680078012802D1FDF7A0FF63
:102CF00001E0F6F707FC10BD7407002010B5054889
:102D000000680078012802D1FEF7BEF901E0F6F76D
:102D1000D7FF10BD7407002010B51D480068807AE9
:102D2000002829D11A480068007A002803D0022020
:102D300017490968887216480068C079002803D0CE
:102D40000120134909688872114800680079012838
:102D500012D100200E49096808710D49096888726E
:102D600007200B490968C8700A484068002803D04A
:102D70000848416800208847054800680078012815
:102D800002D1FEF75BFA01E0F7F774F810BD00001E
:102D900074070020A41A002010B5044621460848F4
:102DA00001F034FA07480078002805D1002C03D040
:102DB00032210548FCF758FF0248047010BD00009E
:102DC00001030000B600002050C300000020244989
:102DD00009684870AA2022490968887000202049A3
:102DE000096848621E49096808711D4909684871E7
:102DF0001B49096888711A490968C8711849096826
:102E0000087217490968887215490968C872144917
:102E10000968087324201249096848731049096831
:102E200088730F490968C87300200D490968087440
:102E30000B49096848740A4909688874084909688F
:102E4000C874074909684861002105480068816124
:102E500003480068C16102480068016270470000D1
:102E60007407002010B50A780D4B1860034628330C
:102E70000C4C236024235343044628341B190A4C6A
:102E800023600A4C4B6863608B68A360CB68E36087
:102E90004B6963610B6923610B78237010BD0000DF
:102EA000740700206C07002070070020A41A00207F
:102EB00007480068C078062808D105480068007AED
:102EC000002803D1012002490968087270470000F8
:102ED0007407002010B50446012C09D1642220217A
:102EE0000020FFF7F5FB0121084602F09BFF08E0F8
:102EF000002220211046FFF7EBFB0021012002F009
:102F000091FF10BD10B50024032000F0F7FA00284F
:102F100001D0012400E00024204610BD10B5044675
:102F2000032C0ED1642215210020FFF7D1FB0022D3
:102F300014211046FFF7CCFB01210E2002F072FF96
:102F400039E0022C1CD1FDF7CBF8002809D064220F
:102F500014210020FFF7BCFB01210E2002F062FFCC
:102F600008E0002214211046FFF7B2FB00210E20DA
:102F700002F058FF002215211046FFF7A9FB1AE0C6
:102F8000012C0ED1642214210020FFF7A1FB0121A6
:102F90000E2002F047FF002215211046FFF798FB94
:102FA00009E0002215211046FFF792FB00221421B0
:102FB0001046FFF78DFB10BD10B50024F9F7D8FAC5
:102FC000094988420DD3FDF7CBF8002807D1FCF75B
:102FD000FDFF012801DD032404E0022402E00224B5
:102FE00000E00124204610BDB80B000010B50446D7
:102FF000012C09D164221D210020FFF769FB01216A
:10300000002002F00FFF08E000221D211046FFF70C
:103010005FFB0021084602F005FF10BD10B500243B
:10302000022000F06BFA002810D00124104800782C
:10303000052805DA0E480078401C0D49087015E097
:1030400005200B490870002048700FE00024084854
:103050004078052805DA06484078401C0449487045
:1030600004E005200249487000200870204610BD89
:10307000D200002010B50446012C09D164221E2183
:103080000020FFF725FB0121092002F0CBFE08E01C
:1030900000221E211046FFF71BFB0021092002F031
:1030A000C1FE10BD70B5002400250026FCF79CFE73
:1030B0000546FCF7A5FE064602210848F7F7EEFE96
:1030C000552800D108E0012E01D1002404E0012D93
:1030D00001D1012400E00024204670BDCC0700206F
:1030E00010B50446012C09D164221F210020FFF7EE
:1030F000EFFA0121082002F095FE08E000221F21CE
:103100001046FFF7E5FA0021082002F08BFE10BD03
:1031100070B500250024FCF79FFE044603210C48EF
:10312000F7F7BCFE552803D101200A4908800AE0C0
:10313000762C03DA01200749088004E0782C02DBB2
:1031400000200449088003480588284670BD000017
:10315000CC070020D400002010B50446012C09D172
:10316000642221210020FFF7B3FA0121072002F099
:1031700059FE08E0002221211046FFF7A9FA00219C
:10318000072002F04FFE10BD10B50024FCF730FF01
:10319000002801D1012400E00024204610BD704722
:1031A0000020704710B50446012C09D16422162175
:1031B0000020FFF78DFA0121032002F033FE08E022
:1031C000002216211046FFF783FA0021032002F0A7
:1031D00029FE10BD10B50024052000F08FF900284D
:1031E00001D0012400E00024204610BD10B50446A3
:1031F000012C09D1642219210020FFF769FA01216D
:10320000052002F00FFE3CE0022C17D1FCF768FF0E
:10321000002809D0642219210020FFF759FA012162
:10322000052002F0FFFD2CE0002219211046FFF7D7
:103230004FFA0021052002F0F5FD22E0032C17D102
:10324000FCF754FF002809D0642219210020FFF761
:103250003FFA0121052002F0E5FD12E000221921CC
:103260001046FFF735FA0021052002F0DBFD08E0EB
:10327000002219211046FFF72BFA0021052002F049
:10328000D1FD10BD10B50024FCF7E6FE01282FD1BA
:1032900004211948F7F702FE552801D1012428E03E
:1032A000FCF7BAFD01280BD0FCF7B6FD022807D0C9
:1032B000FCF7B2FD032803D0FCF7AEFD052801D1D1
:1032C000012416E0FCF7A8FD042801D1022410E037
:1032D000FCF7A2FD062801D103240AE0FCF79CFDBF
:1032E000002803D0FCF798FD072802D1002400E055
:1032F0000024204610BD0000CC07002010B5044675
:10330000012C0ED164221B210020FFF7E1F90022DD
:103310001A211046FFF7DCF901210A2002F082FD94
:103320000DE064221A210020FFF7D2F900221B21B0
:103330001046FFF7CDF901210A2002F073FD10BD00
:1033400010B50024FCF778FF012801D1012400E02A
:103350000024204610BD10B5F9F724F90446204694
:1033600010BD000010B5034B07220349034800F0CD
:1033700013F910BD5733010034C801003C1400207C
:1033800070B506465C488068002804D05A498868B1
:103390008047054600E000250024A6E05648416825
:1033A0000C20604308184088A84207D05248416862
:1033B0000C2060430818408802287DD14E4841689F
:1033C0000C2060430818806800280CD04A494A68DD
:1033D0000C21614351188868804747490968E20019
:1033E0008918487009E0444841680C206043095C32
:1033F00041480068E200801841703F480068E100E1
:10340000401840783C490968E200895C88420FD046
:1034100039480068E1004018417837480068E20008
:103420008154002034490968E200891848605AE054
:1034300031480068E100401841782F4842680C206C
:1034400060431018407881421FD12B480068E1008A
:1034500040184168284842680C2060431018808852
:1034600081420BD824480068E10040184068801968
:1034700021490968E2008918486034E001201E49AA
:103480000968E200891848802DE01B480068E100C7
:1034900040184168184842680C2060431018C088E2
:1034A00081420DD814480068E10040184068811935
:1034B00011480068E20000E009E08018416012E075
:1034C00000200D490968E200891848800BE00020BF
:1034D00009490968E2008918488000210648006807
:1034E000E20080184160601C84B203488089A042D9
:1034F00000DD53E770BD0000081A00200146064AAF
:1035000092898A4205DD044A1268CB00D21850889D
:1035100000E0002070470000081A0020002000BFD3
:1035200014E00D494A680C2141435118498801298A
:103530000AD10021084A1268C300D2185180064AF5
:103540001268C300D2185160411C88B202498989AF
:103550008142E6DC70470000081A0020002000BF0E
:1035600013E00C494A680C2141435118498800294D
:1035700009D1084A1268C300D2185180054A12685E
:10358000C300D2185160411C88B202498989814226
:10359000E7DC7047081A0020F0B504460020164DFD
:1035A000AB6069602C60AA8100BF1FE0124D6E689D
:1035B0000C254543755D104E3668C700F6197570C9
:1035C0000D4D6E680C254543755D0B4E3668C70082
:1035D000F5550025084E3668C700F6197580064E69
:1035E0003668C700F6197560451CA8B2024DAD8952
:1035F0008542DBDCF0BD0000081A002070B50546EE
:103600000E46002E05D031462846F4F799FD0446B3
:1036100000E02C46204670BD10B5FCF7E9FC002800
:1036200009D105480078032805D10448007800280E
:1036300001D1F9F78FFC10BDA4000020A3000020E9
:1036400001200149887170479C0000200020034937
:103650000871487101208871704700009C000020AB
:1036600070B5049C2578914216DD01280AD18D425F
:1036700006DAFF26F61AAE420ED3EE18F5B20BE0CC
:10368000154609E0022807D1954204DD9D4203DB7F
:10369000EE1AF5B200E00D46257070BD0D4A416886
:1036A000516081699161C168D160416A5162016A6A
:1036B0001162016811604169516181689160C1695D
:1036C000D16101691161816A91620021024A117020
:1036D00070470000781A00206A07002010B5FFF735
:1036E0001DFFF8F7EFFD00210148F7F7D7FC10BDEB
:1036F000D807002010B500200B490870F8F7E2FD4C
:10370000FFF72CFF06F088FE06F024FFFBF77AFE99
:10371000FAF71AFCFFF794FFF9F7C0F955210348AF
:10372000F7F7BCFC10BD0000B5000020D807002052
:103730001CB500203449087004F05EFF0020FCF73F
:10374000E5FD08F077FCF7F7A7FF55212F48F7F7BD
:10375000A5FCF8F7E1FFF6F7CBFEF7F749F905F01E
:1037600019F9F8F7AFFDFAF7EDF9F9F723FAF9F7D8
:10377000A1F9FFF7F7FDFEF74DF9FFF759F9FAF751
:10378000F9F8FBF76BFEFAF7DFFB214AFF219131D5
:10379000002006F0A7FF1E4AFF219131012006F00C
:1037A000A1FF00221146104606F0E0FE0022012192
:1037B000104606F0DBFE00220221104606F0D6FE7F
:1037C00000221146012006F0D1FE06F00BFE06F0A5
:1037D000C1FEFFF73BFFF9F779FE00200D49887124
:1037E0004871087101208870487014200870072201
:1037F0006846F4F73CFD0199009800F057FD02215E
:10380000012000F033FC1CBDB5000020D8070020CB
:103810000090D003C60000207047000010B5044699
:10382000552C03D105494869804702E003490868DF
:10383000804700200249087010BD0000781A00205F
:103840006A07002010B546480078030008F0CAF85F
:103850000A06111B26303B4650517381414840688F
:10386000002802D03F494868804701203C49087041
:1038700000BF3C488068002804D03A4988688047E7
:103880003749087069E03748C068002802D03549D8
:10389000C868804703203249087000BF314800697A
:1038A000002804D02F49086980472D49087054E04A
:1038B0002C484069002802D02A49486980470020E6
:1038C0002749087049E027488069002802D0254927
:1038D0008869804706202249087000BF2148C069D6
:1038E000002804D01F49C86980471D49087034E08A
:1038F00000BF1B48007807280AD11A48006A002830
:1039000002D01849086A804709201549087011E05B
:103910001348007808280AD11248406A002802D0CB
:103920001049486A804709200D49087002E00020CC
:103930000B49087000BF0A480078002808D00948E1
:10394000806A002804D00749886A804704490870C3
:1039500003E000200249087000BF00BF10BD000056
:103960006A070020781A00207047000010B5002276
:10397000FF219131104606F0B5FE0022FF21913162
:10398000012006F0AFFE002008F0EEFB05F050FE2F
:1039900005F0A4FE05F0BAFE00F05CFAF7F7B8F8FF
:1039A0000220FCF7B3FC002006490870FFF768F915
:1039B000FFF78EF8FFF7B4F8F6F70AFF00F04AFBBE
:1039C00010BD00000C01002010B5012405F080FAA4
:1039D000012801D1052407E0F8F7C4FD0349884216
:1039E00001D2012400E00224204610BD204E000038
:1039F00010B5062405F06CFA002800D1002405F06B
:103A00006DFA012803D005F069FA072800D90924C6
:103A1000204610BD10B5F7F77BF8002211460120B3
:103A200006F0D6FE00213A48F7F738FB002400BF25
:103A300000F0C6FC32217D200001FCF715F90020C2
:103A4000344908700AE00022324801781046FEF737
:103A50003FFE30480078401C2E4908702D48007801
:103A60002428F0DB00202C49087009E000212A48B6
:103A7000007806F0BFFA28480078401C26490870F4
:103A8000254800780E28F1DBFFF74AF8F6F776FDB7
:103A900005F070F921480078401C2049087008465C
:103AA0000078052812D300200870FFF727F81C487B
:103AB00000780A2805D3002019490870FFF7F8F9A3
:103AC00004E017480078401C1549087005F006FA14
:103AD0000128ADD905F002FA0728A9D200200E4925
:103AE000087008E00C48007806F09EFA0A48007852
:103AF000401C09490870084800780E28F2DBF6F7E8
:103B000077FF55210248F7F7C9FA204610BD00009B
:103B1000D8070020CF000020CD000020CE000020DC
:103B2000D000002010B5032408E000F049FC01207B
:103B300000F050FB002801D0042400E0F5E700BFAE
:103B4000204610BD10B500202949086004F054FD3E
:103B50000120FCF7DBFBF7F79FFD55212548F7F720
:103B60009DFA08F067FAF6F7C3FCF9F7B3FFF6F72A
:103B70003FFF05F00FF9F9F7E5FFFAF7CDF9F9F78F
:103B800019F8FFF7EFFBFDF745FFFFF7E7FCFFF73D
:103B900057FDFEF74DFFFBF761FCFAF7D5F9164A22
:103BA000FF219131002006F09DFD134AFF21913144
:103BB000012006F097FD00221146104606F0D6FCC3
:103BC00000220121104606F0D1FC002202211046FD
:103BD00006F0CCFC00221146012006F0C7FC06F0DE
:103BE00001FC06F0B7FC0221012000F03FFA10BDF5
:103BF00044000020D80700200090D00310B50248F0
:103C0000FFF74CFD10BD000010C901000021014A62
:103C10001175704740600040014600BFF020084029
:103C200000110A23584302460807000F8018C0B24B
:103C300070470146002204E0501CC2B208460A3810
:103C4000C1B20A29F8DA1007000E084370470000D5
:103C500010B5044601218020F7F7AAFA607A0128FE
:103C600005D14248C078102108434049C870607AA5
:103C7000A22805D13E48007F802108433C490877AF
:103C8000607A3B49087700203A4948770846407FE8
:103C90002178084337494877E07B002805D008465B
:103CA000407F20210843334948773248407FC0088D
:103CB000C000A17A08432F4948770846807FF72142
:103CC00008402C498877E078FFF7B3FF29498874CA
:103CD000A078FFF7AEFF2749C8746078FFF7A9FF07
:103CE000244908752078002805D10846007D2179EF
:103CF000084320490875E079FFF79BFF1D49887547
:103D00006079FFF796FF1B494875A079FFF791FF8F
:103D10001849C875207AFFF78CFF164908760846BF
:103D2000807F4006400E8877E07A002806D008465B
:103D3000807F402108430F49887703E00D48807F4A
:103D40000C498877A07BFFF774FF0A498876607B6F
:103D5000FFF76FFF0749C876207B08770846807F0A
:103D6000102188430349887710BD000020040240D9
:103D700060040440404F044010B504461B48807F57
:103D800001210843194988772078FFF752FF174926
:103D900008756078FFF74DFF1449C874A078FFF7E5
:103DA00048FF1249887420780C2806DD0846407FB9
:103DB000082108430D49487709E00C48407F0B492A
:103DC00048770846007DE1780843084908750748A8
:103DD000807F400840000549887700BF0348807F06
:103DE000022108400028F9D110BD0000404F0440D6
:103DF00010B5002014490876162007F019FE00219E
:103E0000124801761248407F8021084310494877C4
:103E10000846807F012108430D49887700BF0C4880
:103E2000807F022108400028F9D00948807F40089F
:103E300040000749887700BF0548807F022108407D
:103E40000028F9D110BD00004060004040610040F2
:103E5000404F044010B50020074908700021202081
:103E6000F7F7A6F9012105480175002004490875F6
:103E7000152007F0C5FD10BD005004404061004012
:103E80004060004070B504460D46002C14D0002D53
:103E900012D0042D10D800F013F800280CD1002601
:103EA00008E00649885D22460121F5F769F9A41C5E
:103EB000701CC6B2AE42F4DB70BD0000F4000020FE
:103EC00000200549897DC907C90F002901D00120BB
:103ED00000E00020704700000050044030B585B07D
:103EE00005460C460020039004900090019002903B
:103EF000072C0BDC0120A04081B2684681810121A2
:103F0000C17303A90220FBF7B7FB3EE0082C01D0E8
:103F1000092C0BD10120A04081B26846818101218A
:103F2000C17303A90120FBF7A7FB2EE00A2C03D0E5
:103F30000B2C01D00D2C0BD10120A04081B2684682
:103F400081810121C17303A90020FBF795FB1CE0CF
:103F50000C2C01D00F2C0BD10120A04081B268465F
:103F600081810121C17303A90E20FBF785FB0CE0C1
:103F70000E2C0AD10120A04081B268468181012126
:103F8000C17303A90C20FBF777FB00216846017081
:103F9000C17041700121817000210171C1720D2138
:103FA0008172FF21017200214172F5F749F903493D
:103FB0001520FDF711FC05B030BD00000D3C0100DF
:103FC00010B5002010490875152007F019FD0021D3
:103FD0000E4801751520002809DB00BF00BFC2068E
:103FE000D20E012191400A4A116000BF00BF00BFFC
:103FF000084880798011032805D006480078802180
:1040000008430449087010BD406000404061004012
:1040100000E100E00050044010B5F5F70BFA10BDC8
:1040200010B501231A4600211846F7F77DF8012242
:1040300011461046F7F7EEF8F7F7DAF8034807F0FD
:10404000EBFF02480249086010BD00000090D00359
:10405000B806002000BF0448006904210843024953
:10406000086130BF00BF704700ED00E0F3B585B0D8
:104070000546002003900490EEB22804070E0F2F8F
:1040800054DA082E52DA002009E00C214143284A74
:10409000515AA94201D1044603E0411CC8B2172875
:1040A000F3D300BF0120B04086B20C20604320490A
:1040B0004018C3780C20604340188278F8B231462B
:1040C0000190FBF77DFB6846868101218173002109
:1040D000C17302214174F8B203A9FBF7CDFA0C2198
:1040E0006143134A8918C888FCF736FA0C206043EC
:1040F0000F494018C1886846018169460698887250
:1041000002A8FCF743F90C226243094BD2189168CC
:104110000C226243D21804201056FDF75DFB0C21DF
:104120006143034A8918C888FCF79AF907B0F0BDC3
:10413000BCCA0100FEB505460C460020C0430290F3
:10414000EFB22804060E0F2E42DA082F40DA0120C3
:10415000B8406946088080202040002816D1012000
:104160008870A007800F022801D1487109E0A007DC
:10417000800F012802D16946487102E0002069469B
:104180004871F0B26946FBF777FA1FE000206946F4
:1041900088700E202040002800D000BF1020204052
:1041A000002802D16946087102E0012069460871C1
:1041B000E007C00F002802D16946887102E00120A3
:1041C00069468871F0B26946FBF756FA0020029002
:1041D0000298FEBD30B50146CAB20C04230E002081
:1041E0000F2B0FDA082A0DDA01249440A2B2064CF4
:1041F00003252D026419E45C1440002C01D0012039
:1042000000E0002030BD000000000440F8B5044686
:104210000F460020C0430090E6B22004050E0F2D8B
:1042200011DA082E0FDA0120B04086B2002F04D137
:10423000E8B23146FBF71CFB03E0E8B23146FBF77E
:1042400027FB002000900098F8BD00001649897FE8
:1042500001221143144A917700BF1349897F02223A
:1042600011400029F9D01049897C81700E49C97C20
:1042700041700D49097D01700B498A7D8271497D2C
:1042800001710949CA7D42710A7EC271897F49085C
:104290004900054A917700BF0349897F02221140F6
:1042A0000029F9D170470000404F044003B585B0A4
:1042B0000020019002900390049000216846417311
:1042C000817E01A8C1706846417E01A88170684660
:1042D000017E4171002101A8017108216846017128
:1042E000817D01A8C1716846C17D4172417D01A8EF
:1042F00081716846017D01A80172002168468173C1
:10430000C17301A881730C21417341216846017476
:104310000021C17401A8FFF79BFC1A200449888280
:1043200004491620FDF758FA00F006F807B000BD62
:10433000204F044021C1010010B5FFF759FD10BD09
:1043400070B504460D46601E0D49884200D901240F
:10435000002C00D1012440200A490870084600784A
:104360006043094948610321081F07F079FB0020D9
:1043700005498861072008610448056070BD000098
:10438000FFFFFF00E400002000E000E0E00000206C
:104390000020C043002809DBC206D20E0121914053
:1043A000054A1160BFF34F8FBFF36F8F00BF00202E
:1043B000024908618861704780E100E000E000E0A8
:1043C00010B507F0F3FA10BD1A20084908722B2027
:1043D00048723C2088724D20C8727F2004490968C9
:1043E0000860AC2003494870704700000004024098
:1043F000E80000200010024000B5184800780128AD
:1044000012D117480078642809DB02201549487149
:1044100008710020124908701049087004E0104823
:104420000078401C0E4908700F480078012814D10C
:104430000E480078012804D100200C4908700C496E
:1044400008700B480078322802DBF8F7ADF904E079
:1044500007480078401C0649087000BD8906002006
:1044600088060020780600208206002084060020AE
:1044700083060020FFB581B00E461746012F07D1F5
:10448000F748407D00090001C01DF549487505E069
:10449000F348407D00090001F1494875049801285E
:1044A0007ED10A210198F3F74BFE0546ED48445DA5
:1044B000E007C00F002807D0E948007C0009000190
:1044C000C01DE749087405E0E548007C00090001CB
:1044D000E349087402202040002807D0E048C07B50
:1044E000F02188437030DE49C87305E0DC48C07BAA
:1044F000F0218843DA49C87304202040002807D0FF
:10450000D748807C00090001C01DD549887405E0AA
:10451000D348807C00090001D149887408202040DC
:10452000002807D0CE48407CF02188437030CC4929
:10453000487405E0CA48407CF0218843C849487463
:1045400010202040002807D0C548407C0009000109
:10455000C01DC349487405E0C148407C0009000102
:10456000BF49487420202040002807D0BC48007C68
:10457000F02188437030BA49087405E0B848007CDF
:10458000F0218843B649087440202040002808D014
:10459000B348807CF02188437030B149887406E0CC
:1045A0008BE0AF48807CF0218843AD4988740A21B4
:1045B0000198F3F7C5FD0D46AA48445DE007C00F1A
:1045C000002807D0A648807BF02188437030A4499A
:1045D000887305E0A248807BF0218843A049887356
:1045E00002202040002807D09D48807B0009000160
:1045F000C01D9B49887305E09948807B0009000134
:104600009749887304202040002807D09448007DF3
:10461000F021884370309249087505E09048007D8C
:10462000F02188438E49087508202040002807D0D3
:104630008B48007D00090001C01D8949087505E00F
:104640008748007D00090001854908751020204039
:10465000002807D08248C07CF02188437030804910
:10466000C87405E07E48C07CF02188437C49C8744A
:1046700020202040002807D07948C07B0009000195
:10468000C01D7749C87305E07548C07B000900016B
:104690007349C87340202040002807D07048C07C70
:1046A00000090001C01D6E49C87454E06C48C07C0C
:1046B000000900016A49C8744DE06948007C00099E
:1046C0000001674908740846C07BF02188436449AB
:1046D000C8730846807C0009000188740846407C45
:1046E000F02188435E4948740846407C0009000177
:1046F00048740846007CF0218843594908740846EC
:10470000807CF0218843564988740846807BF021DC
:104710008843534988730846807B000900018873E9
:104720000846007DF02188434D4908750846007D04
:104730000009000108750846C07CF02188434849FB
:10474000C8740846C07B00090001C8730846C07CD5
:1047500000090001C8740A9801287DD10A21304659
:10476000F3F7EEFC05463F48445DE007C00F002824
:1047700007D03B48407B00090001C01D3849487301
:1047800005E03748407B00090001354948730220A5
:104790002040002807D03248007BF0218843703049
:1047A0002F49087305E02E48007BF02188432C49EF
:1047B000087304202040002807D02948807DF0217C
:1047C000884370302649887505E02548807DF021B2
:1047D00088432349887508202040002807D02048B6
:1047E000807D00090001C01D1D49887505E01C4839
:1047F000807D000900011A4988751020204000289A
:1048000007D01748407DF02188437030144948751F
:1048100005E01348407DF021884311494875202068
:104820002040002807D00E48407BF021884370309C
:104830000B49487305E00A48407BF021884308494A
:1048400048734020204000280ED00548C07D000954
:104850000001C01D024900E092E0C8750AE00000B6
:104860002412002008C801006D48C07D0009000125
:104870006B49C8750A213046F3F762FC0D4669485A
:10488000445DE007C00F002807D06548C07AF021DA
:10489000884370306249C87205E06148C07AF021EF
:1048A00088435F49C87202202040002807D05C4836
:1048B000C07A00090001C01D5949C87205E0584876
:1048C000C07A000900015649C8720420204000281F
:1048D00007D05348407E00090001C01D504948766A
:1048E00005E04F48407E000900014D494876082008
:1048F0002040002807D04A48007EF02188437030CD
:104900004749087605E04648007EF021884344493F
:10491000087610202040002807D04148007E00097A
:104920000001C01D3E49087605E03D48007E0009B3
:1049300000013B49087620202040002807D0384855
:10494000007B00090001C01D3549087305E03448AB
:10495000007B0009000132490873402020400028F4
:1049600007D02F48C07DF021884370302C49C8758E
:1049700054E02B48C07DF02188432949C8754DE09B
:104980002748407B00090001254948730846007B01
:10499000F0218843224908730846807DF02188432E
:1049A0001F4988750846807D000900018875084602
:1049B000407DF02188431A4948750846407BF02124
:1049C0008843174948730846C07D00090001C8752F
:1049D0000846C07AF02188431149C8720846C07A57
:1049E00000090001C8720846407E000900014876AF
:1049F0000846007EF0218843094908760846007E73
:104A00000009000108760846007B000900010873D0
:104A10000846C07DF02188430149C87505B0F0BD46
:104A20002412002008C80100FFB581B00E461746C9
:104A3000019801287ED10498002828D1FB480078ED
:104A4000012824D0F7F794FDF94988421FD3FBF7DA
:104A500047FB00280DD0F748807DF0218843703057
:104A6000F44988750846C07C00090001C01DC8745F
:104A70001AE0F048807DF02188431030ED498875B8
:104A80000846C07C00090001401CC8740CE0E948DD
:104A9000807DF02188437030E64988750846C07CE7
:104AA00000090001C01DC874E248C07CF0218843A1
:104AB0007030E049C8740846007EF02188437030A9
:104AC000DC4908760846807D00090001401C887595
:104AD0000846407DF02188431030D6494875084685
:104AE000407D00090001401C48750846007DF0210A
:104AF00088431030CF4908750846007D0009000141
:104B0000401C0875330006F06DFF062E261E140C9F
:104B1000042FC848007D00090001C01DC549087563
:104B200000BFC448007DF02188437030C14908753A
:104B300000BF00E0AFE1BF48407D00090001C01D9B
:104B4000BC49487500BFBB48407DF02188437030A8
:104B5000B849487500BFB748807D00090001C01DF5
:104B6000B449887500BF00E000BF00BF049800286A
:104B70005ED1AE48007801285AD0F7F7F9FCAC496D
:104B8000884255D3AB48C07FF0218843A949C877F4
:104B90000846807F0009000188770846407FF021A1
:104BA0008843A44948770846007FF0218843A149FB
:104BB00008770846C07DF02188439E49C87508469D
:104BC000C07F00090001C8770846807FF021884334
:104BD000984988770846407F00090001C01D487742
:104BE0000846807EF0218843924988760846807E78
:104BF0000009000188760846407E000900014876D9
:104C00000846007E0009000108760846007F00097A
:104C1000000108770846C07EF02188438549C876A0
:104C20000846407EF0218843703082494876B8E1DA
:104C300064213846F3F784FA0546012D07D17D48F3
:104C4000C07FF021884370307A49C87705E0794801
:104C5000C07FF02188437749C8770A213846F3F7A7
:104C60006FFA0A210090F3F76BFA0D46642F02D316
:104C70007148445D01E07148445DE007C00F0028C1
:104C800007D06C48807F00090001C01D6949887702
:104C900005E06848807F00090001664988770220A6
:104CA0002040002807D06348407FF02188437030BF
:104CB0006049487705E05F48407FF02188435D49BF
:104CC000487704202040002807D05A48007FF02170
:104CD000884370305749087705E05648007FF02137
:104CE00088435449087708202040002807D05148BD
:104CF000C07DF021884370304E49C87505E04D48AD
:104D0000C07DF02188434B49C87510202040002801
:104D100007D04848C07F00090001C01D4549C87739
:104D200005E04448C07F000900014249C8772020BF
:104D30002040002807D03F48807FF0218843703012
:104D40003C49887705E03B48807FF021884339491A
:104D5000887740202040002807D03648407F00094F
:104D60000001C01D3349487705E03248407F000903
:104D70000001304948770A213846F3F7E1F90D463A
:104D80002D48445DE007C00F002807D02948807EE9
:104D9000F021884370302749887605E02548807ED9
:104DA000F02188432349887602202040002807D03C
:104DB0002048807E00090001C01D1E49887605E05C
:104DC0001C48807E000900011A4988760420204092
:104DD000002807D01748407E00090001C01D154972
:104DE000487605E01348407E0009000111494876E5
:104DF00008202040002807D00E48007E000900014E
:104E0000C01D0C49087605E00A48007E0009000133
:104E10000849087610202040002811D00548007F5E
:104E200000090001C01D034908770FE0B50000200C
:104E3000B80B0000F812002008C801001BC80100D0
:104E40005948007F00090001574908772020204079
:104E5000002807D05448C07EF02188437030524962
:104E6000C87605E05048C07EF02188434E49C87698
:104E700040202040002807D04B48407EF021884346
:104E80007030494948768CE04748407EF02188439D
:104E90004549487685E04448807D00090001424943
:104EA00088750846407DF02188433F49487508468B
:104EB000407D0009000148750846007DF0218843C7
:104EC000394908750846007D000900010875084643
:104ED000C07C00090001C8740846807DF021884329
:104EE000314988750846C07CF02188432E49C87432
:104EF0000846007EF02188432B4908760846C07F8B
:104F0000F02188432849C8770846807F00090001BE
:104F100088770846407FF021884323494877084630
:104F2000007FF0218843204908770846C07DF021A2
:104F300088431D49C8750846C07F00090001C8772D
:104F40000846807FF0218843174988770846407FCC
:104F50000009000148770846807EF0218843124905
:104F600088760846807E0009000188760846407EE3
:104F70000009000148760846007E00090001087615
:104F80000846007F0009000108770846C07EF0212E
:104F900088430549C8760846407EF0218843024987
:104FA000487605B0F0BD0000F812002010B50146AB
:104FB000002200200A0EFE4B985CC307DB0F002B7B
:104FC00007D0FC4BDB7FF024A3437033F94CE3772D
:104FD00005E0F84BDB7FF024A343F64CE377022394
:104FE0000340002B07D0F34BDB7F1B091B01DB1DAC
:104FF000F04CE37705E0EF4BDB7F1B091B01ED4C29
:10500000E37704230340002B07D0EA4B9B7F1B0967
:105010001B01DB1DE74CA37705E0E64B9B7F1B09DB
:105020001B01E44CA37708230340002B09D0E14B7C
:1050300020335B781B091B01DB1DDE4C20346370C1
:1050400007E0DC4B20335B781B091B01D94C203473
:10505000637010230340002B09D0D64B20331B78FC
:10506000F024A3437033D34C2034237007E0D14B9A
:1050700020331B78F024A343CE4C2034237020230C
:105080000340002B09D0CB4B20331B781B091B019D
:10509000DB1DC84C2034237007E0C64B20331B783F
:1050A0001B091B01C34C2034237040230340002BF9
:1050B00007D0C04B9B7FF024A3437033BD4CA37734
:1050C00005E0BC4B9B7FF024A343BA4CA377FF239E
:1050D0001B040B401A0CB64B985CC307DB0F002B6C
:1050E00007D0B44B1B7F1B091B01DB1DB14C237781
:1050F00005E0B04B1B7F1B091B01AE4C237702233D
:105100000340002B07D0AB4BDB7EF024A34370336E
:10511000A84CE37605E0A74BDB7EF024A343A54C27
:10512000E37604230340002B07D0A24B9B7EF024A0
:10513000A34370339F4CA37605E09E4B9B7EF024E7
:10514000A3439C4CA37608230340002B07D0994B24
:105150005B7FF024A3437033964C637705E0954B57
:105160005B7FF024A343934C637710230340002B11
:1051700007D0904B5B7F1B091B01DB1D8D4C6377B8
:1051800005E08C4B5B7F1B091B018A4C6377202356
:105190000340002B07D0874B1B7FF024A3437033C1
:1051A000844C237705E0834B1B7FF024A343814C81
:1051B000237740230340002B07D07E4BDB7E1B0967
:1051C0001B01DB1D7B4CE37605E07A4BDB7E1B0984
:1051D0001B01784CE376FF231B020B401A0A744B29
:1051E000985CC307DB0F002B07D0724B1B7EF024AB
:1051F000A34370336F4C237605E06E4B1B7EF02487
:10520000A3436C4C237602230340002B07D0694B49
:105210001B7E1B091B01DB1D664C237605E0654BDD
:105220001B7E1B091B01634C237604230340002BC8
:1052300007D0604BDB7D1B091B01DB1D5D4CE3755B
:1052400005E05C4BDB7D1B091B015A4CE375082311
:105250000340002B07D0574B9B7E1B091B01DB1D16
:10526000544CA37605E0534B9B7E1B091B01514C0C
:10527000A37610230340002B07D04E4B5B7EF02417
:10528000A34370334B4C637605E04A4B5B7EF024BE
:10529000A343484C637620230340002B07D0454BA3
:1052A0005B7E1B091B01DB1D424C637605E0414B15
:1052B0005B7E1B091B013F4C637640230340002BA0
:1052C00007D03C4BDB7DF024A3437033394CE375AE
:1052D00005E0384BDB7DF024A343364CE375CAB2BE
:1052E000334B985CC307DB0F002B07D0314B1B7D82
:1052F000F024A34370332F4C237505E02D4B1B7D09
:10530000F024A3432B4C237502230340002B07D02A
:10531000284B1B7D1B091B01DB1D264C237505E05B
:10532000244B1B7D1B091B01224C237504230340C6
:10533000002B07D01F4BDB7C1B091B01DB1D1D4C09
:10534000E37405E01B4BDB7C1B091B01194CE37468
:1053500008230340002B07D0164B9B7CF024A3436B
:105360007033144CA37405E0124B9B7CF024A343D0
:10537000104CA37410230340002B07D00D4B5B7D12
:10538000F024A34370330B4C637505E0094B5B7D40
:10539000F024A343074C637520230340002B0BD05C
:1053A000044B5B7D1B091B01DB1D024C637509E08F
:1053B00008C80100D81200200C4B5B7D1B091B01A3
:1053C0000A4C637540230340002B07D0074BDB7C5E
:1053D000F024A3437033054CE37405E0034BDB7CFE
:1053E000F024A343014CE37410BD0000D812002048
:1053F00000B501287ED1FE4AD278F0239A4370325C
:10540000FB4BDA701A46127912091201D21D1A7179
:105410001A461279F0239A437032F54B1A711A46E4
:10542000527912091201D21D5A711A465279F0238B
:105430009A437032EE4B5A711A46D2791209120110
:10544000D21DDA711A46D279F0239A437032E84BB2
:10545000DA711A46527A12091201D21D5A721A468C
:10546000527AF0239A437032E14B5A721A46927A7A
:10547000F0239A437032DE4B9A721A469278F023E8
:105480009A437032DA4B9A701A46D27A1209120194
:10549000D21DDA721A46527812091201D21D5A70C0
:1054A0001A46D27AF0239A437032D14BDA721A46F6
:1054B000203AD27FF0239A437032CD4B203BDA77EB
:1054C000CB4A127B12091201D21D20331A731A46DD
:1054D000203A927F12091201D21D203B9A77C44ACA
:1054E000127BF0239A437032C14B1A731A46203A4A
:1054F000127F00E0F2E1F0239A437032BC4B203B74
:105500001A77BB4A527B12091201D21D20335A73FB
:105510001A46203AD27E12091201D21D203BDA76B9
:10552000B44AD278F0239A437032B24BDA701A46FA
:10553000127B12091201D21D1A731A46127912092E
:105540001201D21D1A711A46927AF0239A437032D0
:10555000A84B9A721A461279F0239A437032A54BDF
:105560001A711A46527912091201D21D5A711A463D
:10557000927912091201D21D9A711A46127A1209F1
:105580001201D21D1A721A46127AF0239A4370320F
:10559000984B1A721A46527A12091201D21D5A7287
:1055A000934A927912091201521C914B9A711A4630
:1055B0009279F0239A4310328D4B9A711A46127ADF
:1055C00012091201521C1A721A46127AF0239A43D7
:1055D0001032874B1A721A46927A12091201521C23
:1055E0009A721A46D27812091201521CDA701A46BF
:1055F000927812091201521C9A701A465278F023BE
:105600009A4310327A4B5A701A461278F0239A4312
:105610001032774B1A701A46127812091201521C76
:105620001A701A46203AD27F12091201521C203BEE
:10563000DA771A46927FF0239A4310326C4B203B64
:105640009A771A46527FF0239A431032684B203BD8
:105650005A771A46527F12091201521C5A771A467B
:10566000127F12091201521C1A771A46D27EF023B9
:105670009A4310325E4B203BDA761A46927EF02334
:105680009A4310325A4B203B9A765A4A127BF023A7
:105690009A431032574B1A731A46D27AF0239A4320
:1056A0001032544BDA721A46D27A12091201521C85
:1056B000DA721A46927A12091201521C9A721A462A
:1056C000527AF0239A4310324A4B5A721A46527950
:1056D000F0239A431032474B5A711A46D279F0237D
:1056E0009A431032434BDA710B0006F07BF919F341
:1056F000E9DFD5CBC1B7ADA3998F87786E645A50D7
:10570000463E362E261E160EF5003A4AD279F02372
:105710009A437032374BDA7100BF364A5279F02320
:105720009A437032334B5A7100BF324A527AF02397
:105730009A4370322F4B5A7200BF2E4A927A120946
:105740001201D21D2B4B9A7200BF2A4AD27A12093B
:105750001201D21D274BDA7200BF264AD27AF023FB
:105760009A437032234BDA7200BF224A127BF02335
:105770009A4370321F4B1A7300BF1D4A203A927E23
:10578000F0239A4370321A4B203B9A7600BF184A96
:10579000203AD27EF0239A437032154B203BDA76C2
:1057A00000BF134A203A127F12091201D21D104B7A
:1057B000203B1A7700BF0E4A203A527F120912018D
:1057C000D21D0B4B203B5A7700BF094A203A527F2B
:1057D000F0239A437032064B203B5A7700BF044AAD
:1057E000203A927FF0239A437032014B203B03E032
:1057F00044120020181300209A7700BFDC4AD27FA1
:1058000012091201D21DDA4BDA7700BFD84A2032D2
:10581000127812091201D21DD54B20331A7000BF25
:10582000D34A20321278F0239A437032D04B20337F
:105830001A7000BFCE4A20325278F0239A43703259
:10584000CB4B20335A7000BFC94A203292781209DC
:105850001201D21DC64B20339A7000BFC44A2032B9
:10586000D27812091201D21DC14B2033DA7000BF69
:10587000BF4A2032927A12091201D21DBC4B20334A
:105880009A7200BFBA4A2032127AF0239A437032D9
:10589000B74B20331A7200BFB54A2032127A120970
:1058A0001201D21DB24B20331A7200BFB04A20320F
:1058B0009279F0239A437032AD4B20339A7100BF36
:1058C000AB4A2032927912091201D21DA84B203323
:1058D0009A7100BF01E0FFE700BF47E1A44A203210
:1058E000D278F0239A43A24B2033DA701A46127909
:1058F000120912011A711A461279F0239A439C4B2D
:1059000020331A711A465279120912015A711A4635
:105910005279F0239A43964B20335A711A46D27922
:1059200012091201DA711A46D279F0239A43904B88
:105930002033DA711A46527A120912015A721A4643
:10594000527AF0239A438A4B20335A721A46927A3B
:10595000F0239A43864B20339A721A469278F023AA
:105960009A43834B20339A701A46D27A1209120155
:10597000DA721A465278120912015A701A46D27A0D
:10598000F0239A437A4B2033DA72794AD27FF0239C
:105990009A43774BDA771A462032127B12091201AA
:1059A00020331A73724A927F12091201203B9A77B0
:1059B0001A462032127BF0239A436D4B20331A7320
:1059C0006B4A127FF0239A43694B1A771A462032AA
:1059D000527B1209120120335A73654AD27E120992
:1059E0001201203BDA76634AD278F0239A43614B66
:1059F000DA701A46127B120912011A731A461279CA
:105A0000120912011A711A46927AF0239A43594BDD
:105A10009A721A461279F0239A43564B1A711A4613
:105A20005279120912015A711A4692791209120119
:105A30009A711A46127A120912011A721A46127AC9
:105A4000F0239A434B4B1A721A46527A12091201EA
:105A50005A72474A2032927912091201444B20337C
:105A60009A711A469279F0239A43414B20339A71E6
:105A70001A46127A120912011A721A46127AF02381
:105A80009A433B4B20331A721A46927A120912013A
:105A90009A721A46D27812091201DA701A4692786E
:105AA000120912019A701A465278F0239A43304B29
:105AB00020335A701A461278F0239A432C4B203325
:105AC0001A701A461278120912011A70284AD27FE7
:105AD00012091201203BDA771A46927FF0239A438B
:105AE000234B9A771A46527FF0239A43204B5A77DA
:105AF0001A46527F120912015A771A46127F12096A
:105B000012011A771A46D27EF0239A43184BDA769E
:105B10001A46927EF0239A43154B9A76154A127BC9
:105B2000F0239A43134B1A731A46D27AF0239A43FE
:105B3000104BDA721A46D27A12091201DA721A4638
:105B4000927A120912019A721A46527AF0239A43F3
:105B5000084B5A721A465279F0239A43054B5A71F0
:105B60001A46D279F0239A43024BDA7100BD000045
:105B7000241200201813002070B505460C46012D94
:105B80007ED1A548407D00090001C01DA24948758D
:105B90000846007DF021884310309F49087508466B
:105BA000007D00090001401C08750846C07CF021FA
:105BB000884310309849C8740846807CF021884397
:105BC0001030954988740846807C00090001401C0B
:105BD0008874FAF7C5FA022869D19048007801283C
:105BE00065D0FAF77DFA00282FD08B48007DF02190
:105BF00088437030884908750846007D0009000117
:105C0000C01D08750846C07CF02188437030824969
:105C1000C8740846807CF021884370307E498874BF
:105C20000846807C00090001C01D88740846407D3C
:105C3000F02188437030784948750846407CF0214F
:105C40008843703074494874E4E07348007DF02163
:105C500088431030704908750846007D000900012E
:105C6000401C08750846C07CF021884310306A4902
:105C7000C8740846807CF02188431030664900E0F3
:105C80009BE088740846807C00090001401C8874F1
:105C90000846407DF021884310305F49487508462A
:105CA000407CF021884310305B494874B2E0FAF739
:105CB0008DF9002820D1FAF713FA00280ED05648A3
:105CC000407DF02188437030534948750846407C38
:105CD000F02188437030504948740DE04E48407DB3
:105CE000F021884310304C4948750846407CF0212B
:105CF0008843103048494874FAF768F901282AD1D6
:105D000046480078012826D0F6F732FC44498842FC
:105D100021D34148407DF021884370303E49487589
:105D20000846407CF021884370303B494874FAF7BC
:105D3000D7F9002807D03848007DF021884370301B
:105D40003549087566E03448007DF02188431030FD
:105D5000314908755EE0230005F044FE062C241C42
:105D6000140C042D2C48807C00090001C01D2A4918
:105D7000887400BF2848807CF02188437030264911
:105D8000887400BF2448C07CF021884370302249C9
:105D9000C87400BF2048007D00090001C01D1E49D5
:105DA000087500BF1C48007DF021884370301A49F7
:105DB000087500BF00E000BF2CE01748407DF021CF
:105DC0008843154948750846007DF02188431249EB
:105DD00008750846007D0009000108750846C07C6A
:105DE000F02188430C49C8740846807CF021884320
:105DF000094988740846807C0009000188740846B7
:105E0000407D0009000148750846407CF021884328
:105E10000149487470BD000044120020B500002004
:105E2000B80B000030B50246002901D1002000E087
:105E30000720130005F0D6FD0F09141F2B37435020
:105E40005D67727C88929FA9B500574B5B7EF024FA
:105E5000A3430401F0252C402343534C6376A1E077
:105E6000524B9B79F024A3430401F0252C4023439B
:105E70004E4CA37196E04D4B2033DB791B091B017F
:105E80000407240F2343494C2034E3718AE0464B36
:105E90002033DB7C1B091B010407240F2343424CE6
:105EA0002034E3747EE0404B40331B781B091B0118
:105EB0000407240F23433C4C4034237072E03A4BD8
:105EC0002033DB7FF024A3430401F0252C4023433F
:105ED000354C2034E37765E0334B20335B7BF02493
:105EE000A3430401F0252C4023432F4C203463733B
:105EF00058E02E4B9B791B091B010407240F2343F9
:105F00002A4CA3714EE0294B9B7CF024A34304014F
:105F1000F0252C402343254CA37443E0234BDB7E28
:105F20001B091B010407240F2343204CE37639E0AF
:105F30001D4B2033DB7F1B091B010407240F234368
:105F4000194C2034E3772DE0174B9B7E1B091B0176
:105F50000407240F2343144CA37623E0134B203370
:105F60009B79F024A3430401F0252C4023430F4CDC
:105F70002034A37116E00D4BDB7D1B091B010407C8
:105F8000240F2343094CE3750CE0074B20335B7C63
:105F90001B091B010407240F2343034C20346374A3
:105FA00000E000BF00BF30BD24120020F812002026
:105FB000F7B582B007460E460121FF200830FEF7F4
:105FC00025F90121FC48FEF721F9FC480078012859
:105FD0007ED0F6F7CDFAFA49884279D3FAF702F87B
:105FE000032843D1F9F7F8FF002803D0F9F7F4FFAD
:105FF00001283BD1002F1CD1FAF772F800280CD0F1
:10600000F048407CF0218843EE4948740846807C83
:1060100000090001C01D8874EEE0EA48407CF021D0
:106020008843E84948740846807C00090001887468
:10603000E2E0FAF755F800280CD0E248407CF02165
:1060400088437030DF4948740846807C00090001AD
:106050008874D1E0DB48407CF0218843D9494874FA
:106060000846807C000900018874C5E0F9F7B4FF98
:10607000002803D0F9F7B0FF012865D1002F0CD11B
:10608000D048407CF0218843CE4948740846807C43
:1060900000090001C01D88740BE0CA48407CF02153
:1060A00088437030C74948740846807C0009000165
:1060B0008874F9F791FF002821D1C2482030C078B8
:1060C000F02188437030BF492031C870BD4800E0DE
:1060D00064E0807D00090001203988750846807DD4
:1060E000F0218843B7498875642223210020FCF7FA
:1060F000EFFA002222211046FCF7EAFA7CE0F9F7D9
:106100006BFF012878D1AF482030C078F021884358
:10611000AC492031C870AB48807D00090001C01D2A
:10612000203988750846807DF02188437030A54964
:106130008875002223211046FCF7CAFA6422222126
:106140000020FCF7C5FA57E09E48407CF0218843C8
:106150009C4948740846807C000900018874084600
:106160002030C078F021884396492031C870954886
:10617000807D00090001203988750846807DF02166
:10618000884390498875002223211046FCF7A0FA25
:10619000002222211046FCF79BFA2DE08948407C22
:1061A000F02188437030874948740846807C000994
:1061B0000001C01D887408462030C078F021884353
:1061C000703080492031C8707E48807D0009000110
:1061D000C01D203988750846807DF02188437030C5
:1061E00078498875642223210020FCF771FA642223
:1061F00022210020FCF76CFAF9F7EEFE002808D007
:106200006E480078012804D0F6F7B2F96C4988424C
:1062100076D26D48864209D96A4820304079F0210B
:106220008843703067492031487107E06548203065
:106230004079F021884363492031487163493046F1
:10624000F1F77EFF0A210190F1F77AFF0D465E48D3
:10625000401C864202D35E48445D01E05D48445DD7
:10626000E007C00F002809D056482030C078000948
:106270000001C01D53492031C87007E0514820304B
:10628000C078000900014F492031C8700220204029
:10629000002809D04B4820308078F02188437030A6
:1062A00048492031887007E0464820308078F02146
:1062B000884344492031887004202040002809D0B8
:1062C000404820304078F021884370303D492031EB
:1062D000487007E03B4820304078F0218843394936
:1062E000203148700820204000280AD0354820304E
:1062F000407900090001C01D32492031487108E091
:10630000A1E2304820304079000900012D492031B8
:10631000487110202040002809D02A4820300079F8
:10632000F0218843703027492031087107E0254863
:1063300020300079F0218843224920310871202043
:106340002040002809D01F482030007900090001B2
:10635000C01D1C492031087107E01A48203000791F
:106360000009000117492031087140202040002811
:1063700009D014482030807800090001C01D11495F
:106380002031887007E00F48203080780009000134
:106390000C49203188707D21C9003046F1F7D0FECC
:1063A0000A210190F1F7CCFE0D460848864213D32E
:1063B0000748445D12E0000005050000B50000201C
:1063C000B80B0000D81200209F86010010270000A3
:1063D00008C801001BC80100F948445DE007C00F70
:1063E000002807D0F748C07FF02188437030F54976
:1063F000C87705E0F348C07FF0218843F149C877AA
:1064000002202040002807D0EE48C07F000900018C
:10641000C01DEC49C87705E0EA48C07F00090001CB
:10642000E849C87704202040002807D0E548807F4D
:1064300000090001C01DE349887705E0E148807F3D
:1064400000090001DF49887708202040002809D092
:10645000DC482030407800090001C01DD9492031B6
:10646000487007E0D7482030407800090001D5493E
:106470002031487010202040002809D0D148203019
:106480000078F02188437030CE492031087007E051
:10649000CC4820300078F0218843CA492031087068
:1064A00020202040002809D0C6482030007800096C
:1064B0000001C01DC3492031087007E0C1482030E9
:1064C000007800090001BF492031087040202040B9
:1064D000002807D0BB48807FF02188437030B9493D
:1064E000887705E0B748807FF0218843B5498877F1
:1064F00064213046F1F724FE0A210190F1F720FED5
:106500000D467D20C000864202D3AF48445D01E0C5
:10651000AB48445DE007C00F002807D0A948007FC2
:1065200000090001C01DA749087705E0A548007FC4
:1065300000090001A349087702202040002807D065
:10654000A048C07EF021884370309E49C87605E09F
:106550009C48C07EF02188439A49C8760420204098
:10656000002807D09748807EF021884370309549F5
:10657000887605E09348807EF021884391498876AB
:1065800008202040002807D08E48407FF021884313
:1065900070308C49487705E08A48407FF021884375
:1065A0008849487710202040002807D08548407F40
:1065B00000090001C01D8349487705E08148407FFC
:1065C000000900017F49487720202040002807D09B
:1065D0007C48007FF021884370307A49087705E0D5
:1065E0007848007FF0218843764908774020204092
:1065F000002807D07348C07E00090001C01D714902
:10660000C87605E06F48C07E000900016D49C87674
:106610000A213046F1F794FD0A210190F1F790FD2F
:106620000D46642E02D36848445D01E06448445D31
:10663000E007C00F002807D06248007EF0218843A1
:1066400070306049087605E05E48007EF02188439E
:106650005C49087602202040002807D05948007E77
:1066600000090001C01D5749087605E05548007E25
:10667000000900015349087604202040002807D073
:106680005048C07D00090001C01D4E49C87505E095
:106690004C48C07D000900014A49C87508202040C7
:1066A000002807D04748807E00090001C01D4549E9
:1066B000887605E04348807E0009000141498876DC
:1066C00010202040002807D03E48407EF02188431B
:1066D00070303C49487605E03A48407EF0218843D6
:1066E0003849487620202040002807D03548407E91
:1066F00000090001C01D3349487605E03148407E5D
:10670000000900012F49487640202040002807D08A
:106710002C48C07DF021884370302A49C87505E0B7
:106720002848C07DF02188432649C8750A21304693
:10673000F1F706FD0D462448445DE007C00F002830
:1067400007D02048007DF021884370301D4908752E
:1067500005E01C48007DF02188431A490875022095
:106760002040002807D01748007D00090001C01D07
:106770001449087505E01348007D0009000111491E
:10678000087504202040002807D00E48C07C00096E
:106790000001C01D0B49C87405E00A48C07C00090F
:1067A00000010849C8740820204000280ED0054880
:1067B000807CF02188437030024988740CE000002E
:1067C0001BC80100D812002008C80100FA48807CCC
:1067D000F0218843F849887410202040002807D011
:1067E000F548407DF02188437030F349487505E055
:1067F000F148407DF0218843EF4948752020204032
:10680000002807D0EC48407D00090001C01DEA497E
:10681000487505E0E848407D00090001E6494875F3
:1068200040202040002807D0E348C07CF021884366
:106830007030E149C8746DE2DF48C07CF0218843C4
:10684000DD49C874F7E7F9F7C7FB01287CD1DA48BE
:1068500020304079F0218843D749203148710846DB
:10686000C07800090001C87008468078F02188438C
:10687000D1492031887008464078F0218843CE49BC
:1068800020314870084640790009000148710846E7
:106890000079F0218843C849203108710846007901
:1068A000000900010871084680780009000188701D
:1068B0007D21C9000498F1F743FC0546BF48445DBB
:1068C000E007C00F002807D0BB48C07FF0218843F5
:1068D0007030B949C87705E0B748C07FF0218843D8
:1068E000B549C87702202040002807D0B248C07FB1
:1068F00000090001C01DB049C87705E0AE48C07F5F
:1069000000090001AC49C87704202040002807D0C6
:10691000A948807F00090001C01DA749887705E0CC
:10692000A548807F00090001A349887708202040FE
:1069300000280AD0A0482030407800090001C01D7E
:106940009D492031487008E0ECE19B4820304078B8
:10695000000900019849203148701020204000288B
:1069600009D0954820300078F02188437030924952
:106970002031087007E0904820300078F0218843EB
:106980008D492031087020202040002809D08A48F5
:106990002030007800090001C01D874920310870AF
:1069A00007E0854820300078000900018249203145
:1069B000087040202040002807D07F48807FF021C9
:1069C000884370307C49887705E07B48807FF021E0
:1069D00088437949887764210498F1F7B1FB0A214B
:1069E0000190F1F7ADFB0D467D21C9000498884266
:1069F00002D37348445D01E07048445DE007C00F76
:106A0000002807D06C48007F00090001C01D6A49BA
:106A1000087705E06848007F0009000166490877AB
:106A200002202040002807D06348C07EF021884320
:106A300070306149C87605E05F48C07EF021884328
:106A40005D49C87604202040002807D05A48807E3F
:106A5000F021884370305849887605E05648807E9A
:106A6000F02188435449887608202040002807D028
:106A70005148407FF021884370304F49487705E006
:106A80004D48407FF02188434B49487710202040F3
:106A9000002807D04848407F00090001C01D464932
:106AA000487705E04448407F0009000142494877A3
:106AB00020202040002807D03F48007FF021884355
:106AC00070303D49087705E03B48007FF02188435E
:106AD0003949087740202040002807D03648C07E3A
:106AE00000090001C01D3449C87605E03248C07E67
:106AF000000900013049C8760A210498F1F720FB0B
:106B00000A210190F1F71CFB0D462D48445DE0077A
:106B1000C00F002807D02848007EF021884370303D
:106B20002549087605E02448007EF0218843224963
:106B3000087602202040002807D01F48007E000968
:106B40000001C01D1C49087605E01B48007E0009B5
:106B500000011949087604202040002807D0164873
:106B6000C07D00090001C01D1349C87505E0124829
:106B7000C07D000900011049C87508202040002888
:106B800007D00D48807E00090001C01D0A498876A3
:106B900005E00948807E0009000107498876102039
:106BA000204000280ED00448407EF02188437030F9
:106BB000014948760CE00000D81200201BC80100F3
:106BC00008C80100FE48407EF0218843FC49487611
:106BD00020202040002807D0F948407E000900010D
:106BE000C01DF749487605E0F548407E00090001E0
:106BF000F349487640202040002807D0F048C07D67
:106C0000F02188437030EE49C87505E0EC48C07D3E
:106C1000F0218843EA49C8750A210498F1F790FAEF
:106C20000D46E848445DE007C00F002807D0E4485F
:106C3000007DF02188437030E149087505E0E048A7
:106C4000007DF0218843DE4908750220204000289D
:106C500007D0DB48007D00090001C01DD849087538
:106C600005E0D748007D00090001D54908750420DA
:106C70002040002807D0D248C07C00090001C01D78
:106C8000CF49C87405E0CE48C07C00090001CC495A
:106C9000C87408202040002807D0C948807CF02113
:106CA00088437030C649887405E0C548807CF0216F
:106CB0008843C349887410202040002807D0C0486A
:106CC000407DF02188437030BD49487505E0BC48DF
:106CD000407DF0218843BA49487520202040002893
:106CE00007D0B748407D00090001C01DB449487570
:106CF00005E0B348407D00090001B14948754020D6
:106D00002040002807D0AE48C07CF0218843703076
:106D1000AB49C87426E2AA48C07CF0218843A84940
:106D2000C8741FE2F9F758F902287DD1A448203031
:106D30004079F0218843A249203148710021A248BE
:106D4000F4F7ACF8552830D1A048FEF72FF99C484D
:106D50002030C0780009000199492031C8700846E8
:106D60008078F02188439649203188700846407821
:106D7000F021884392492031487008464079000943
:106D80000001487108460079F02188438C49203180
:106D900008710846007900090001087108468078EA
:106DA00000090001C01D8870DCE189480078401CA2
:106DB0008749087082482030C07800090001C01D52
:106DC0007F492031C87008468078F02188437030B0
:106DD0007B492031887008464078F0218843784903
:106DE0002031487008464079000900014871084682
:106DF0000079F021884370307149203108710846CC
:106E0000007900090001C01D08710846807800095A
:106E10000001C01D88706F480078002809D1FEF776
:106E2000C5F800206A4900E04DE008706A49086032
:106E300098E167480078642824DA68480078654952
:106E40000978884204DB63480078401E6349087073
:106E500060480278624960480068F7F77DFF0028C3
:106E60002CD15E48007880005D490858002825D064
:106E70005A48007880000858574908600020544953
:106E800008701BE052480078642817DB53480078EC
:106E9000401C52490870084600784E4909788842DB
:106EA00002DB00204D4908704C48007880004C49B6
:106EB000085849490860002045490870464800685C
:106EC000FEF774F84EE1F9F787F80328B0D13C4893
:106ED00020304079F02188433949203148710846F3
:106EE000C07800090001C01DC87008468078F021F4
:106EF000884333492031887008464078F021884320
:106F000070302F492031487008464079000900014F
:106F1000C01D487108460079F02188432849203176
:106F200008710846007900090001C01D0871084673
:106F3000807800090001C01D88702148C07FF021C1
:106F400088431F49C8770846C07F00090001C877F9
:106F50000846807F00090001887708462030407885
:106F6000000900012031487008460078F02188436C
:106F700013492031087008460078000900010870A4
:106F80000F48807FF02188430D4988770846007FAD
:106F900000090001C01D08770846C07EF021884323
:106FA00070300749C8760846807EF02188437030EB
:106FB000034988760846407FF0218843703011E00D
:106FC000D812002008C80100CC0700200B0B0B0BC7
:106FD00060000020720000205C00002058000020AB
:106FE00004110020604948770846407F00090001ED
:106FF000C01D48770846007FF021884370305A4909
:1070000008770846C07E00090001C876F9F724F821
:10701000002855D15448007EF021884370305249F1
:1070200008760846007E0009000108760846C07D03
:1070300000090001C8750846807E000900018876B5
:107040000846407EF021884370304749487608461C
:10705000407E00090001C01D48760846C07DF02131
:10706000884370304049C8750846007DF021884348
:1070700070303D4908750846007D0009000108751B
:107080000846C07C00090001C8740846807CF021D5
:107090008843354988740846407DF0218843703024
:1070A000314948750846407D00090001C01D4875FA
:1070B0000846C07CF021884370302B49C87451E0E9
:1070C0002948007EF0218843703027490876084619
:1070D000007E00090001C01D08760846C07D000939
:1070E0000001C01DC8750846807E00090001887631
:1070F0000846407EF021884370301B494876084698
:10710000407E00090001C01D48760846C07DF02180
:1071100088431549C8750846007DF0218843124907
:1071200008750846007D0009000108750846C07C06
:1071300000090001C8740846807CF02188430A4990
:1071400088740846407DF021884307494875084601
:10715000407D0009000148750846C07CF021884345
:107160000149C87405B0F0BDD8120020FFB581B048
:1071700006461D46002000900027002E7ED0FE48C7
:107180008079F02188437030FB49887108462038A7
:10719000007FF02188437030F74920390877F7489D
:1071A000007801286BD0F5F7E3F9F549884266D3FA
:1071B000F8F718FF04284BD1002D24D1F8F790FFE1
:1071C000002810D0EC482038807D00090001EA49F1
:1071D000203988750846807DF02188437030E64963
:1071E0002039887597E0E4482038807D0009000147
:1071F000E149203988750846807DF0218843DE49C1
:107200002039887587E0F8F76BFF002810D0DA483E
:107210002038807D00090001C01DD74920398875BC
:107220000846807DF0218843D3492039887572E073
:10723000D1482038807D00090001CF492039887568
:107240000846807DF0218843CB492039887562E06B
:10725000002D22D1C8482038807D00090001C64990
:10726000203988750846807DF02188437030C249F6
:10727000203988750846807EF02101E052E32AE03B
:1072800088437030BC4920398876BB480079F021AA
:1072900088437030B84908713DE0B7482038807D98
:1072A00000090001C01DB449203988750846807D59
:1072B000F0218843B049203988750846807EF02146
:1072C0008843AD4920398876AB480079F02188435E
:1072D000A94908711FE0A8482038807D00090001F5
:1072E000C01DA549203988750846807DF021884356
:1072F0007030A149203988750846807EF021884386
:1073000070309D49203988769B480079F021884368
:107310007030994908710A9801287DD10A21029894
:10732000F0F70EFF0090974900980C5CE007C00F43
:10733000002807D09048C07900090001C01D8E497F
:10734000C87105E08C48C079000900018A49C871FC
:1073500002202040002807D08748807900090001DA
:10736000C01D8549887105E08348807900090001C6
:107370008149887104202040002807D07E48407948
:1073800000090001C01D7C49487105E07A48407938
:10739000000900017849487108202040002807D0E2
:1073A0007548007AF021884370307349087205E00F
:1073B0007148007AF02188436F49087210202040FC
:1073C000002807D06C48007A00090001C01D6A49F6
:1073D000087205E06848007A0009000166490872F1
:1073E00020202040002807D06348C079F02188433E
:1073F00070306149C87105E05F48C079F021884369
:107400005D49C87140202040002809D05A48407981
:10741000F0218843703000E08FE05749487105E063
:1074200055484079F0218843534948710A21029810
:10743000F0F786FE0091534900980C5CE007C00FFE
:10744000002807D04C48C07800090001C01D4A49F7
:10745000C87005E04848C078000900014649C87076
:1074600002202040002807D043488078F02188433C
:1074700070304149887005E03F488078F0218843AA
:107480003D49887004202040002807D03A484078C1
:10749000F021884370303849487005E0364840781C
:1074A000F02188433449487008202040002807D044
:1074B0003148407800090001C01D2F49487005E09F
:1074C0002D484078000900012B49487010202040C9
:1074D000002807D02848007900090001C01D26496E
:1074E000087105E02448007900090001224908716B
:1074F00020202040002807D01F48C078F021884372
:1075000070301D49C87005E01B48C078F0218843E1
:107510001949C87040202040002807D016488078BC
:1075200000090001C01D144988705DE01248807890
:10753000000900011049887056E00F484079F02199
:10754000884370300C494871084680780009000172
:10755000C01D88700846C07900090001C87108463E
:10756000807900090001887108464079000900010E
:1075700048710846007A07E064120020B500002038
:10758000B80B000008C80100F0218843FE490872CA
:107590000846007A0009000108720846C079F02107
:1075A0008843F949C8710846C07800090001C870CD
:1075B00008468078F0218843F3498870084640786F
:1075C000F0218843F04948700846407800090001DE
:1075D0004870084600790009000108710846C07823
:1075E000F0218843E849C8700B9801287ED10A2110
:1075F0000398F0F7A5FD0746E448C45DE007C00F17
:10760000002809D0E0482038407F00090001C01D53
:10761000DD492039487707E0DB482038407F000902
:107620000001D9492039487702202040002809D09C
:10763000D5482038007F00090001C01DD2492039FB
:10764000087707E0D0482038007F00090001CE49C4
:107650002039087704202040002809D0CA48203863
:10766000C07E00090001C01DC7492039C87607E067
:10767000C5482038C07E00090001C3492039C876BA
:1076800008202040002809D0BF482038807FF02102
:1076900088437030BC492039887707E0BA482038E1
:1076A000807FF0218843B849203988771020204016
:1076B000002809D0B4482038807F00090001C01D8F
:1076C000B1492039887707E0AF482038807F00092A
:1076D0000001AD49203988772020204000280BD0B8
:1076E000A9482038407FF021884300E0C4E0703092
:1076F000A5492039487707E0A3482038407FF0218A
:107700008843A1492039487740202040002809D0EB
:107710009D482038C07EF021884370309A49203936
:10772000C87607E098482038C07EF0218843964903
:107730002039C8760A210398F0F702FD0F469348D6
:10774000C45DE007C00F002809D08F482038407E74
:1077500000090001C01D8C492039487607E08A489D
:107760002038407E000900018749203948760220F0
:107770002040002809D084482038007EF02188432A
:10778000703081492039087607E07F482038007E34
:10779000F02188437C4920390876042020400028C5
:1077A00009D079482038C07DF0218843703076496F
:1077B0002039C87507E074482038C07DF02188431F
:1077C00071492039C87508202040002809D06E482A
:1077D0002038C07D00090001C01D6B492039C875E3
:1077E00007E069482038C07D00090001664920395A
:1077F000C87510202040002809D063482038807EBA
:1078000000090001C01D60492039887607E05E4804
:107810002038807E000900015B49203988762020CD
:107820002040002809D058482038407EF021884365
:10783000703055492039487607E053482038407E5B
:10784000F0218843504920394876402020400028C4
:1078500009D04D482038007E00090001C01D4A496A
:10786000203908762DE148482038007E00090001C3
:1078700045492039087624E143482038C07EF0216C
:107880008843703040492039C8760846007E000998
:107890000001C01D08760846407F000900014877B6
:1078A0000846007F0009000108770846C07E0009ED
:1078B0000001C8760846807FF0218843324920398C
:1078C00088770846807F0009000188770846407F56
:1078D000F02188432C49203948770846407E00092A
:1078E000000148760846007EF02188432649203969
:1078F00008760846C07DF021884323492039C875A1
:107900000846C07D00090001C8750846807E000950
:10791000000188760846407EF02188431A492039C4
:107920004876CEE018482038C07EF02188431649BA
:107930002039C8760846007E00090001087608460E
:10794000407F0009000148770846007F00090001D8
:1079500008770846C07E00090001C8760846807F87
:10796000F02188430849203988770846807F00093C
:10797000000188770846407FF0218843024920397A
:1079800048770846407E03E06412002008C80100E2
:107990000009000148760846007EF02188434A49E4
:1079A00008760846C07DF02188434749C8750846D7
:1079B000C07D00090001C8750846807E00090001ED
:1079C00088760846407EF02188433F49487608463D
:1079D00020304079F02188433B49203148710846E6
:1079E00080780009000188700846C079000900010C
:1079F000C8710846807900090001887108464079FD
:107A00000009000148710846007AF02188432E4998
:107A1000203108720846007A000900010872084601
:107A2000C079F021884328492031C8710846C078C0
:107A300000090001C87008468078F0218843224977
:107A40002031887008464078F02188431E49203153
:107A500048700846407800090001487008460079DF
:107A60000009000108710846C078F02188431649D2
:107A70002031C8701448807D0009000120398875C4
:107A80000846807DF02188430F4988750846807E2E
:107A9000F02188430C4988760846007FF02188430E
:107AA00009490877084620300079F02188430649C3
:107AB0002031087108468079F0218843024920313D
:107AC000887105B0F0BD000044120020F7B582B007
:107AD0000D4617460026029801287CD1632D0ADD49
:107AE0000121FF200630FCF791FB0121FF20073028
:107AF000FCF78CFB16E0092D0ADD0121FF20063082
:107B0000FCF784FB0021FF200730FCF77FFB09E036
:107B10000021FF200630FCF779FB0021FF20073011
:107B2000FCF774FBFA48007801286ED0F4F720FDCA
:107B3000F849884269D3F8F755FA032866D1002F2F
:107B400030D1F8F7CDFA002816D0F348407BF02169
:107B50008843F14948730846C07B00090001C01DF5
:107B6000C873642208210020FAF7B2FD002209211F
:107B70001046FAF7ADFD90E0E748407BF0218843DE
:107B8000E54948730846C07B00090001C87300221C
:107B900008211046FAF79CFD002209211046FAF749
:107BA00097FD7AE0F8F79CFA002818D0DA48407B75
:107BB000F02188437030D84948730846C07B0009DB
:107BC0000001C873002208211046FAF781FD6422E3
:107BD0000921002000E0ACE1FAF77AFD5DE0CE4833
:107BE000407BF0218843CC4948730846C07B00099C
:107BF0000001C873002208211046FAF769FD00222F
:107C000009211046FAF764FD47E02FE0002F16D156
:107C1000C148407BF0218843BF4948730846C07B78
:107C200000090001C01DC873642208210020FAF772
:107C30004FFD002209211046FAF74AFD2DE0B64813
:107C4000407BF02188437030B34948730846C07BBD
:107C500000090001C873002208211046FAF738FD18
:107C6000642209210020FAF733FD16E0AA48407B80
:107C7000F02188437030A84948730846C07B00094A
:107C80000001C01DC873642208210020FAF720FDFE
:107C9000642209210020FAF71BFD64212846F0F731
:107CA0004FFA0646012E09D19B482038807B0009F7
:107CB0000001C01D98492039887307E09648203894
:107CC000807B000900019449203988730A212846E5
:107CD000F0F736FA0A210190F0F732FA0E46642DD9
:107CE00002D38E48845D01E08D48845DE007C00FBB
:107CF000002807D08848407AF021884370308649B0
:107D0000487205E08448407AF021884382494872ED
:107D100002202040002807D07F48407A0009000157
:107D2000C01D7D49487205E07B48407A000900018A
:107D30007949487204202040002809D0764820382C
:107D4000007CF0218843703073492039087407E0C3
:107D500071482038007CF02188436F49203908742D
:107D600008202040002809D06B482038007C0009FA
:107D70000001C01D68492039087407E066482038B2
:107D8000007C00090001644920390874102020405B
:107D9000002809D060482038C07BF021884370302B
:107DA0005D492039C87307E05B482038C07BF0216B
:107DB000884359492039C87320202040002809D021
:107DC00055482038807BF021884370305249203953
:107DD000887307E050482038807BF02188434E4963
:107DE0002039887340202040002809D04A48203894
:107DF000C07B00090001C01D47492039C87307E056
:107E000045482038C07B0009000143492039C87328
:107E10000A212846F0F794F90E464048845DE007B1
:107E2000C00F002807D03C48407B00090001C01D5E
:107E30003949487305E03848407B0009000136495C
:107E4000487302202040002807D03348007BF021EF
:107E5000884370303049087305E02F48007BF021DB
:107E600088432D49087304202040002807D02A4861
:107E7000007B00090001C01D2749087305E0264862
:107E8000007B0009000124490873082020400028D5
:107E900007D02148C07AF021884370301E49C8724B
:107EA00005E01D48C07AF02188431B49C8721020A4
:107EB0002040002807D01848C07A00090001C01DE2
:107EC0001549C87205E01448C07A0009000112493A
:107ED000C87220202040002807D00F48807A00096F
:107EE0000001C01D0C49887205E00B48807A00092A
:107EF00000010949887240202040002812D006481D
:107F0000807AF02188437030034988727FE0000056
:107F1000B5000020B80B00006412002008C8010062
:107F20001BC801003B48807AF02188433949887298
:107F30006DE0002208211046FAF7CAFB0022092151
:107F40001046FAF7C5FB3348407BF021884331499E
:107F500048730846C07B00090001C87308462038F2
:107F6000807B00090001203988732A48407AF0217B
:107F70008843284948720846407A0009000148723F
:107F800008462038007CF0218843224920390874B3
:107F90000846007C0009000108740846C07BF021F7
:107FA00088431C492039C8730846807BF0218843E8
:107FB0001849203988730846C07B00090001C8733E
:107FC0001448407B00090001203148730846007BBB
:107FD000F02188430F4908730846007B000900011F
:107FE00008730846C07AF02188430A49C8720846D7
:107FF000C07A00090001C8720846807AF0218843DF
:10800000044988720846807A00090001887205B028
:10801000F0BD000064120020F8B507460D460026AA
:10802000002F7DD0FE48C07900090001C01DFC4929
:10803000C8710846807AF02188437030F849887208
:10804000F7F77CFE01286CD164212846F0F78EF802
:1080500086B2F448845DE007C00F002807D0F048DE
:10806000C07BF02188437030ED49C87305E0EC48CF
:10807000C07BF0218843EA49C873022020400028D1
:1080800007D0E748C07B00090001C01DE449C87360
:1080900005E0E348C07B00090001E149C873042002
:1080A0002040002807D0DE48807B00090001C01D69
:1080B000DB49887305E0DA48807B00090001D84974
:1080C000887308202040002807D0D548407C00094C
:1080D0000001C01DD249487405E0D148407C000928
:1080E0000001CF49487410202040002807D0CC4818
:1080F000007CF02188437030C949087405E0C84805
:10810000007CF0218843C6490874202020400028C4
:108110000AD0C348007C00090001C01DC04901E02D
:10812000ACE12FE1087405E0BD48007C00090001C6
:10813000BB49087440202040002807D0B848807B05
:10814000F02188437030B649887305E0B448807BDD
:10815000F0218843B24988730A212846EFF7F0FFDF
:108160000A210090EFF7ECFF0E46642D01D2002D9E
:1081700002D1AD48845D01E0AA48845DE007C00FEC
:10818000002807D0A648007BF02188437030A4491E
:10819000087305E0A248007BF0218843A0490873DA
:1081A00002202040002807D09D48007B00090001E4
:1081B000C01D9B49087305E09948007B0009000138
:1081C0009749087304202040002807D09448C07ABB
:1081D00000090001C01D9249C87205E09048C07AAC
:1081E000000900018E49C87208202040002807D0ED
:1081F0008B48407CF021884370308949487405E001
:108200008748407CF02188438549487410202040ED
:10821000002807D08248407BF02188437030804995
:10822000487305E07E48407BF02188437C494873D1
:1082300020202040002807D07948407B0009000119
:10824000C01D7749487305E07548407B000900016F
:108250007349487340202040002807D07048C07AF6
:10826000F021884370306E49C87205E06C48C07ACE
:10827000F02188436A49C8720A212846EFF760FF57
:108280000E466948845DE007C00F002807D06448A7
:10829000407A00090001C01D6149487205E060484C
:1082A000407A000900015E494872022020400028FF
:1082B00007D05B48007AF021884370305849087233
:1082C00005E05748007AF021884355490872042098
:1082D0002040002807D05248C079F02188437030F0
:1082E0004F49C87105E04E48C079F02188434C4998
:1082F000C87108202040002807D04948807C000928
:108300000001C01D4649887405E04548807C00098D
:1083100000014349887410202040002807D04048BD
:10832000807A00090001C01D3D49887205E03C4883
:10833000807A000900013A498872202020400028F4
:1083400007D03748407AF02188437030344948726A
:1083500005E03348407AF021884331494872402093
:108360002040002807D02E48007A00090001C01DD7
:108370002B49087282E02A48007A00090001284946
:1083800008727BE02648C07AF02188437030244987
:10839000C8720846007A00090001C01D087208462C
:1083A000C07BF02188431E49C8730846C07B000982
:1083B0000001C8730846807B0009000188730846E5
:1083C000407C0009000148740846007CF021884385
:1083D000134908740846007C000900010874084627
:1083E000807BF02188430E4988730846007BF0218A
:1083F00088430B4908730846007B00090001087395
:108400000846C07A00090001C8720846407CF02185
:108410008843034948740846407BF021884305E0BF
:10842000F81200201BC8010008C801001449487355
:108430000846407B0009000148730846407A00095D
:10844000000148720846007AF02188430C490872FE
:108450000846C079F02188430949C8710846807CE4
:108460000009000188740846807A000900018872BA
:108470000846407AF021884301494872F8BD00005F
:10848000F812002070B500BF0A2108480078EFF705
:108490006DFEFF21F531484384B22046EFF766FEBA
:1084A000C5B229460120FCF7A3FF70BD6200002081
:1084B00070B5044600250A210E480078EFF740FE0B
:1084C000054629460120FDF757FB01232246294690
:1084D0001846FCF7A9FA074800783B2805DA054852
:1084E0000078401C0349087002E000200149087030
:1084F00070BD000061000020F0B504460D46264620
:1085000000210020002A0CDD122007E06F5CB7423A
:1085100002D10020197003E04F1CF9B29142F5DB43
:1085200001E000271F70F0BD30B504461320002C79
:1085300008D1002A04D015788D420BDC002009E018
:10854000132007E0002A04D0D55C8D4202D1002020
:1085500000E0132030BD002000BF704770B5044616
:108560000D4600200021002A0DDD312008E04E00DC
:10857000AE5BA64202D10020197003E04E1CF1B29E
:108580009142F4DB00BF70BD10B502460020535C81
:10859000002B05D0535C034C2478A34200D0332039
:1085A00010BD00008A06002030B503460C460025A9
:1085B000F7F786FB195D0840002800D17E25284684
:1085C00030BD10B503460024F7F77AFB18400028A9
:1085D00000D17F24204610BD10B5F4F721FDF4F73B
:1085E000D7FEF5F7D3F810BD002002E000BF411C14
:1085F000C8B22828FAD3704710B500210948FBF704
:1086000099FDFFF7F1FFFFF7EFFF00210548401C40
:10861000FBF790FDFFF7E8FFFFF7E6FF02200249B6
:10862000087010BD02060000B7000020024908785B
:108630000221014A11707047B700002070B5002474
:1086400000211448FBF776FDFFF7CEFFFFF7CCFFC4
:1086500000251BE06006040E00210E48401EFBF7BB
:1086600069FDFFF7C1FFFFF7BFFFFFF7BDFF094837
:10867000FBF7B0FD044380210648401EFBF75AFD7E
:10868000FFF7B2FFFFF7B0FF681CC5B2082DE1DBB2
:10869000204670BD0306000010B502201149087085
:1086A00000211148FBF746FDFFF79EFFFFF79CFFF7
:1086B00000210D48401EFBF73DFDFFF795FFFFF73A
:1086C00093FF80210848FBF735FDFFF78DFFFFF78B
:1086D0008BFF80210448401EFBF72CFDFFF784FF31
:1086E00010BD0000B70000200306000010B50220F6
:1086F0000D49087080210D48FBF71CFDFFF774FF42
:10870000FFF772FF00210948401EFBF713FDFFF73A
:108710006BFFFFF769FF00210448FBF70BFDFFF734
:1087200063FFFFF761FF10BDB700002003060000E4
:1087300010B50446022012490870012C00D910BD62
:10874000002C04D000210F48FBF7F4FC03E080214B
:108750000C48FBF7EFFCFFF747FF00210948401EDC
:10876000FBF7E8FCFFF740FFFFF73EFF80210548DD
:10877000401EFBF7DFFCFFF737FF00BFDFE700001D
:10878000B70000200306000070B50446022024490B
:108790000870002524E080202040002804D000211B
:1087A0002048FBF7C7FC03E080211E48FBF7C2FC12
:1087B000FFF71AFFFFF718FF00211A48401EFBF7CA
:1087C000B9FCFFF711FFFFF70FFF80211548401E8E
:1087D000FBF7B0FCFFF708FF6006040E681CC5B28B
:1087E000082DD8DB00210F48FBF7A4FCFFF7FCFEA7
:1087F000FFF7FAFE00210B48401EFBF79BFCFFF73A
:10880000F3FEFFF7F1FE0748FBF7E4FC04490870AC
:1088100080210448401EFBF78DFCFFF7E5FE70BD8C
:10882000B70000200306000010B5054800680028C6
:1088300002D003480068804700F086F810BD0000B1
:10884000E000002010B519480078012811D0174821
:10885000007802280DD01648FBF7F8FC1449087878
:10886000FBF7DAF9124908704878FBF7D5F9104997
:1088700048706420F6F73AFCF2F7FAF9FFF7ACFE1D
:10888000F5F76CFBFBF7B8FD0A4800780A2807D318
:10889000002008490870FAF70BFBFAF7F1F904E039
:1088A00004480078401C0349087010BDA300002054
:1088B000AD0000200C01002010B50A20FAF760FD81
:1088C000F9F700FEF4F7F6FC0A20F2F799FE01F042
:1088D000DDFF0A20F6F7EEFD01F02EFBF4F706FEB1
:1088E00010BD10B5F8F7FCFFF8F7DAFFF5F74EF911
:1088F000F4F77EF9F4F7F0F810BD000010B5F3F7C7
:1089000057FE7D2109010648F3F7F6FA00F032FA26
:10891000F1F734FE02210348F2F7B6FD10BD000066
:10892000D8070020CC07002010B5F2F7F7F8FAF7C7
:10893000E5F801F0A9FDF7F7F3F8F8F7CFFF10BD60
:1089400010B5F6F751FB10BD10B53220F6F70CF953
:10895000F7F782F906480068401C05490860084698
:108960000068142803D300200860EFF795FE10BDBF
:10897000100100200CB500BF0548006800900448B5
:1089800000680190019900988842F5D100980CBDCB
:108990000801002000B589B00C4807900C480690EB
:1089A0000C4801900C4800900C4805900C4804902D
:1089B0000C4803900C4802900C48089000F002FC10
:1089C00069460B4800F070F909B000BD51C50000C0
:1089D000AD9101000F8A0100398A01001D8A010052
:1089E000478A01002B8A0100558A0100F5890100A0
:1089F0003CC90100704710B5FAF724FFF5F732FBC8
:108A000002F080F8F2F798F8FAF78AF810BD10B57E
:108A10000120F0F7ADFC0446204610BD10B5012042
:108A2000F0F79AFC0446204610BD10B50120F0F77F
:108A3000F1FA0446204610BD10B50020F0F798FC6E
:108A40000446204610BD10B50020F0F785FC044612
:108A5000204610BD10B50020F0F7DCFA0446204691
:108A600010BD000070B531480068314909684018F0
:108A70002E490860084600687D21C900884211D34C
:108A80002A480068EFF75CFB06467D21C9002748AD
:108A90000068EFF755FB25480160264800688019FB
:108AA000244908602448406821490968401822493F
:108AB000486008460068002837D1002508468468C9
:108AC0002EE02068002829D01B49606849680022F0
:108AD000D243511A884205D2174960684968401844
:108AE000606002E00020C0436060A1686068884266
:108AF00014D3206801280AD100202060002D03D162
:108B00000D492069886004E02069286101E00020A7
:108B10006060E068002801D0E0688047254624694D
:108B2000002CCED100200449486070BD0401002013
:108B30000001002008010020F815002010B5FBF707
:108B400027FC322000F00AF803493220FBF7F8FB3B
:108B500000F008F910BD0000658A010010B5044658
:108B60000D48046000200D4908600D4908600D495A
:108B7000086048608860FFF7FDFE0B490860002030
:108B8000486088600120C8600320086105204861B2
:108B90000720886110BD00000001002004010020B2
:108BA00008010020F8150020DC15002070B5FFF743
:108BB00022FFFFF7DFFE05463A480068A84203D8C7
:108BC000384800682C1A06E0364800680021C9437E
:108BD000081A4019441C334805604068001931499F
:108BE000486008464068022806D308460079C00756
:108BF000C00F4860FFF782FE2A48806800192949A3
:108C0000886008468068052807D388680521EFF743
:108C100097FA24488160FFF793FE2248C068001944
:108C20002049C8600846C0680A2807D3C8680A21D6
:108C3000EFF786FA1B48C160FFF73EFE194800694E
:108C400000191849086108460069142807D3086903
:108C50001421EFF775FA13480161FFF742FE11483E
:108C6000406900190F49486108464069322807D316
:108C700048693221EFF764FA0A484161FFF754FE70
:108C80000848806900190749886108468069642896
:108C900007D388696421EFF753FA02488161FFF72F
:108CA000D1FD70BDDC1500200288264B1A80428859
:108CB0005A8082889A80C288DA8002891A81428921
:108CC0005A8182899A81C289DA81028A1A82428A09
:108CD0005A82828A1C4B1A80C28A1C4B1A80028BD1
:108CE0001B4B1A80428B5A80828B9A80C28BDA800F
:108CF000028C1A81428C5A81828C9A81C28CDA81D0
:108D0000028D1A82428D5A82828D124B1A80C28D38
:108D1000114B1A80114B0A681A604A685A608A68B7
:108D20009A60CA68DA600A691A614A695A618A698E
:108D30009A61CA69DA610A6A1A625522084B1A7086
:108D4000704700003E0700203A0700203C07002043
:108D5000520700203607002038070020541A002050
:108D60003507002010B50024FAF748FF2046FAF72F
:108D700055FD10BD10B500F035F900F03FFB04487B
:108D8000006A002802D00249086A804710BD00002E
:108D9000541A002000B589B00C4807900C48069082
:108DA0000C4801900C4800900C4805900C48049029
:108DB0000C4803900C4802900C48089000F096FA7A
:108DC00069460B48FFF770FF09B000BD51C50000B0
:108DD000AD9101000F8A0100398A01001D8A01004E
:108DE000478A01002B8A0100558A0100F58901009C
:108DF0003CC9010010B580201B4948711A201A494E
:108E0000203908722B2048723C2088724D20C8728D
:108E1000002016494860F2F72DFA15490860002035
:108E2000C043144908601449086014481449086094
:108E3000114903221202891848600F498918886075
:108E40000D498918C8600C49891808610A498918B0
:108E5000486109498918886107498918C861AC20A7
:108E60000849487010BD00002004024000B00140D5
:108E7000B806002080E200E000E100E0C0C0C0C011
:108E800000E400E0001002400146002007E042003C
:108E9000054B9A5A8A4200DD03E0421CD0B20A28F0
:108EA000F5D300BF704700003E07002001460020B8
:108EB00007E04200054B9A5A8A4200DD03E0421C5B
:108EC000D0B20A28F5D300BF704700005207002037
:108ED0000148007A70470000301A00200148007AEB
:108EE00070470000241A0020FEB5002700200190E2
:108EF0000090009045E03648C069002803D034480F
:108F0000C1690220884732488068002804D030496F
:108F100088688047044600E000242D48C068002887
:108F200004D02B49C8688047054600E00025AC42C4
:108F300001DD264600E02E4626488088B04203DA4E
:108F40002448C089B04205DC00270198401CC0B20B
:108F5000019003E0781CC7B2002001900098401CEB
:108F6000C0B2009000980A2800D30EE0052F02D36B
:108F70000520194908720198052802D309201649CD
:108F800008721548007A0028B5D000BF1248007A50
:108F900000281CD05520114908700D488069002810
:108FA0000AD00B49886980470D49087208498869C9
:108FB00080470B49487203E0002009490872487253
:108FC0000348006A002802D00149086A8047FEBDB4
:108FD000541A0020520700203C1A002034070020B9
:108FE000481A0020FEB56B488069002820D06949E6
:108FF000886980476849497A884210D16648408824
:1090000066490988884205DA63484088401C6249FD
:10901000488012E06048407A5F4908720DE0002005
:109020005D4948805B49886980475B49487204E034
:109030000020594948800872487256480068002844
:1090400003D054490868804701905248406800287E
:1090500003D050494868804700900198012857D1B3
:1090600000980128FBD14B484069002804D04949A9
:1090700048698047064600E0002646480069002807
:1090800004D0444908698047074600E00027B742FA
:1090900001DD3D4600E035464148007832280FD2D8
:1090A0003F48406840193E49486008460078401CE7
:1090B00008700A4611785068EFF742F885B211E05F
:1090C00000203749087048600846406840194860E9
:1090D00008460078401C08700A4611785068EFF77F
:1090E0002FF885B22846FFF7CFFE04462C48417A78
:1090F000A1423DD100202B490880294840882A49B7
:109100000988884205DA26484088401C244948805E
:109110003EE02348007A07280ED9092C03D0082CFA
:1091200001D0072C06D109201D49087200201A49D8
:10913000087201E01A4804721948007A01280CD11B
:10914000012C01D0022C06D1012015490872002003
:109150001149087201E0124804721148007A01288E
:1091600016D00F48007A072812D80D4804720FE075
:1091700000200B4948800B480088401C09490880A2
:1091800008460088052803D300200880044844725C
:10919000FEBD0000541A0020301A00203C070020B9
:1091A000241A0020680700203A07002010B5002488
:1091B0000120FBF70FF8012801D1012400E0002471
:1091C000204610BD10B5002034490870344908709D
:1091D0004880486008724872324908704880486088
:1091E00008724872304908704880486008724872B6
:1091F0002E49087048804860087248722C480078F0
:1092000055283ED07D20C0002A49088002202A49E6
:1092100008807D20C0002949088002202849088054
:109220000020284908802848488028488880284805
:10923000C880284808817D20C0014881264888814F
:109240002648C881264808820020C0434882002062
:10925000244908801C4848801C4888801C48C880D5
:109260001C4808817D20C00148811B4888811B481B
:10927000C8811B4808820020C043488255200C4901
:1092800008701948C069002804D01748C169FF2038
:1092900005308847FFF728FE10BD00003407002086
:1092A000241A0020301A00203C1A0020481A0020FE
:1092B0003507002036070020380700203A07002035
:1092C0003C0700203E07002064190000581B0000E6
:1092D000282300001C2500007440000044480000C2
:1092E000384A000052070020541A002010B5002010
:1092F0002F4908702F4908704880486008724872EA
:109300002D49087048804860087248722B490870DF
:10931000488048600872487229490870488048604F
:10932000087248722748007855283ED07D20C0003A
:10933000254908800220254908807D20C000244955
:109340000880022023490880002023490880234800
:109350004880234888802348C880234808817D208E
:10936000C0014881214888812148C881214808825C
:109370000020C043488200201F49088017484880C9
:10938000174888801748C880174808817D20C00189
:109390004881164888811648C881164808820020EE
:1093A000C0434882552007490870FFF79DFD10BD56
:1093B00034070020241A0020301A00203C1A002014
:1093C000481A002035070020360700203807002003
:1093D0003A0700203C0700203E07002064190000E7
:1093E000581B0000282300001C25000074400000CA
:1093F00044480000384A000052070020FEB5694882
:109400008069002820D06749886980476649497A81
:10941000884210D16448408864490988884205DA46
:1094200061484088401C6049488012E05E48407AAC
:109430005D4908720DE000205B4948805949886900
:1094400080475949487204E0002057490872487221
:10945000488054480068002804D052490868804772
:10946000019001E0002001904E484068002804D09F
:109470004C4948688047009001E000200090019826
:10948000012853D100980128FBD1464840690028A3
:1094900004D0444948698047064600E00026414818
:1094A0004069002804D03F4908698047074600E02A
:1094B0000027B74201DD3D4600E035463C480078D4
:1094C00032280FD23A484068401939494860084666
:1094D0000078401C08700A4611785068EEF730FE9C
:1094E00085B211E0002032490870486008464068A3
:1094F0004019486008460078401C08700A461178F8
:109500005068EEF71DFE85B22846FFF7CFFC0446F3
:109510002748417AA14234D14088264909888842A7
:1095200005DA23484088401C2149488039E0002062
:10953000214908801E48007A092809D1092C01D048
:10954000082C03D109201A49087201E01848047256
:109550001748007A012809D1012C01D0022C03D12F
:1095600001201349087201E0114804721048007A82
:10957000012816D00E48007A092812D00C4804722F
:109580000FE000200A4948800B480088401C0A4927
:10959000088008460088052803D300200880044876
:1095A0004472FEBD541A0020481A002038070020DB
:1095B0003C1A00203607002066070020012803D14E
:1095C0004A1E0B4B1A8312E0022803D14A1E084B95
:1095D0005A830CE0042804D14A1E054BE0331A8359
:1095E00005E0082803D14A1E014BE0335A83704737
:1095F000602A044008B50D49C97C009100210B4A3E
:10960000D174012806D11146C97804221143074AB2
:10961000D17003E00549C978044AD1700349C9787B
:1096200001221143014AD17008BD0000602A0440A4
:1096300008B50948C078042108430749C87008469E
:10964000C078FE2108400449C8700846C07C0090DC
:109650000020C87408BD0000602A0440012803D11E
:109660004A1E0B4B1A8112E0022803D14A1E084BF6
:109670005A810CE0042804D14A1E054BC0339A835A
:1096800005E0082803D14A1E014BC033DA83704736
:10969000802A044008B51049C978009100210E4A7B
:1096A000D170012808D10C492039C978082211430A
:1096B000094A203AD17005E007492039C978064A9D
:1096C000203AD17004492039C97802221143024A54
:1096D000203AD17008BD0000802A044008B50A482D
:1096E000C078082108430849C8700846C078FD21A1
:1096F00008400549C87004482030C0780090002018
:1097000001492031C87008BD602A04400648C0786D
:10971000FE2108400449C8700846C078FD21084071
:109720000149C87070470000602A044010B5044623
:1097300001211020F1F74CFD207800F09FFB2078EC
:1097400000280CD1FE48C078FE210840FC49C870B2
:109750000846C07804210843F949C8700FE0F8486A
:10976000C0782278012191408843F549C8700846A5
:10977000C0782278042191400843F149C870A0784C
:1097800005280AD1E078052807D0EE4880680078DF
:1097900040210843EB4989680870E07800287DD1B2
:1097A000A07D2178490088400001E17C22785200A8
:1097B000914009010843E349096809780843E149F0
:1097C0000968087020788100DE48443040580078ED
:1097D000217B084321788A00DA494431895808708E
:1097E0003820005DA178084321788A00D5491831D6
:1097F000895808706078C007C00F00281DD02078F5
:109800008100D048203040580078617B0422114309
:10981000084321788A00CB49203189580870207884
:109820008100C848443040580178A07B014320782B
:109830008200C4484430805801706078022108409A
:1098400002281ED120788100BE4820304058007880
:10985000E17B40221143084321788A00B949203135
:109860008958087020788100B64844304058017803
:10987000207C4000014320788200B2484430805868
:109880000170607804210840042820D120788100EC
:10989000AC48283040580078E17B00E03BE00C22E7
:1098A0001143084321788A00A64928318958087055
:1098B00020788100A348443040580178A07C800083
:1098C0000143207882009F484430805801706078BE
:1098D0000821084008281ED12078810099482830A6
:1098E00040580078E17BC0221143084321788A0068
:1098F0009449283189580870207881009148443073
:1099000040580178607DC0000143207882008D4876
:10991000443080580170E07801287DD18948006882
:1099200000788849096808702078810085482830C7
:1099300040580078002120788200824828308058E2
:1099400001703820005DA178084321788A007D49A4
:109950001831895808707A48C07900207849C87150
:109960006078C007C00F00281BD0207881007548A0
:10997000203040580078E17D084321788A00714901
:10998000203189580870A088401E6E49496D0880B2
:109990006B48C07921788A000021914008436849CA
:1099A000C87160780221084002281DD1207881000A
:1099B0006448203040580078617E09010843C1B2F4
:1099C000207882005F48203080580170E088401E77
:1099D0005C49896D08805A48C07921788A00002145
:1099E000914008435649C871607804210840042812
:1099F0003BD1207881005348283040580078E17EE0
:109A0000084321788A004F492831895808702089F5
:109A1000401E4C49C96D00E05AE008804848C079B2
:109A200021788A000021914008434549C871607F30
:109A300001280CD120788100424828304058007815
:109A400021788A003F492831895808700DE0207834
:109A500081003C482830405800780821084321788C
:109A60008A003849283189580870607808210840F0
:109A700008283CD1207881003248283040580078AE
:109A8000A17F09010843C1B2207882002D48283007
:109A9000805801706089401E2A49096E0880284854
:109AA000C07921788A000021914008432449C87177
:109AB0002020005D01280CD1207881002148283029
:109AC0004058007821788A001E492831895808704A
:109AD0000DE0207881001B48283040580078802114
:109AE000084321788A001749283189580870E0789E
:109AF000022802D0E07803287ED11248006800785E
:109B00001049096808703820005DA1780843217861
:109B10008A000C49183189580870A088401E0949EC
:109B2000496D088060780221084002283CD16078A5
:109B3000217889008840034949680978084303E08F
:109B4000602A044004160020CA4949680870E08869
:109B5000401EC849896D08806078C043217889001B
:109B60008840C449C96C09780840C249C96C08706A
:109B700020788100BF483830405801782420005DAB
:109B8000014320788200BB48383080580170232080
